S00A000047572E737265637C
S214400000A55AA55A0100000000000000001040005C
S21440100000F0422021144400854B4500874B4500A4
S214401010894B45008B4B45008D4B4500000000003A
S2144010200000000000000000000000008F4B45005C
S214401030C34B450000000000C54B4500C74B45006C
S21444010047573334342056302E322E352032303250
S214440110332E31312E362031323A30300A0D00003B
S20C4401803412AA5500000000E9
S214440200A55AA55A01000000000000000010440052
S2144402100000000000104400000000000000000041
S2144402200000000000000000000000000000000085
S2144402300000000000000000000000000000000075
S2144402400000000000000000000000000000000065
S2144402500000000000000000000000000000000055
S21444100000F0422021144400854B4500874B4500A0
S214441010894B45008B4B45008D4B45000000000036
S2144410200000000000000000000000008F4B450058
S214441030C34B450000000000C54B4500C74B450068
S214441040C94B4500C94B4500C94B4500C94B4500F3
S214441050C94B4500C94B4500C94B4500C94B4500E3
S214441060C94B4500C94B4500C94B4500C94B4500D3
S214441070C94B4500C94B4500C94B4500C94B4500C3
S214441400C94B4500C94B450000BF00BF00BF00BFE5
S214441410FFF7FABF000000000000000000000000D4
S21444142072B64FF000004FF000014FF000024FF04C
S21444143000034FF000044FF000054FF000064FF055
S21444144000074F4801684FF0807201EA0201002904
S2144414501CD14C4801684FF0807241EA0201016099
S214441460494801684FF0010241EA020101604748D9
S21444147045F6F02101604AF20F5101604048016888
S2144414804FF0807201EA02010029F7D040484149F2
S2144414900160414801684FF00000814200D003E0FB
S2144414A03E4880F3088803E03D4880F3088822E0FD
S2144414B03C484CF2205101604DF6281101603A48F0
S2144414C03A4901600AE03A484CF2205101604DF630
S2144414D028110160374835490160FFE7364800283F
S2144414E009D03649364A521A013A04DD0020002310
S2144414F009C1083AFCDA3348002810D03249086853
S2144415004FF0010240EA020008603049304A521A5D
S214441510013A04DD0020002309C1083AFCDA2D48CC
S214441520002810D02C4908684FF0010240EA020017
S21444153008602A492A4A521A013A04DD0020002348
S21444154009C1083AFCDA274800684FF05A31884205
S214441550F9D0114801684FF00000814200D001E004
S21444156013F034FB13F05EFB62B613F059FB00F045
S2144415703BF800BFFEE700BFAFF30080AFF3008048
S21444158010C32D4030C32D4004C32D4000C02D4011
S21444159008ED00E0001043200400264000F04220FE
S2144415A0000043201000274000002740400000FF72
S2144415B010C0464000C046400100000000004020E5
S2144415C0004044200100000094EF00E000000020AA
S2144415D0000001200100000090EF00E00000000041
S2144415E000800000C42440202DE9F04F87B05B4CB7
S2144415F001F034FC5A4815F037F85A494E20002575
S21444160025F0E2F958481CF0BFF958481CF0E0F9B8
S21444161001F097FB4CF24453E05800F017F901F000
S214441620D3FD00F03BFA00F017FA00F095F9504964
S21444163000201FF025FB4F4900201FF037FB0021F8
S21444164008461FF0DDFB002144F6206208461FF0E2
S21444165093FB2846013501F031FF062DF9D101F000
S2144416606DFB4CF23853444D4FF47A7054F8038073
S214441670E75805F1040BE25854F803900592E258F3
S2144416800292E2580392E2580492E25854F803A0B5
S214441690E6582C46019201F018FB08F0EBF8374860
S2144416A001F044FC00F0B4F82A6806F57A739A42CE
S2144416B002D32E6808F0CDF822680AF1C8039A428D
S2144416C003D3D4F800A008F0BDF8019B2268643325
S2144416D09A4203D32368019308F0A1F8049B226836
S2144416E032339A4201D323680493039B226814330B
S2144416F09A4203D32368039303F0ABFB029B22680E
S2144417000A339A4203D32368029308F04CF82268BB
S21444171009F105039A4203D3D4F8009007F0C1FFB9
S214441720059B226802339A4203D32368059300F04C
S21444173070F822687B1C9A4200D32768DBF80020A6
S21444174008F101039A4203D3DBF8008008F056F808
S21444175008F096F80CF000FDA6E700BF0C394120CF
S214441760D0844600E803402014924600448D460048
S214441770741740206817402044FE4120347B4600BE
S214441780024B586800F00300704700BF0000264034
S214441790024600F03F00931010B583EA5203540803
S2144417A0534084EA121483EA121384EAD2049B0157
S2144417B084EA521403F0400314F0010F43EA000392
S2144417C00CBF80240024234319B99A4218BFFF2033
S2144417D010BD01290CBF1846FF20F9E73C2A0CD05F
S2144417E07D2A0AD0FE2A08D0BF2A06D092B20144E7
S2144417F0814204D1D043C0B270470022F7E710F8C4
S214441800013B1A4492B2FF2A84BFFF3A92B2EFE7F2
S21444181070470AF031BD704710B5074C002001F000
S214441820B7F92080012001F0B3F9044B22881880D0
S214441830034B1A8010BD00BF2218402020184020B9
S214441840CC1740207047704770477047002110B54A
S2144418500446084618F0C2F80121002018F0BEF8E5
S2144418600221002018F0BAF80321002018F0B6F838
S214441870002017F0AFFF0E49002017F0C1FE0D4BB5
S214441880A2B20020197817F0F9FF0B49002018F08F
S2144418906BFB0A49002018F067FB0949002018F042
S2144418A063FB08490020BDE8104018F05DBB00BF4C
S2144418B08C894600C4894600148B4600F48A460048
S2144418C0D48A4600B48A4600F8B50D4606461F49F3
S2144418D028461F4F0DF090FE044670B14CF2445318
S2144418E0F85806F54553123307EB83077D60032EFD
S2144418F02BD8DFE806F01A212427002128460DF0CD
S21444190071FE80B94CF24453F8580DF06BFC2946EE
S2144419100DF0C0FC0DF010F800220E4B0DF08EF9C1
S2144419200DF03AFBDDE72046DBE782B200210020DB
S214441930BDE8F84018F062BD82B20121F7E782B2F2
S2144419400221F4E782B20321F1E7F8BD0000C84261
S2144419500C3941200000594008B503481DF006FAEA
S214441960024B187008BD00BF0C9546008C474020BB
S214441970F7B50123104C114D6370A21CEB68A91CEB
S2144419800F480235009335F8023C1DF091F80022CA
S2144419902073A01C6178134615F8017B013310F8B8
S2144419A0016BDBB2B7421CBF012200210A2BF3D1E4
S2144419B002B1617003B0F0BD8C474020801F4020C8
S2144419C0209546004B7C062B0AD10122054B1A74FF
S2144419D0CA7B1A2A04D1032203F111011DF0A8BBC5
S2144419E0704700BF801F40204B7C062B0AD1012243
S2144419F0054B1A74CA7B2A2A04D1032203F1110127
S214441A001DF096BB704700BF801F40201FB50023C3
S214441A101A210446039301238DF807301DF0CEFCAB
S214441A200B4B03930B4B1A7C002AFCD01B7C63B1F4
S214441A3002A920461DF0C6FB8DF80700039B5A1EDC
S214441A40039213B19DF80730F1E704B010BD00BF10
S214441A50006A1800801F402008B5A1201BF0DAFF5A
S214441A6000220A49A1201BF0D4FF094B094902224F
S214441A700120C3F8F413C3F8982DC3F8F813C3F839
S214441A80902D0549BDE808401CF0C4BC0BE8450051
S214441A9000002940040028008094460008B5A2208F
S214441AA01BF0B8FF00220B49A2201BF0B2FF0A4BE2
S214441AB00A4A01210020C3F8E023C3F8AC1DC3F84A
S214441AC0E42302220649C3F8A42DBDE808401CF0CE
S214441AD0E1B900BF11E84500000029400200280093
S214441AE0A494460010B50822174901204FF48034C8
S214441AF01CF04CFD01230822144900201CF0B6FAC1
S214441B00002108461CF000FC022801D1013CF7D114
S214441B104FF48034002101201CF042FD022801D1FC
S214441B20013CF7D1094A0823A2F1080012F8011B28
S214441B30013B10F8014BA14204BF013102F8011CDD
S214441B4013F0FF03F2D110BD941F40209C1F402089
S214441B5082B00190019B5A1E0192002BFAD102B02A
S214441B607047044B4FF400224FF4FA70C3F8C02277
S214441B70FFF7EEBF00002940044B4FF420124FF409
S214441B80FA70C3F8C022FFF7E3BF00BF0000294045
S214441B902DE9F04104460D46104600293ED1DFF8B3
S214441BA0908050260B46C1B2564308F1100728468B
S214441BB0BA19B04419F032FC1C484FF4FB534FF4A6
S214441BC0FB62D8F81410083603FB04033744D3F8F2
S214441BD0FC3802FB043203F17A0602F5107C02F567
S214441BE0427240F82C1098F8581040F82210FB2205
S214441BF012FB046200EB4212A94211D84FF4FB5286
S214441C000133642102FB0404B3FBF1F201FB1233FB
S214441C10C4F8FC3804F5215401232360BDE8F08160
S214441C2017F8016B013502F8016BE5E70C394120E2
S214441C308C4740202DE9F04104460D4610460029C5
S214441C403ED1DFF8908050260B46C1B2564308F585
S214441C50F2670120BA19B04419F0E0FB1C484FF46F
S214441C60FB534FF4FB62D8F89417083603FB04037F
S214441C703744D3F8FC3802FB043203F17A0602F503
S214441C80107C02F5427240F82C1098F8D81740F8A9
S214441C902210FB2212FB046200EB4212A94211D826
S214441CA04FF4FB520133642102FB0404B3FBF1F20C
S214441CB001FB1233C4F8FC3804F521540123236095
S214441CC0BDE8F08117F8016B013502F8016BE5E7D2
S214441CD00C3941208C4740202DE9F04104460D46FE
S214441CE0104600293ED1DFF8908050260B46C1B2FC
S214441CF0564308F571670220BA19B04419F08EFBB2
S214441D001C484FF4FB534FF4FB62D8F8141F0836B4
S214441D1003FB04033744D3F8FC3802FB043203F1D4
S214441D207A0602F5107C02F5427240F82C1098F8B8
S214441D30581F40F82210FB2212FB046200EB4212AA
S214441D40A94211D84FF4FB520133642102FB040428
S214441D50B3FBF1F201FB1233C4F8FC3804F521540A
S214441D6001232360BDE8F08117F8016B013502F8C2
S214441D70016BE5E70C3941208C4740202DE9F041C2
S214441D8004460D46104600293ED1DFF89080502682
S214441D900B46C1B2564308F5B3670320BA19B0449C
S214441DA019F03CFB1C484FF4FB534FF4FB62D8F845
S214441DB09C15083603FB04033744D3F8FC3802FB6F
S214441DC0043203F17A0602F5107C02F5427240F8BA
S214441DD02C1098F8E01540F82210FB2212FB0462FF
S214441DE000EB4212A94211D84FF4FB52013364214E
S214441DF002FB0404B3FBF1F201FB1233C4F8FC38D3
S214441E0004F5215401232360BDE8F08117F8016BE3
S214441E10013502F8016BE5E70C394120845840202F
S214441E202DE9F04104460D46104600293ED1DFF820
S214441E30908050260B46C1B2564308F618570420E5
S214441E40BA19B04419F0EAFA1C484FF4FB534FF45D
S214441E50FB62D8F81C1D083603FB04033744D3F84A
S214441E60FC3802FB043203F17A0602F5107C02F5D4
S214441E70427240F82C1098F8601D40F82210FB225D
S214441E8012FB046200EB4212A94211D84FF4FB52F3
S214441E900133642102FB0404B3FBF1F201FB123369
S214441EA0C4F8FC3804F5215401232360BDE8F081CE
S214441EB017F8016B013502F8016BE5E70C39412050
S214441EC0845840202DE9F04104460D46104600292A
S214441ED03ED1DFF8908050260B46C1B2564308F5F3
S214441EE068770520BA19B04419F098FA1C484FF49C
S214441EF0FB534FF4FB62D8F8A413083603FB0403E1
S214441F003744D3F8FC3802FB043203F17A0602F570
S214441F10107C02F5427240F82C1098F8E81340F80A
S214441F202210FB2212FB046200EB4212A94211D893
S214441F304FF4FB520133642102FB0404B3FBF1F279
S214441F4001FB1233C4F8FC3804F521540123236002
S214441F50BDE8F08117F8016B013502F8016BE5E73F
S214441F600C3941207C6940204FF4FB52054B02FB60
S214441F700033D3F8F808D3F8FC38C31A584258410B
S214441F80704700BF0C3941202DE9F74FCC4D002156
S214441F90CC4E4FF4FB692C4641F6987837464FF0C2
S214441FA0640A0846FFF7E0FF50BBD6F8F83809FB4A
S214441FB0013202F5427257F822C008FB01420092F1
S214441FC04FF4FB524A4302EB43123A44019200F167
S214441FD0010EC0B2844534D809FB0132013385F87A
S214441FE020C002F5107257F822206A624FF00102B0
S214441FF085F82120B3FBFAF20AFB1233C6F8F83808
S2144420000131454406F5FB560629CAD194F82130D9
S214442010012B2DD1002384F82130636AB3F5BE7FAB
S21444202000F0E18000F29480452B14D83F2B1FD952
S214442030413B042B00F2CB80DFE803F0CCDEE1E446
S214442040E700019A02EB000B009A9BF840BF02F8A7
S21444205000B07046BBE7B3F5BA7F00F0BE80B3F578
S214442060BC7F00F0BD8040F25512934200F0BE8023
S21444207041F6B973E25C012A0FD10022E25441F6DC
S214442080BC73E358932B00F0D08000F2C180912BB0
S21444209000F0C580922B00F0C58043F65173E25C95
S2144420A0012A14D10022E25443F65473E358962B83
S2144420B000F0E38000F2C480822B00F0DB8000F264
S2144420C0B780722B00F0DF80732B00F0DF8045F67C
S2144420D0E963E25C012A14D10022E25445F6EC633B
S2144420E0E3589B2B00F0F88000F2DE808D2B00F046
S2144420F0028100F2D180722B00F0F780732B00F03F
S214442100F78047F68163E25C012A0BD10022E25451
S21444211047F68463E358722B00F0F380732B01D1A7
S21444212002F06AFD49F61963E25C012A40F0F18048
S2144421300022E25449F61C63E358722B00F0E48014
S214442140732B40F0E68003B0BDE8F04F02F084BD48
S214442150B3F5B06F2FD016D840F20132934233D045
S2144421600AD840F22122934243D0B3F5407F7FF40D
S2144421707FAF01F09DFD7BE7B3F5AE6F7FF478AF9C
S21444218001F0C2FD74E740F29552934216D00AD845
S21444219040F28552934214D0B3F5B26F7FF468AFE1
S2144421A001F074FE64E740F2777293427FF460AFC6
S2144421B001F096FE5CE701F0F7FD59E701F078FE82
S2144421C056E701F03BFE53E701F092FD50E701F07D
S2144421D016FC4DE701F026FC4AE701F0A7FC47E76A
S2144421E001F0C6FC44E701F0E5FC41E701F076FC6B
S2144421F03EE701F0FDFC3BE701F032FC38E701F036
S2144422003BFC35E701F048FC32E701F055FC2FE78C
S214442210B3F5A87F7FF441AF01F0CAFE3DE701F075
S21444222071FE3AE701F094FE37E701F0A3FE34E787
S2144422308C2B25D0922B7FF44AAF02F01BF846E74E
S214442240AA2B26D007D89A2B0ED0A02B7FF43FAFCC
S21444225002F030F93BE7C82B09D0B3F5F36F7FF4AF
S21444226036AF02F0F1F932E702F0E4F82FE702F075
S214442270ADF92CE701F06CFF29E702F083F826E776
S21444228001F090FF23E701F0E9FE20E701F02EFF7E
S2144422901DE702F05BF91AE7932B2FD0972B7FF4B8
S2144422A030AF02F0C1FA2CE7C92B18D00CD8A12BBA
S2144422B018D0AA2B7FF425AF02F086FB21E700BF97
S2144422C0087840200C39412040F2997293427FF4BA
S2144422D018AF02F05FFC14E702F0FEFA11E702F0D2
S2144422E0B3FB0EE702F038FB0BE702F0C1F908E750
S2144422F002F006FA05E702F0E5FB02E702F032FADE
S214442300FFE602F05BFC0DE703B0BDE8F04F02F0D9
S21444231085BC03B0BDE8F08FEC4BED489A6D596F21
S21444232002F07042DFF8CCC301F07F412DE9F0475C
S214442330E84F4FF000089A654FF00009DA6D596788
S2144423403A40996FE44EDA6501401A6E996702F096
S2144423500042996C5C691A6601F06041B3F86420E7
S21444236041F4C821DFF890E33240DFF890A3996443
S214442370A3F86420B3F86820D8493240A3F868200C
S2144423800022C3E90212D64983F86F2021405C6CD0
S2144423901A675961596A5A6539405962196C01F08D
S2144423A000411964CF490C405C64CF4CC3E91342E6
S2144423B0D3F88040D3F8985004F07F4483F88C20B8
S2144423C0C3F8D4E0C3F88040D3F8844004F07F4494
S2144423D0C3E92142B3F8904004EA0C04A3F89040C1
S2144423E0D3F8904062F35034C3F89040D3F8944006
S2144423F004F07C44C3F89440BC4C2540C3F8985041
S214442400D3F8D85005F04045C3F8D850D3F8DC503C
S21444241005F07845C3E9375293F8E45062F3000573
S21444242083F8E450D3F8AC5005F04045C3F8AC50BC
S214442430B3F8B05062F30D05A3F8B050D3F8C050CB
S21444244005F00045C3F8C050B3F8C4503540A3F86F
S214442450C450D3F8C45025F47F15C3F8C450D3F8F9
S214442460C850C3F838E105F07045C3F8C850D3F8EF
S214442470CC5005F07F45C3F8CC50B3F8D05005EAAD
S2144424800A05A3F8D050D3F8B45005F04045C3E944
S2144424902D5293F8BC5025F0030583F8BC50D3F86E
S2144424A09C5005F04045C3F89C50D3F8A0500D40CE
S2144424B0C3E92852D3F8A8500540C3F8A850D3F827
S2144424C0E85005F07E4545F48035C3F8E850D3F827
S2144424D0EC500D40C3F8EC50D3F83C512540C3F8BB
S2144424E03C51D3F8405105F07845C3F84051B3F811
S2144424F0445105F47845C3E94022C3E93E89A3F82C
S2144425004451D3F8485183F8542105F07E45C3F826
S2144425101C21A3F8282145F48035C3F84851D3F844
S2144425204C510D40C3F84C51D3F8505105F060451A
S214442530C3F85051D3F82C5105F07045C3F82C51CC
S214442540D3F8305105F07F45C3F83051B3F83451D1
S21444255005EA0A0AD3F8085105F04045A3F834A121
S214442560C3F80851D3F80C512940614DC3E94312CE
S214442570D3F814110140C3F81411D3F8181101F01C
S2144425807C41C3F81811090E21F03C0183F81B1155
S21444259093F8201121F0030183F82011D3F8241175
S2144425A001F06041C3F82411D3F868113940C3E9F7
S2144425B05689C3F86811A3F86C21D3F87011A3F8B0
S2144425C074210F40D3F8C811C3F8B02101F07C4100
S2144425D083F8B421C3F8B821C3F8C811D3F8CC1192
S2144425E083F8BC212140C3F8C02183F8C421C3F832
S2144425F0CC11D3F8D411C3F8782101F0004183F804
S2144426008021C3F8A021C3F87071C3E97512D3F8CA
S2144426107C1101F07F41C3F87C11D3F88411294022
S214442620C3E9611293F88C1121F00F01C3E97822B3
S21444263083F88C11C3E96422C3E96622A3F8A42173
S21444264093F80812C3F8A82162F30101A3F8AC2159
S21444265083F80C2283F80812D3F80812C3F8182219
S21444266021F07F6183F83022C3F8342221F47F219D
S21444267083F83822C3F83C2221F47F6183F8402251
S214442680C3F8442221F00C0183F84822C3F84C22B4
S214442690C3F80812D3F8101283F85A2201F0004106
S2144426A0C3F81012B3F814120E40D3F81C1201F0FB
S2144426B07F41A3F81462C3F81C12D3F820120140D9
S2144426C0C3F82012D3F828121AE000BFA0744020A2
S2144426D00000FCFF0000F0FF00C0FFFF0000E281A6
S2144426E000F807F8000080FF0080204E0000C0FF7E
S2144426F00000FEFF00E0FFFF0000C04B00F0FFFFBD
S2144427002140C3E98A12D3F850120C40D3F854122D
S21444271001F07E41C3F85042C3F85412D3F89C12D9
S214442720A3F8CC2201F07E41C3F8D022C3F89C1211
S214442730D3F8A01201F00041C3F8A01293F8A412F3
S21444274021F00F0183F8A412D3F8A81201F07841BF
S214442750C3F8A812D3F8AC1201F07F41C3F8AC1208
S214442760B3F8B01201EA0C01A3F8B012D3F8B412CD
S2144427702940C3F8B412D3F8C81201F00041C3F894
S214442780C81293F8D41262F3000183F8D412D3F833
S214442790D81201F07F41C3F8D812D3F8DC120140B6
S2144427A0C3F8DC12D3F8E01201F04041C3F8E0125B
S2144427B0D3F8E41201F07841C3F8E412D3F8E812EF
S2144427C001F07841C3E9AE89C3E9BA1293F8F0122E
S2144427D0C3F8442362F3000183F8F012D3F8F412EA
S2144427E001F07841C3F8F412D3F8F81201F07F41AF
S2144427F0C3F8F812B3F8FC1201EA0C0CD3F8001331
S21444280001F07E41A3F8FCC2C3F80013D3F80413C6
S2144428102940C3E9C11293F80C1362F3000183F80C
S2144428200C13D3F8101301F07F41C3F81013D3F8F8
S21444283014130840D3F818130D40D3F83013C3F8D4
S214442840140301F04041C3F81853C3F83013D3F8C7
S214442850341301F07841C3F83413D3F8381301F035
S2144428607841C3E9CE1293F8401362F30001C3E9FA
S214442870C88983F8401393F84813C3F8542362F383
S214442880000183F84813D3F84C1301F07F41C3F892
S2144428904C1393F8521321F0030183F8521393F820
S2144428A0581362F3000193F85E2322F0030283F880
S2144428B0581383F85E23BDE8F08741F698730849B9
S2144428C0002258430B182830DA64084483F848201A
S2144428D02023013B00F8012B13F0FF03F9D1704786
S2144428E00878402041F6987310B558430B4C41F68F
S2144428F092732218D35A28225A4300231118503070
S214442900104421441A46204481F870304B67013302
S21444291000F8012BDBB2202BF9D110BD08784020FB
S2144429202DE9F8439946234B0546884603EB0013A6
S2144429309B6A402B31D820494FF4FB5303FB0013CA
S21444294042F644015B5843B341F698761B4C002745
S2144429504FF0280C06FB00F3E11801F5FC5110314A
S214442960F8B248451BD328467543FFF7A6FF41F601
S2144429709071601928260122435A06FB03551344D6
S2144429802C4484F87120C4F8748084F87090C82469
S214442990B3FBF4F204FB12334352BDE8F8830888D1
S2144429A012F807E00CFB003020443844013780F826
S2144429B050E0D5E7801F40200C394120087840205D
S2144429C041F6987241F692732DE9F347444D02FB63
S2144429D000F10446434F6A18D35A282202FB0312D6
S2144429E02A4492F87020082A2FD807EB00120821B0
S2144429F0916241F698764FF0280941F6947A20463B
S214442A00664309FB03F206F1500305EB06089119E9
S214442A101344354A29442B4402EB041200934B6F6B
S214442A2018F80A1018F082FC18F80A300D21013301
S214442A30B3FBF1F201FB123308F80A308246E0B1E8
S214442A4002282FD002B0BDE8F087102A03D807EB3F
S214442A5000121021CCE7182A03D807EB00121821DD
S214442A60C6E7202A03D807EB00122021C0E7402AF5
S214442A70BFD807EB00124021BAE72046FFF732FFE3
S214442A8041F69271C82038F8013009FB03660133D9
S214442A90B3FBF0F2354400FB123385F871A028F8F6
S214442AA00130CFE72046FFF71DFF41F69271002222
S214442AB0C82038F8013009FB03660133354485F8ED
S214442AC07120B3FBF0F200FB123328F80130D7E94B
S214442AD02232013342F10002C7E92232B2E700BF94
S214442AE008784020801F4020A41F4020F8B50024CA
S214442AF00A4D41F698760A4F06FB04F22821E0B2C6
S214442B00D35B01FB03232B4493F87130012B01D193
S214442B10FFF756FF0134062CEED1F8BD0878402066
S214442B209A97402008B50B21034823F095FE034BA3
S214442B3083F8200B08BD00BF021729407C6940205B
S214442B4001290A4628BF0122072819D8DFE800F0E1
S214442B5004070B0D1012141600210A4801E00A213E
S214442B60094823F040BE0C21F7E702210748F8E75E
S214442B700D21F2E70E21F0E70F21EEE70021F5E7FD
S214442B80704700BF021729401017294000172940F4
S214442B9007281AD8DFE800F004070B0E10131517A1
S214442BA008210B4801E00B210A4823F055BE0121B9
S214442BB00948FAE70B21F4E704210848F5E705211C
S214442BC0FBE70821F9E70A21F7E7FF20704700BF33
S214442BD0061729400217294012172940041729408E
S214442BE001284FF002010CBF0022012210B5044612
S214442BF0034823F0F8FD034A4CF24053D45010BD2A
S214442C00081729400C39412005281DD8DFE800F074
S214442C1003080C1014180D4A4CF27453D05A7047DB
S214442C200A4A4CF27653F9E7084A4CF27853F5E7E9
S214442C30064A4CF27A53F1E7044A4CF27C53EDE7E9
S214442C40024A4CF27E53E9E7FF2070470C39412094
S214442C5008B50621002012F046FB024A4CF2745393
S214442C60D05208BD0C39412010B50221012012F083
S214442C703AFB064C4CF276532B21E052012012F0DC
S214442C8032FB4CF27E53E05210BD00BF0C3941205B
S214442C9010B50321022012F026FB094C4CF278535F
S214442CA00421E052022012F01EFB4CF27A53052116
S214442CB0E052022012F017FB4CF27C53E05210BD57
S214442CC00C394120002112F0FBB9084A4CF2385323
S214442CD082B00749D35800930B68009A9B1A019315
S214442CE0019B8342F8D902B0704700BF0C3941209B
S214442CF044FE412038B50F4D0F4C95F890305BB9E3
S214442D0001234CF23C5285F89030A3580133A3502B
S214442D10BDE8384006F072BD09F0D6FF4CF23C528E
S214442D20002385F89030A3580133A3504CF2385210
S214442D30EBE700BF801F40200C3941200020FFF7FE
S214442D404FBF10B58D20244C1AF064FE0022234950
S214442D508D201AF05EFE8F201AF05CFE0022204979
S214442D608F201AF056FE97201AF054FE00221D4972
S214442D7097201AF04EFE9A201AF04CFE00221A496A
S214442D809A201AF046FE194900201DF08BF918497E
S214442D9002201DF087F917490A201DF083F91649C9
S214442DA00D201DF07FF92146012200201DF0FCFB7A
S214442DB004F59671012202201DF0F6FB04F26C51D4
S214442DC001220A201DF0F0FB04F28C5101220D2052
S214442DD0BDE810401DF0E8BB183C4120B10A46004F
S214442DE0B70A4600BD0A4600C30A46000C9646008B
S214442DF0E0954600B49546008895460010B48AB9D6
S214442E000949D1F86C3891F8B848CA18013301F624
S214442E10B801DBB282F8584610BC012241F84C3C5B
S214442E201DF012BD10BC70470C39412010B48AB94D
S214442E300949D1F8743891F8D848CA18013301F6CC
S214442E40D801DBB282F8584710BC012241F8643CF2
S214442E501DF0FABC10BC70470C394120194B0121B7
S214442E6042F644000022195044F2A470195046F227
S214442E700470195048F2646019504AF2C45019500C
S214442E804CF22450195042F648015A5044F2A87164
S214442E905A5046F208715A5048F268615A504AF2FB
S214442EA0C8515A504CF22851C3E9C1225A504CF2E8
S214442EB048524CF2503199504CF244524FF44861C7
S214442EC0995070470C39412010B5064B4FF4FB54CB
S214442ED004FB003042F64803C15042F64C03C2504D
S214442EE010BD00BF0C394120094BD3E9C1218A42A9
S214442EF00BD01A4492F8042202700020D3F804231C
S214442F000132D2B2C3F8042370470120704700BF91
S214442F100C39412007B501220DF107018DF8070051
S214442F2000201DF095F903B05DF804FB0FB470B5AE
S214442F30C2B0002446AA02AE52F8041B30460192A0
S214442F400EF07AFA30460BF039FBC5B2E3B29D4236
S214442F5004D842B0BDE8704004B07047305D0134D8
S214442F60FFF7D8FFF2E708B58E201AF053FD9620F7
S214442F701AF050FD0748FFF7D9FF074900201CF018
S214442F8011F8012005491CF00DF80548BDE8084035
S214442F90FFF7CCBF887946005C95460030954600DE
S214442FA0907946000B2938B5044614D142F64403BA
S214442FB00E4D00220E48EA50FFF7B8FF42F648038B
S214442FC0EB581BB142F64C02A85898472046BDE839
S214442FD0384018F021BF074B1A6832B10022064821
S214442FE01A60BDE83840FFF7A1BF38BD0C39412010
S214442FF0967946004C614120B27946000B2938B593
S21444300005460E4C13D144F2A47300220C48E250F9
S214443010FFF78CFF44F2A873E3581BB144F2AC723A
S214443020A05898472846BDE8384018F0F5BE44F204
S214443030A073E2580AB10022E25038BD0C39412050
S214443040D17946000B2938B5044614D146F20473A8
S2144430500E4D00220E48EA50FFF768FF46F208730A
S214443060EB581BB146F20C72A85898472046BDE868
S214443070384018F0D1BE074B1A6832B100220648D1
S2144430801A60BDE83840FFF751BF38BD0C394120BF
S214443090ED7946000CA04120097A46000B2938B544
S2144430A004464FF4FB55134815D105FB040542F678
S2144430B0440300221048EA50FFF738FF42F648031C
S2144430C0EB581BB142F64C02A85898472046BDE838
S2144430D0384018F0A1BE05FB040404F521542368C7
S2144430E033B1002305482360BDE83840FFF71EBFD0
S2144430F038BD00BF0C394120277A4600437A460043
S2144431000B2938B504464FF4FB55134815D105FB37
S214443110040542F6440300221048EA50FFF706FF2F
S21444312042F64803EB581BB142F64C02A85898475F
S2144431302046BDE8384018F06FBE05FB040404F58D
S2144431402154236833B1002305482360BDE8384042
S214443150FFF7ECBE38BD00BF0C394120627A46000A
S2144431607E7A46000B2938B504464FF4FB5513487F
S21444317015D105FB040542F6440300221048EA50E4
S214443180FFF7D4FE42F64803EB581BB142F64C0216
S214443190A85898472046BDE8384018F03DBE05FB81
S2144431A0040404F52154236833B1002305482360FE
S2144431B0BDE83840FFF7BABE38BD00BF0C394120E1
S2144431C09D7A4600B97A460038B50A243C4D2946CD
S2144431D0002012F099FC38B1013C14F0FF04F6D1FB
S2144431E021463848FFF7A2FE0A24374D29460120D7
S2144431F012F08AFC38B1013C14F0FF04F6D10121E8
S2144432003048FFF793FE0A24304D2946022012F038
S2144432107BFC38B1013C14F0FF04F6D10221294866
S214443220FFF784FE00222A49B4200A241AF0F1FB50
S21444323000222849B5201AF0ECFB00222649B62085
S2144432401AF0E7FBB4201AF0E5FBB5201AF0E2FBCF
S214443250B6201AF0DFFB002012F0ECF838B1013C3F
S21444326014F0FF04F7D121461C48FFF75FFE0A24FA
S214443270012012F0DFF838B1013C14F0FF04F7D116
S21444328001211648FFF752FE0A24022012F0D2F813
S21444329038B1013C14F0FF04F7D102210F48FFF780
S2144432A045FE0121002012F047F90121084612F09C
S2144432B043F901210220BDE8384012F03DB900BF71
S2144432C0F8884600F47A46009C88460040884600C3
S2144432D0E5604500EB604500F1604500D87A46005D
S2144432E038B51C4C0546206804302044FFF7FCFDE6
S2144432F0012801D1012038BD2368E21810790A2834
S21444330010D00D280ED0082815D123B1013B124801
S2144433102360FFF70BFE2368AB42EBD32544002023
S214443320E87006E00D48FFF701FE236800202344BA
S21444333018712060DFE7A0F120035E2BEBD8FFF77F
S214443340E9FD2368E11801330A792360303A81F8AD
S2144433500421E0E70C394120097B4600187B4600EF
S21444336010B58020FFF7BCFF90B90A4C23797BB197
S2144433700949201D0BF018F920B90848BDE810404B
S214443380FFF7D4BD211D0648BDE81040FFF7CEBD6B
S21444339010BD00BF0C3941200D7B4600137B460010
S2144433A01B7B46002DE9F04F082389B00024924643
S2144433B03B4A054689464FF064081068EDB25168AA
S2144433C002AF012622468DF810408DF81C40DFF8E7
S2144433D0E8B0CDE905346B4403C35146484623F070
S2144433E002FA04AA214640F255532846CDF80480F2
S2144433F000978DF81C608DF81040059418F0FAFB81
S214443400284B04AA2146284602934FF607738DF8A4
S2144434101060ADF80C300623CDE9007805935B4682
S21444342018F0E8FB204A0623214602924FF6FF7224
S214443430059328465B46ADF80C2004AA8DF8106028
S214443440CDE9007818F0D6FB184A062321460292A6
S214443450284604AA05935B46ADF80C408DF81060E8
S214443460CDE9007818F0C6FB114B124A214628468F
S2144434708DF81060CDE90232082304AA05935B4612
S214443480CDE9007818F0B6FB0A20FFF71EFC32465A
S2144434905146484623F0A7F909B0BDE8F08F00BF6F
S2144434A0446F46001000500010019FFF1002C000F9
S2144434B07102030405060708F100DA182DE9F04105
S2144434C00446002855D16D201AF0A4FA2246C04975
S2144434D06D201AF09EFA6E201AF09CFA2246BD49D8
S2144434E06E201AF096FA01220821BB4823F07BF995
S2144434F001220521B84823F076F9B84AB84920464F
S21444350017F00AFE0121204618F0C8FD22460D2178
S214443510204618F01FFC204618F09EFD2346B14A6C
S2144435200D21204617F036FF2346AF4A0D2120468C
S21444353017F074FFFEF7F0FE2046FFF7BEF9AB4BDC
S214443540012242F644015A5003F521531A6041F6CB
S21444355098700023A64A4443A648A35004441A46F7
S214443560013384F871202834C82BF9D10020BDE8F3
S214443570F081012846D0022840F0898074209E4F6E
S2144435801AF048FA00229D4974201AF042FA75202F
S2144435901AF040FA00229A4975201AF03AFA0122A3
S2144435A00421984823F01FF901220621964823F067
S2144435B01AF90025954A20469549DFF8B88217F04F
S2144435C0ABFD204618F048FD05F10D0658F8353099
S2144435D0904A0220F6B223F060430135314617F094
S2144435E0D9FE3A46002331460220503717F016FFDC
S2144435F00B2DE9D17D4B012246F204715A5003F556
S214443600CE43A3E77120844F1AF004FA002283497C
S21444361071201AF0FEF972201AF0FCF90022804953
S21444362072201AF0F6F922460721774823F0DBF891
S21444363022460221734823F0D6F80025794A2046CC
S2144436407949DFF8348217F067FD204618F004FD08
S21444365005F10D0658F83530744A0120F6B223F0C9
S21444366060430135314617F095FE3A46002331460D
S2144436700120503717F0D2FE042DE9D144F2A4714C
S2144436805A4B01225A5044F2A0715A505FE703281D
S21444369059D0042800F0F48005287FF458AF7B20E6
S2144436A0634D1AF0B7F9002262497B201AF0B1F94B
S2144436B07C201AF0AFF900225F497C201AF0A9F961
S2144436C001220E21504823F08EF801225B48114611
S2144436D023F089F85A4A5B49204617F01DFD2046D8
S2144436E018F0BAFC012255492046FFF75BFE564ABD
S2144436F05449204617F010FD204618F0ADFC2B68C0
S214443700524A0D2123F06043204617F043FE00231F
S2144437104F4A0D21204617F081FEAB684B4A0E21D6
S21444372023F06043204617F035FE0023494A0E2115
S214443730204617F073FE4CF224512C4B01225A506B
S2144437404CF22051A1E77720434F1AF063F9002248
S214443750424977201AF05DF978201AF05BF9002286
S2144437603F4978201AF055F9012200213D4823F0BC
S2144437703AF801223B4800251146DFF8008123F041
S21444378032F8394A3949204617F0C6FC204618F024
S21444379063FC05F10D0658F83530354A0320F6B279
S2144437A023F060430135314617F0F4FD3A460023D2
S2144437B031460320503717F031FE0A2DE9D148F23E
S2144437C064610A4B01225A5048F260615DE700BFCB
S2144437D015D845001BD8450008172940EC8C4600F0
S2144437E05841402014204020AC4B40200C39412006
S2144437F09897402008784020AC5A40205DD8450031
S21444380063D845000E1729400C1729403C8C4600C7
S21444381008384020342040202C5340203FD84500D0
S21444382045D84500948C4600B03C40202420402097
S214443830547246009FD84500A5D845001017294025
S2144438404C6F4600102A4020348B460064204020AB
S2144438502C7140207C7140202C6240207BD845004F
S21444386081D8450006172940E48B46006033402043
S21444387044204020C47246001C73460074724600BE
S2144438807920294D1AF0C6F80022284979201AF0E2
S214443890C0F87A201AF0BEF8002225497A201AF099
S2144438A0B8F801220A21234822F09DFF012209216B
S2144438B0204822F098FF204A2049204617F02CFC46
S2144438C0204618F0C9FB09221A492046FFF76AFD2C
S2144438D01B4A1A49204617F01FFC204618F0BCFB2A
S2144438E02B68184A0D2123F06043204617F052FDFA
S2144438F00023154A0D21204617F090FDAB68114A67
S2144439000E2123F06043204617F044FD00230F4A5F
S2144439100E21204617F082FD4AF2C4510C4B012278
S2144439205A504AF2C051B0E6647246008DD84500FB
S21444393093D84500081729404C6F4600B82E4020BF
S2144439408C8B460054204020AC694020FC694020C3
S2144439500C39412041F69872084B02FB003310B5EF
S21444396003EB8104E278A07800EB0220627802EB55
S214443970002213F8210000EB022010BD08784020F6
S21444398010B5094B41F6987404FB0030130A00EB5B
S214443990810181F8282081F82930130C120E81F811
S2144439A02A3081F82B2010BD0878402013B502AB8E
S2144439B0044603E9060041F69871094A9DF8043026
S2144439C001FB0022009903F03F0321F06041FEF71B
S2144439D0A7FF204602B0BDE81040FEF76EBF00BF0A
S2144439E030784020FDF730BF7047704770477047C7
S2144439F07047704770477047704770477047074B2B
S214443A00074A196858799160197941EA00219181E9
S214443A109979DB799173D373704700BF0878402057
S214443A20A07440200C4A0D4810B55178137801F024
S214443A300104C1F3410143EA042343EA4123917854
S214443A40D27843EAC12343EAC243426902F0784249
S214443A501343436110BD00BF08784020A074402043
S214443A60034B04491A7C097861F300021A747047C0
S214443A70A0744020087840200549064B0A7E1B78EF
S214443A8022F01F0203F01F0313430B76704700BF58
S214443A90A0744020087840200549064B0A7F1B78CE
S214443AA022F01F0203F01F0313430B77704700BF37
S214443AB0A0744020087840200649074B91F82020FF
S214443AC01B7822F00F0203F00F03134381F82030D3
S214443AD0704700BFA074402008784020114B12481D
S214443AE010B55A78997802F003041B7843EA042305
S214443AF0C2F3810443EA8423C2F30114920943EADD
S214443B00043343EA823301F00302C1F3810143EAFA
S214443B100243426A120D43EA814312051343436249
S214443B2010BD00BF08784020A07440200E4B0F4ABA
S214443B305878197841EA002158791185997801F026
S214443B400F0182F82A10D97882F82B10197941EAA5
S214443B50002191859979DB7901F00F0182F82F30A5
S214443B6082F82E10704700BF08784020A07440208A
S214443B700E4B0F4A5878197841EA00215879118635
S214443B80997801F00F0182F83210D97882F8331010
S214443B90197941EA002191869979DB7901F00F0180
S214443BA082F8373082F83610704700BF08784020D5
S214443BB0A07440200C4B0D4A5878197841EA0021ED
S214443BC058791187997801F00F0182F83A101979DB
S214443BD041EA002191879979DB7901F00F0182F857
S214443BE03F3082F83E10704708784020A07440204A
S214443BF02D492E4A10B50B78487803F07F0343EAE4
S214443C00C013887843EAC033C87843EAC053106C7C
S214443C1000F00040034348791364C0F340040B7932
S214443C20897982F8443000F001031B0243EA4423B6
S214443C30C0F3800443EA8423C0F3C00443EAC423A5
S214443C40C0F3001443EA0433C0F3401443EA443355
S214443C50C0F38014C00943EA843343EAC03301F016
S214443C60010043EA0043C1F3400043EA4043C1F342
S214443C70800043EA8043C1F3C00043EAC043C1F333
S214443C80001043EA0053C1F34010C1F3801143EAE5
S214443C90405343EA8153516C21F4FF0121F4FE4121
S214443CA00B43536410BD00BF08784020A0744020E6
S214443CB00D4A0E4810B55178137801F00F04C1F33D
S214443CC0001143EA042343EA0133917843EA41333B
S214443CD0D17843EA4153816C01F060410B438364DD
S214443CE05368C36410BD00BF08784020A0744020C9
S214443CF0034A044B1168526819655A65704700BFF9
S214443D0008784020A0744020244A254970B5557848
S214443D10137805F003069078D47843EA0623C5F36F
S214443D20810643EA8623C5F30116AD0943EA063302
S214443D3043EA8533C0F3011543EA0543850900F099
S214443D400F0043EA854304F0030543EA0553C4F3EE
S214443D50810543EA8553C4F30115A40943EA056380
S214443D6043EA84638C6D04F07044234354798B6532
S214443D701379D27981F85C30230104F0030403F408
S214443D80706343EA0233CA6D43EA0050054B40EA87
S214443D90046013401843C86570BD00BF08784020CF
S214443DA0A0744020FF0000FC70B5224D224A2C78B7
S214443DB0E878C4F3401604F00F03297943EA06135F
S214443DC0C4F38016E40943EA461343EA84136C7842
S214443DD043EAC413AC7843EAC43300F0030443EA2A
S214443DE0C453C0F3810443EA4463C0F30114800916
S214443DF043EAC46343EA4073106E00F00040034352
S214443E0001F0030013668B0803F004030343880899
S214443E1000F0080003438808C90900F01000034373
S214443E2043EA411392F8641021F03F010B4382F8B1
S214443E30643070BD08784020A0744020114A12486F
S214443E4010B55178137801F0030443EA0423C1F310
S214443E50810443EA8423C1F30114890943EA043301
S214443E6043EA8133A0F868305388A0F86A309388D0
S214443E70A0F86C30937980F86E30D37980F86F3040
S214443E8010BD00BF08784020A0744020064B074A67
S214443E901968587911671979DB7941EA002182F863
S214443EA07630A2F87410704708784020A0744020FA
S214443EB0084A09491378907881F87830537818433B
S214443EC0D378064A9B0443EA0023886F0240134390
S214443ED08B67704708784020A0744020FF0000FCA1
S214443EE008B5054B18880BF081F904490BF0D2F954
S214443EF0034BD86708BD00BF08784020CDCCCC3DE6
S214443F00A0744020104B41F69871104A595C82F8D0
S214443F10801041F69B71585C41F69A71595C41EAAF
S214443F200021A2F8811041F69D71585C41F69C71BF
S214443F30595C41EA0021A2F8841041F69F715B5C0B
S214443F4082F88630704700BF08784020A07440202E
S214443F50064A41F69871064B5158C3F8881041F604
S214443F609F71525C83F88C20704700BF08784020CD
S214443F70A07440200C4A41F69F730C4910B541F694
S214443F809974D05C41F69873D35C125D02F00102DA
S214443F9043EA0223D1F89020520C43EA40235204C9
S214443FA01343C1F8903010BD08784020A0744020D8
S214443FB0284941F69973284A70B5C85C41F69A7305
S214443FC0CD5C41F69B7300F00306CC5C41F69873D7
S214443FD0CB5C43EA0623C0F3810643EA8623C0F358
S214443FE00116800943EA063343EA803305F00300AA
S214443FF0C5F3810543EA004304F0030043EA8543DE
S21444400043EA0053C4F38100A40943EA8053D2F838
S214444010940043EA046300F07C40034341F69F70F7
S214444020C2F8943041F69C73CB5C82F8983041F6E3
S2144440309D73CB5C095C1B0203F47C5343EA8133D7
S214444040D2F8981021F47F1121F47C510B43C2F826
S214444050983070BD08784020A0744020214843F62C
S2144440603073214930B5C35A5BBAA1F89C3043F645
S2144440703373C25C43F63273C2F30115C45C9309CE
S21444408043EA850304F00F05240943EA051343F67F
S2144440903675455DED0843EA0523C2F3800543EAD9
S2144440A04533B1F89E5005F440452B43A1F89E3065
S2144440B043F63473C55C43F63573C35C43EA052361
S2144440C0A1F8A030C2F3C003520143EA440302F00D
S2144440D060021A4391F8A23023F07F031A4381F812
S2144440E0A22030BD08784020A0744020164A43F6EB
S2144440F03073164910B5D35A5BBAA1F8A43043F6C8
S2144441003273D05C43F63373D35C43EA0023A1F89E
S214444110A63043F63673D05C43F63473D45C43F629
S2144441203573D35C43EA042200F00103C0F3400035
S21444413043EA4203D1F8A820920C43EA404392044F
S2144441401343C1F8A83010BD08784020A07440201E
S214444150124A43F63071124B515A49BAA3F8AC107E
S21444416043F63271505C43F63371515C41EA0021A8
S214444170B3F8AE0061F30D0043F63671A3F8AE0013
S21444418043F63770515C125C42EA0122B3F8B01031
S21444419062F30D01A3F8B010704700BF08784020C2
S2144441A0A074402030B543F63073304C3049E35A5F
S2144441B05BBAA1F8B43043F63673E05C43F6377323
S2144441C0E25C43F63273E55C00F0030343EA85039E
S2144441D0C0F3800543EA8523C2F3800543EAC5233A
S2144441E0850943EA0533B1F8B65005F440452B43F8
S2144441F0C2F3C005A1F8B63043F63373E35C81F8E6
S214444200B830C0F3C0031B0243EA452302F003055B
S21444421043EA852343F63475655D43EA0533C0F3C4
S2144442200015C0F3401043EA0553C2F3001543EAB1
S21444423045539509120943EA8553D1F8B85002F01C
S214444240020225F47F05024325F47F452B43C1F83B
S214444250B83043F63573E35C81F8BB3091F8BC3034
S21444426023F003031A4381F8BC2030BD087840206D
S214444270A0744020F0B543F63273404F404DFE5C88
S21444428043F63473F95C43F63373C6F3801CF85C28
S21444429043F63573FC5C43F63673FA5CF30943EA3B
S2144442A04C0343F6317C42EA042217F80CC043EA36
S2144442B08C03C6F3401C43EA8C23C6F3001C43EA33
S2144442C0CC23C1F3400C43EA0C3343F6307C17F856
S2144442D00C7043EA4733C6F3C00743EA4753C6F372
S2144442E0800743EA8753C0F3001743EAC753470996
S2144442F043EA0763C4F30117A40943EAC763C6F352
S214444300400706F0010643EA477343EA8673D5F846
S214444310C06006F00046334301F00106C5F8C030DD
S214444320C2F30903C0F3C00243EA862343EAC22326
S214444330C0F3800243EA0233C0F3400200F00100B7
S21444434043EA4233C1F3C00243EA803343EAC43308
S214444350C1F3001443EA44438C09C1F3800143EAA1
S214444360844343EA025343EA4151D5F8C4309B0D93
S2144443709B051943C5F8C410F0BD00BF087840201B
S214444380A0744020284843F6307343F636722749D3
S214444390F0B5C35A43F63275845C43F635725BBA5D
S2144443A0455D825CA709A1F8C83043F6337347EAF3
S2144443B0820743F63772C65C43F63473825CC35C4A
S2144443C0B009B1F8CAC042EA042240EA8500C6F3FE
S2144443D0810543EA0623C6F3011640EA8520144DB8
S2144443E0C3F309030CEA050C43EA862340EA0C00AF
S2144443F043EA0733A1F8CA00C4F38100C4F30114A6
S21444440043EA8053D1F8CC0000F07F400343C1F820
S214444410CC30C2F30903B1F8D02043EA84231540D4
S2144444202B43A1F8D030F0BD08784020A07440203B
S21444443000F0FFFF1D4943F630731D48F0B5CB5AD4
S21444444043F632745BBA0E5DA0F8D43043F6337349
S214444450CA5C43F63573CD5CC2F3810443F63473C9
S2144444602F09CB5C44EA870443F6367743EA0223B3
S214444470C95D41EA052144EA8111A0F8D610C3F388
S2144444800901C2F3001343EA41039109C2F34012FF
S21444449043EAC62343EAC16343EA4273D0F8D820CA
S2144444A002F040421343C0F8D830F0BD08784020AC
S2144444B0A074402070B5234943F6367443F63575E8
S2144444C043F630730C5D4E5DCB5AA5091E485BBA65
S2144444D045EA860543F63776A0F8DC3043F6337370
S2144444E08E5DCA5C43F6347346EA042443F6327659
S2144444F0CB5C8E5D910943EA022341EA8601C2F30E
S2144445008006C3F3090341EA8621B0F8DE6006F468
S21444451078463143A0F8DE10C2F3C00143EA812353
S214444520C2F30011520943EAC52343EA415343EA1E
S2144445308453C0F8E03090F8E43062F3000380F827
S214444540E43070BD08784020A07440201D4A43F6ED
S21444455030731D4870B5D35A5BBAA0F8E83043F6BA
S2144445603273D45C43F63473D55C43F63373D15C10
S2144445702B09C5F3C00543EA011143F63673D65CEE
S21444458043F63573D35CDB0043EA5612C4F3400368
S21444459043EA450304F00105A40843EA850343EAD5
S2144445A0C403B0F8EA4004F47E442343A0F8EA3057
S2144445B041EA0233D0F8EC20D20DD2051343C0F8BA
S2144445C0EC3070BD08784020A07440201B4943F668
S2144445D031731B4830B5CB5C80F8F03043F6327309
S2144445E0CA5C43F63573CD5C43F63473CC5C43F611
S2144445F03073C95C93091B0243EA8123C2F340111A
S21444460043EA8143C2F38001C2F3C00243EAC14392
S214444610D0F8F01043EA02532A0905F00F0543EA9E
S2144446204253084A43EA45630A401343C0F8F0300D
S214444630230943EA041480F8F44030BD0878402047
S214444640A0744020FF0000E0074943F63073074A51
S214444650CB581BBAC2F8003143F63473CB581BBA56
S214444660C2F80431704700BF08784020A074402048
S214444670214845F6C863214930B5C35A5BBAA1F808
S214444680083145F6CB63C25C45F6CA63C2F30115EE
S214444690C45C930943EA850304F00F05240943EAFE
S2144446A0051345F6CE65455DED0843EA0523C2F39A
S2144446B0800543EA4533B1F80A5105F440452B4397
S2144446C0A1F80A3145F6CC63C55C45F6CD63C35CB8
S2144446D043EA0523A1F80C31C2F3C003520143EA6E
S2144446E0440302F060021A4391F80E3123F07F032C
S2144446F01A4381F80E2130BD08784020A07440202B
S214444700164A45F6C863164910B5D35A5BBAA1F89B
S214444710103145F6CA63D05C45F6CB63D35C43EAB6
S2144447200023A1F8123145F6CE63D05C45F6CC633F
S214444730D45C45F6CD63D35C43EA042200F001031F
S214444740C0F3400043EA4203D1F81421920C43EAF2
S214444750404392041343C1F8143110BD08784020F6
S214444760A0744020F0B545F6CA632D4F2D4CFD5C31
S21444477045F6CC63F95C45F6CB63C5F3801CFE5C1A
S21444478045F6CD63F85C45F6CE63FA5CEB0943EA3E
S2144447904C0345F6C96C42EA002217F80CC0C2F333
S2144447A0090243EA8C03C5F3401C43EA8C23C5F351
S2144447B0001C43EACC23C1F3400C43EA0C3345F6D1
S2144447C0C86C17F80C7043EA4733C6F300177609EB
S2144447D043EA475343EA8653C0F30116800943EA43
S2144447E04663C5F3400605F0010543EAC66343EA5B
S2144447F00573D4F8245105F060452B43C4F824319E
S21444480001F0010342EA832242EAC020C1F30012C7
S214444810890940EA423040EA8131A4F82811F0BDC3
S21444482008784020A0744020284845F6C86345F6DA
S214444830CE622749F0B5C35A45F6CA65845C45F648
S214444840CD625BBA455D825CA709A1F82C3145F67A
S214444850CB6347EA820745F6CF62C65C45F6CC632F
S214444860825CC35CB009B1F82EC142EA042240EA35
S2144448708500C6F3810543EA0623C6F3011640EADB
S2144448808520144DC3F309030CEA050C43EA86233A
S21444489040EA0C0043EA0733A1F82E01C4F3810032
S2144448A0C4F3011443EA8053D1F8300100F07F404A
S2144448B00343C1F83031C2F30903B1F8342143EA63
S2144448C0842315402B43A1F83431F0BD08784020AA
S2144448D0A074402000F0FFFF1D4945F6C8631D48FC
S2144448E0F0B5CB5A45F6CA645BBA0E5DA0F83831CB
S2144448F045F6CB63CA5C45F6CD63CD5CC2F3810412
S21444490045F6CC632F09CB5C44EA870445F6CE676C
S21444491043EA0223C95D41EA052144EA8111A0F82D
S2144449203A11C3F30901C2F3001343EA4103910960
S214444930C2F3401243EAC62343EAC14343EA42531E
S214444940D0F83C21920D92051343C0F83C31F0BD9B
S21444495008784020A0744020184845F6C863184993
S21444496030B5C35A5BBAA1F8403145F6CC63C55C52
S21444497045F6CA63C45C45F6CB63C35C43EA04228B
S21444498045F6CD63E409C35CB1F8420143EA052326
S214444990ED09C3F3090343EA85230A4D284003433C
S2144449A0A1F84231C2F30903B1F8442143EA84230F
S2144449B02A401343A1F8443130BD00BF0878402054
S2144449C0A074402000F8FFFF1D4A45F6C8631D4802
S2144449D070B5D35A5BBAA0F8483145F6CA63D45C7E
S2144449E045F6CC63D55C45F6CB63D15C2B09C5F361
S2144449F0C00543EA011145F6CE63D65C45F6CD6361
S214444A00D35CDB0043EA5612C4F3400343EA45034F
S214444A1004F00105A40843EA850343EAC403B0F856
S214444A204A4104F47E442343A0F84A3141EA02331F
S214444A30D0F84C21D20DD2051343C0F84C3170BD8A
S214444A4008784020A07440201B4945F6C9631B489B
S214444A5030B5CB5C80F8503145F6CA63CA5C45F63F
S214444A60CD63CD5C45F6CC63CC5C45F6C863C95C87
S214444A7093091B0243EA8123C2F3800143EA81433C
S214444A80C2F3C001C2F3401243EAC143D0F8501106
S214444A9043EA02532A0905F00F0543EA4253084AFB
S214444AA043EA45630A401343C0F85031230943EAB6
S214444AB0041480F8544130BD08784020A074402047
S214444AC0FF0000E030B545F6C863304C3049E35A41
S214444AD05BBAA1F8183145F6CE63E05C45F6CF6381
S214444AE0E25C45F6CA63E55C00F0030343EA8503EB
S214444AF0C0F3800543EA8523C2F3800543EAC52311
S214444B00850943EA0533B1F81A5105F440452B4369
S214444B10C2F3C005A1F81A3145F6CB63E35C81F8CD
S214444B201C31C0F3C0031B0243EA452302F00305CD
S214444B3043EA852345F6CC65655D43EA0533C0F311
S214444B400015C0F3401043EA0553C2F3001543EA88
S214444B5045539509120943EA8553D1F81C5102F08E
S214444B60020225F47F05024325F47F452B43C1F812
S214444B701C3145F6CD63E35C81F81F3191F8203152
S214444B8023F003031A4381F8202130BD08784020DF
S214444B90A0744020074945F6C863074ACB581BBA59
S214444BA0C2F8603145F6CC63CB581BBAC2F86431C0
S214444BB0704700BF08784020A07440200C4947F650
S214444BC064630C48CA5C47F66563CB5C43EA0222DE
S214444BD047F66263CB5C03F00F0343EA0213D0F854
S214444BE06821120D12051343C0F86831704700BFA0
S214444BF008784020A0744020064A47F66263D15C99
S214444C0047F66363D35C044A43EA0123A2F86C3153
S214444C10704700BF08784020A07440200C4949F6ED
S214444C20FC530C48CA5C49F6FD53CB5C43EA02226B
S214444C3049F6FA53CB5C03F00F0343EA0213D0F869
S214444C407021120D12051343C0F87031704700BF2F
S214444C5008784020A0744020064A49F6FA53D15CAE
S214444C6049F6FB53D35C044A43EA0123A2F8743161
S214444C70704700BF08784020A074402010B5134CFD
S214444C8020890AF0B3FA12490AF004FB114BA27BBE
S214444C901860114B60891A600AF0A8FA0F490AF0A6
S214444CA0F9FA0F490AF0ECF90E4B0F4A1860E37B09
S214444CB0A08903F00F0313600AF098FA0B490AF030
S214444CC0E9FA0AF0ADFC0A4B186010BDA074402007
S214444CD0CDCCCC3D7C1F4020641F40200AD7A33C4B
S214444CE000C02344701F4020601F4020ACC52737B7
S214444CF0681F4020104A1149137D03F003000860E2
S214444D00C3F383000E499B0908600E490B60537D2C
S214444D100D49C3F3410003F0010308600B490B60DF
S214444D2053690B49C3F3C7230B60D38A094AC3F3B9
S214444D30C7031360704700BFA0744020501F402034
S214444D404C1F4020481F4020401F4020441F402006
S214444D50341F40203C1F4020034B044A1B7C03F076
S214444D6001031360704700BFA0744020301F4020EA
S214444D700B4B0C4A1B7E03F001011160C3F3400148
S214444D80094A1160C3F38001084A1160C3F3C001A5
S214444D90074AC3F300131160064A1360704700BF06
S214444DA0A07440202C1F4020281F4020241F402051
S214444DB0201F40201C1F40200B4B0C4A1B7F03F037
S214444DC001011160C3F34001094A1160C3F3800135
S214444DD0084A1160C3F3C001074AC3F300131160C5
S214444DE0064A1360704700BFA0744020181F402036
S214444DF0141F4020101F40200C1F4020081F402036
S214444E00094B0A4A93F8203003F001011160C3F3BA
S214444E104001074A1160C3F38001064AC3F3C00346
S214444E201160054A13607047A0744020041F402058
S214444E30001F4020FC1E4020F81E402008B5FFF707
S214444E408BFFFFF795FFFFF7B7FFBDE80840FFF776
S214444E50D7BF08B5FFF7F2FFBDE80840FCF7F2BC41
S214444E60164A174992F8243003F003000860C3F347
S214444E70810014490860C3F3011013499B09086074
S214444E8012490B6092F82530114903F0030008607C
S214444E90C3F381000F490860C3F301100E499B0910
S214444EA008600E490B6092F826300D4A03F0030161
S214444EB0C3F3810311600B4A13607047A07440200B
S214444EC0041A4020001A4020FC194020F8194020BB
S214444ED0F4194020F0194020EC194020E8194020ED
S214444EE0E4194020E019402010B5194C208D0AF0F2
S214444EF07DF918490AF0CEF917490AF0C1F8174B5C
S214444F00174A186094F82A30A08D03F00F011B0945
S214444F101160144A136094F82B30134A323B1360E2
S214444F200AF064F911490AF0B5F911490AF0A8F8EB
S214444F30104B114A186094F82E3003F00F011B09E9
S214444F4011600E4A136094F82F200D4B1A6010BD62
S214444F50A07440200AD7A33B0AD72343F41E40201C
S214444F60F01E4020EC1E4020E81E40200AD7A33AFC
S214444F70F8D32342E41E4020E01E4020DC1E40209E
S214444F80D81E402010B5194C208E0AF02FF9184927
S214444F900AF080F917490AF073F8174B174A186055
S214444FA094F83230A08E03F00F011B091160144AA6
S214444FB0136094F83320134B1A600AF017F9124919
S214444FC00AF068F911490AF05BF8114B114A186067
S214444FD094F8363003F00F011B0911600E4A136033
S214444FE094F837200D4B1A6010BD00BFA0744020C3
S214444FF00AD7A33B0AD72343D41E4020D01E4020C2
S214445000CC1E4020C81E40200AD7A33AF8D32342D9
S214445010C41E4020C01E4020BC1E4020B81E402057
S21444502010B5174C208F0AF0E1F816490AF032F909
S21444503015490AF025F8154B154A186094F83A3085
S214445040A08F03F00F011B091160124A13600AF087
S214445050CDF811490AF01EF910490AF011F8104B20
S214445060104A186094F83E3003F00F011B09116093
S2144450700D4A136094F83F200C4B1A6010BD00BFD5
S214445080A07440200AD7A33B0AD72343B41E40202B
S214445090B01E4020AC1E40200AD7A33AF8D3234281
S2144450A0A81E4020A41E4020A01E40209C1E402037
S2144450B010B53E4C3E4A94F84030B4F8400003F0F5
S2144450C00101C0F3C7101160C3F34001394A1160AF
S2144450D0C3F38201384AC3F341131160374A13605D
S2144450E00AF084F836490AF0D5F80AF099FA354BAE
S2144450F01860206CC0F3C7300AF078F830490AF0DC
S214445100C9F80AF08DFA304B1860B4F84200C0F380
S214445110C7100AF06BF82D4909F0B2FF0AF080FA7E
S2144451202B4B94F8442018602A4B1A6094F8453068
S214445130294A03F001011160C3F34001274A116074
S214445140C3F38001264A1160C3F3C001254A1160A7
S214445150C3F30011244A1160C3F34011234A11607B
S214445160C3F38011224ADB091160224A136094F883
S2144451704630214A03F001011160C3F340011F4A3F
S2144451801160C3F380011E4A1160C3F3C0011D4A77
S2144451901160C3F300111C4A1160C3F340111B4A4B
S2144451A0C3F3801311601A4A136010BDA0744020E4
S2144451B0981E4020941E4020901E40208C1E402066
S2144451C00AD7233C881E4020841E402000002042EC
S2144451D0801E40207C1E4020781E4020741E4020A6
S2144451E0701E40206C1E4020681E4020641E4020D6
S2144451F0601E40205C1E4020581E4020541E402006
S214445200501E40204C1E4020481E4020441E402035
S214445210401E402038B5264D264B95F8484004F0AD
S2144452200102C4F302101A60C4F34002224B1A600F
S214445230C4F38002214B1A60C4F3C002204BE40935
S2144452401A6009F0CFFF1F4B1F4A18601F4BA86C0B
S2144452501C6095F84930C0F3473003F00F01C3F3A0
S2144452600013323811601A4A136009F0BFFF194B15
S2144452701860B5F84A00C0F34710323809F0B6FF54
S214445280154B1860B5F84C00A0F5004009F0AEFF89
S214445290124B1860B5F84E0009F0A8FF104909F003
S2144452A0F9FF104909F0ECFE0F4B186038BD00BFFB
S2144452B0A07440203C1E4020381E4020341E40200F
S2144452C0301E40202C1E4020241E4020281E4020F5
S2144452D0201E40201C1E4020181E4020141E402025
S2144452E00AD7233C00004843101E40207047304BEA
S2144452F0304A10B593F85940C4F381011170C4F391
S21444530001112D4A1170C4F301012C4AA4091170ED
S21444531093F858202A49C2F381100870C2F301104A
S21444532028490870C2F381002749C2F30102087075
S21444533026490A7093F85D202549C2F38100C2F3DA
S2144453400102087023490A7093F85E202249C2F38A
S21444535003120A7093F85F202049C2F301020A70D0
S21444536093F85A201E4902F003000860C2F38100F5
S2144453701C490860C2F301101B49920908601B4986
S2144453800A6093F85B201A4902F00300C2F38102D4
S2144453900860184993F85C000A7009F027FF16491C
S2144453A009F078FF154B1860154B1C6010BD00BF04
S2144453B0A07440200C1E40200B1E40200A1E402095
S2144453C0091E4020081E4020071E4020061E40207E
S2144453D0051E4020041E402038184020CC1D402086
S2144453E0FC1D4020F81D4020F41D4020F01D4020A8
S2144453F0EC1D402031184020CDCCCC3DE41D40204F
S214445400001E4020264A274992F8603003F00700E1
S2144454100860C3F3C00024490860C3F3001023495E
S2144454200870C3F340102249C3F38013087021491F
S2144454300B70B2F860302049C3F3C7130B60136E89
S2144454401E49C3F3C7330B60B2F862301C49C3F33A
S214445450C1130B6092F863301A49C3F341000860E5
S214445460C3F3C1001849C3F34113086017490B60DE
S21444547092F86430164A03F003011160C3F38001C6
S214445480144A1160C3F3C001134A1160C3F30011F8
S214445490124AC3F340131160114A1360704700BFA9
S2144454A0A0744020C81D4020C41D4020C21D40207A
S2144454B0C11D4020C01D4020BC1D4020B81D4020BA
S2144454C0B41D4020B01D4020AC1D4020A81D4020E7
S2144454D0A41D4020A01D40209C1D4020981D402017
S2144454E0941D402010B5194C194A94F8683094F825
S2144454F06A00C3F38101C3F301131170154A137094
S21444550094F86930144AC3F301011170C3F381015E
S214445510124AC3F381131170114A137009F062FEE4
S214445520104B186094F86B0009F05CFE0E4B94F830
S2144455306C2018600D4B1A7094F86D200C4B1A7042
S21444554094F86E200B4B1A7010BD00BFA074402018
S2144455508A1D4020791D4020891D4020781D40200A
S214445560881D4020841D4020801D40207C1D4020F6
S2144455707B1D40207A1D402010B50C4CB4F87200B8
S21444558009F034FE0A4909F085FE0A4B1860B4F85F
S214445590700009F02BFE064909F07CFE064BB4F871
S2144455A074201860054B1A8010BD00BFA0744020BC
S2144455B0CDCCCC3D741D4020701D40206E1D402037
S2144455C0054A0649B2F87A3092F87820C3F387033E
S2144455D00B70034B1A707047A07440206D1D40201A
S2144455E06C1D402010B5124C124B94F88020B4F831
S2144455F081001A6009F0FAFD0F4909F04BFE0F4985
S21444560009F03EFD0E4B1860B4F8840009F0EEFD38
S2144456100C4909F03FFE0C4B0C4A186094F886304F
S21444562003F00F011B091160094A136010BD00BF47
S214445630A0744020681D4020ACC52737ACC5A73EA3
S214445640641D4020CDCCCC3D601D40205C1D4020D8
S214445650581D402010B5114CB4F8880009F0C6FD1A
S2144456600F4909F017FE0F4909F00AFD0E4B186062
S214445670B4F88A0009F0BAFD094909F00BFE094955
S21444568009F0FEFC094B0A4A186094F88C3003F083
S2144456900F011B091160074A136010BDA074402017
S2144456A00AD7A33C00C02344541D4020501D40202C
S2144456B04C1D4020481D4020114A124992F8903013
S2144456C003F003000860C3F381000F490860C3F386
S2144456D001100E499B0908600D490B6092F8913001
S2144456E00C4903F00100C3F3430308600A490B6006
S2144456F0D2F89030094AC3F343331360704700BF6F
S214445700A0744020441D4020401D40203C1D4020A5
S214445710381D4020341D4020301D40202C1D402084
S214445720184B1B78002B2CD1174A184992F8943002
S21444573003F003000860C3F3810015490860C3F30F
S214445740011014499B09086013490B6092F8953080
S214445750124903F003000860C3F38100104908604F
S214445760C3F301100F499B0908600F490B6092F878
S21444577096300E4A03F00301C3F3810311600C4ACA
S2144457801360704726184020A0744020281D4020EF
S214445790241D4020201D40201C1D4020181D402054
S2144457A0141D4020101D40200C1D4020081D402084
S2144457B0041D402010B50C4C94F89F0000F01F00C8
S2144457C000EB800009F012FD084B1860B4F8A00006
S2144457D009F00CFD064909F05DFD064909F050FC48
S2144457E0054B186010BD00BFA0744020E81C402044
S2144457F0CDCC4C3D00C0CC44E41C402010B50C4CF1
S214445800B4F8A60009F0F2FC0A4909F043FD0A4937
S21444581009F036FC094B1860D4F8A800C0F34F00D2
S214445820A0F5FF407F3809F0E1FC054B186010BD39
S214445830A07440200AD7A33C00C02344D41C402074
S214445840CC1C402010B50D4CB4F8AE00C0F30D008F
S21444585009F0CCFC4FF07A5109F01CFD084B186057
S214445860B4F8B000C0F30D0009F0C0FC4FF07A5114
S21444587009F010FD034B186010BD00BFA074402013
S214445880C41C4020C01C4020704708B5074BB3F8E2
S214445890C400C0F3090009F0A9FC054909F0FAFC64
S2144458A0044909F0EDFB044B186008BDA074402081
S2144458B0CDCCCC3D9A994C42BC1C402010B5174CDC
S2144458C0B4F8CA00C0F3090009F090FC144909F082
S2144458D0E1FC144B1860B4F8CC00C0F3090009F09E
S2144458E085FC0F4909F0D6FC0F4B1860D4F8CC0061
S2144458F0C0F3093009F07AFC094909F0CBFC0B4B9C
S2144459001860B4F8D000C0F3090009F06FFC0449ED
S21444591009F0C0FC064B186010BD00BFA0744020C0
S214445920CDCCCC3DB81C4020B41C4020B01C4020FC
S214445930AC1C402038B5144DB5F8D600800909F0A3
S21444594055FC124909F0A6FC114909F099FBB5F833
S214445950D840104BC4F349041860204609F046FC6E
S2144459600D4909F097FC0D4B1860D5F8D800C0F3E4
S214445970CF2009F03BFC0A4909F08CFC094B18601F
S214445980094B1C6038BD00BFA0744020CDCC4C3DB4
S21444599066667241A81C40209A99193EA41C402071
S2144459A00AD7233CA01C4020341C402010B5164C7B
S2144459B0B4F8DE00C0F3090009F018FC134909F0F6
S2144459C069FC134B1860B4F8E000C0F3090009F012
S2144459D00DFC0E4909F05EFC0E4B1860D4F8E0004E
S2144459E0C0F3C92009F002FC084909F053FC0A4BED
S2144459F01860B4F8E200800909F0F8FB034909F09E
S214445A0049FC064B186010BDA07440209A99193E74
S214445A109C1C4020981C4020941C4020901C4020F5
S214445A2010B5134CB4F8EA00C0F3C50009F0DEFB29
S214445A30104909F02FFC104909F022FB0F4B18605F
S214445A40B4F8EC00C0F30B0009F0D0FB0C4909F0A5
S214445A5021FC0C4B1860D4F8EC00C0F30A3009F073
S214445A60C5FB044909F016FC074B186010BD00BF7F
S214445A70A0744020CDCCCC3DCDCC4C408C1C40209A
S214445A800AD7233C881C4020841C4020704770471B
S214445A9010B50C4C94F80B0100F01F0000EB80008E
S214445AA009F0A4FB084B1860B4F80C0109F09EFBFF
S214445AB0064909F0EFFB064909F0E2FA054B18607F
S214445AC010BD00BFA0744020801C4020CDCC4C3D6F
S214445AD000C0CC447C1C402010B50C4CB4F81201D9
S214445AE009F084FB0A4909F0D5FB0A4909F0C8FACB
S214445AF0094B1860D4F81401C0F34F00A0F5FF40DA
S214445B007F3809F073FB054B186010BDA074402025
S214445B100AD7A33C00C02344781C4020741C402071
S214445B20704708B5074BB3F82801C0F3090009F0DD
S214445B305DFB054909F0AEFB044909F0A1FA044BA4
S214445B40186008BDA0744020CDCCCC3D9A994C42F8
S214445B50501C402010B5174CB4F82E01C0F3090071
S214445B6009F044FB144909F095FB144B1860B4F84B
S214445B703001C0F3090009F039FB0F4909F08AFBEC
S214445B800F4B1860D4F83001C0F3093009F02EFBEF
S214445B90094909F07FFB0B4B1860B4F83401C0F395
S214445BA0090009F023FB044909F074FB064B18600E
S214445BB010BD00BFA0744020CDCCCC3D4C1C402032
S214445BC0481C4020441C4020401C402010B5134C28
S214445BD0B4F83A01800909F009FB114909F05AFB67
S214445BE0104909F04DFA104B1860B4F83C01C0F364
S214445BF0490009F0FBFA0D4909F04CFB09F010FD89
S214445C000B4B1860D4F83C01C0F3C72009F0EEFAF9
S214445C10084909F03FFB084B186010BDA0744020AB
S214445C20CDCC4C3D66667241701C40209A99193E14
S214445C30681C40200AD7233C6C1C402010B50C4CF2
S214445C40B4F84201C0F3090009F0D0FA094909F052
S214445C5021FB094B1860B4F84401C0F3090009F06D
S214445C60C5FA044909F016FB044B186010BD00BF82
S214445C70A07440209A99193E641C4020601C402021
S214445C8008B5FEF7FBFFFFF735F8FFF7E9F8FFF72F
S214445C900FFAFFF7BFFAFFF72AFBFFF7B3FBFFF74E
S214445CA021FCFFF769FCFFF78BFCFFF71DF9FFF7B4
S214445CB069F9FFF7B5F9FFF795FCFFF7CBFCFFF75B
S214445CC0FBFCFFF72DFDFFF7F9FDFFF733FEFFF76B
S214445CD06DFEFFF73FFFFFF779FFBDE80840FFF78B
S214445CE0ADBF10B5124CB4F84A01C0F3C50009F074
S214445CF07DFA104909F0CEFA0F4909F0C1F90F4B65
S214445D001860B4F84C01C0F30B0009F06FFA0C4964
S214445D1009F0C0FA0B4B1860D4F84C01C0F30A30B3
S214445D2009F064FA034909F0B5FA074B186010BD48
S214445D30A0744020CDCCCC3DCDCC4C405C1C402007
S214445D400AD7233C581C4020541C402008B5FFF773
S214445D5067FEBDE80840FFF7C4BF7047704708B504
S214445D60084BD3F86801C0F30F1009F03FFA064910
S214445D7009F090FA054909F083F909F051FC044BFF
S214445D80186008BDA0744020CDCC4C3D00C0CC4427
S214445D90801B402008B5084BB3F86C0109F026FA7E
S214445DA0064909F077FA064909F06AF909F038FC19
S214445DB0044B186008BD00BFA07440200AD7A33C1B
S214445DC000C02344841B402008B5094BD3F8700117
S214445DD0C0F30F1009F00AFA064909F05BFA0649BF
S214445DE009F04EF909F01CFC044B186008BD00BFCE
S214445DF0A0744020CDCC4C3D00C0CC44741B402005
S214445E0008B5084BB3F8740109F0F0F9064909F0EF
S214445E1041FA064909F034F909F002FC044B1860CB
S214445E2008BD00BFA07440200AD7A33C00C023444A
S214445E30741B402008B5FFF7BDFCFFF7DFFCFFF7F7
S214445E4001FDFFF722FDFFF723FEFFF745FEFFF7B0
S214445E5068FEFFF784FFFFF79DFFFFF7B5FFBDE839
S214445E600840FFF7CDBF1A4B186810B5C830194C18
S214445E7009F0B8F9184909F0C1FA08F05DFD0DF0CB
S214445E8021FD09F089F8154B1549A4F878011868DE
S214445E9009F0F8F8134909F0B1FA08F04DFD0DF091
S214445EA011FD09F079F8104BA4F87A011B68A4F8A0
S214445EB07C310E4B186808F03FFD0DF003FD09F0E9
S214445EC06BF80B4B84F87E011B6884F87F3110BD59
S214445ED03C1C4020A0744020CDCCCC3D381C4020F7
S214445EE000C023440AD7A33C341C4020301C402026
S214445EF02C1C4020224B234A1B68234982F88431B9
S214445F00224B09681B6809029B0201F4407103F4A2
S214445F1080630B431E490968C90201F4C0510B4310
S214445F201C490968490301F4C0410B431A490968EE
S214445F30C90301F4C0310B43D2F8841121F4FF3174
S214445F4021F480710B431549C2F88431144B096817
S214445F501B6801F00701A2F88A31124B1B68A2F8AD
S214445F608831114B1B78DB0003F008030B4392F88F
S214445F708C1121F00F010B4382F88C31704700BF1F
S214445F80BC1D4020A07440201C1C4020181C4020EF
S214445F90141C4020101C40200C1C4020C81D4020CF
S214445FA0081C4020041C4020C21D4020184B1949A0
S214445FB0186810B509F022FA174C08F0BDFC0DF02D
S214445FC081FC08F0E9FF154B1249A4F890011868C3
S214445FD009F014FA08F0B0FC0DF074FC08F0DCFF8D
S214445FE00F4B0C49A4F89201186809F007FA08F018
S214445FF0A3FC0DF067FC08F0CFFF0A4BA4F894010D
S2144460001B7884F89731084B1B7884F8963110BD7A
S214446010701D4020CDCCCC3DA0744020741D402043
S214446020E41D40206D1D40206C1D4020044B054956
S21444603093F8E821096861F3000283F8E821704781
S214446040A0744020E01B4020124B13491A68134B9F
S21444605002F001021B6803F0010343EA4203104ABC
S214446060126802F0010243EA82030E4A126802F002
S214446070010243EAC2030C4A126802F0010243EAF0
S214446080021391F8EC2122F01F02134381F8EC31FD
S214446090704700BFD81B4020A0744020DC1B402023
S2144460A0D41B4020D01B4020CC1B4020124B13490D
S2144460B01A68134B02F001021B6803F0010343EA1B
S2144460C04203104A126802F0010243EA82030E4A6F
S2144460D0126802F0010243EAC2030C4A126802F054
S2144460E0010243EA021391F8F02122F01F021343FF
S2144460F081F8F031704700BFC41B4020A074402094
S214446100C81B4020C01B4020BC1B4020B81B40205E
S2144461100F4B10491A68104B02F001021B6803F03B
S214446120010343EA42030D4A126802F0010243EABD
S21444613082030B4A126802F0010243EAC20391F852
S214446140F42122F00F02134381F8F431704700BF64
S214446150B01B4020A0744020B41B4020AC1B402001
S214446160A81B40201C4B1D49186810B509F046F979
S2144461701B4C08F0E1FB0DF0A5FB08F00DFF194B96
S214446180A4F89801186808F0D7FB0DF09BFB08F0BC
S21444619003FF154B1549A4F89A01186808F072FFD6
S2144461A0134909F02BF908F0C7FB0DF08BFB08F0F8
S2144461B0F3FE104B1049A4F89C01186808F062FFDF
S2144461C00E4909F01BF908F0B7FB0DF07BFB08F00D
S2144461D0E3FEA4F89E0110BD741F4020CDCCCC3DF8
S2144461E0A0744020481940206C18402000C0234426
S2144461F00AD7A33C181B4020000048430AD7233C38
S214446200114B1249186810B509F0F8F8104C08F00C
S21444621093FB0DF057FB08F0BFFE0E4B0E491B7860
S214446220A4F8A001A4F8A2310C4B186808F02AFF81
S2144462300B4909F0E3F808F07FFB0DF043FB08F048
S214446240ABFEA4F8A40110BDD0184020CDCCCC3D64
S214446250A0744020DA18402000C02344541840203C
S2144462600AD7A33C184B1949186810B508F00AFF1A
S214446270174909F0C3F8174C08F05EFB0DF022FBF3
S21444628008F08AFE144B1549A4F8A801186808F0CB
S214446290F9FE134909F0B2F808F04EFB0DF012FB74
S2144462A008F07AFE0F4BA4F8AA011B6884F8AC31B8
S2144462B00D4B1A680D4B1B6803F00F0343EA021399
S2144462C084F8AD3110BD00BFD41C402000C0234428
S2144462D00AD7A33CA0744020E41C402000C0CC4411
S2144462E0CDCC4C3DE41B4020981B40209C1B4020BA
S2144462F0164B1749186810B508F0C4FE154909F03E
S2144463007DF8154C08F018FB0DF0DCFA08F044FE56
S214446310124B1349A4F8B001186808F0B3FE1149AB
S21444632009F06CF808F008FB0DF0CCFA08F034FEDF
S2144463300D4BA4F8B2011A680C4B1B6803F00F030C
S21444634043EA021384F8B43110BD00BF781C4020E1
S21444635000C023440AD7A33CA07440207C1C4020A1
S21444636000C0CC44CDCC4C3D881B40208C1B4020E8
S214446370174B186810B500F28F20164C08F032FF01
S214446380154909F03BF808F0D7FA0DF09BFA08F0E7
S21444639003FE124BA4F8B801186800F2666008F0D1
S2144463A021FF0F4909F02AF808F0C6FA0DF08AFAD8
S2144463B008F0F2FD0B4BA4F8BA011A680A4B1B68A6
S2144463C003F00F0343EA021384F8BC3110BD00BF48
S2144463D0841B4020A07440200AD7A33C801B402046
S2144463E0CDCC4C3D781B40207C1B4020174B186876
S2144463F010B500F28F20164C08F0F4FE154908F04C
S214446400FDFF08F099FA0DF05DFA08F0C5FD124B51
S214446410A4F8C001186800F2666008F0E3FE0F496D
S21444642008F0ECFF08F088FA0DF04CFA08F0B4FDDA
S2144464300B4BA4F8C2011A680A4B1B6803F00F03FF
S21444644043EA021384F8C43110BD00BF741B4020D5
S214446450A07440200AD7A33C701B4020CDCC4C3DB2
S214446460681B40206C1B40200A4A0B4B126883F87A
S214446470E0210A4A126883F8E121094A126883F83F
S214446480E221084A126883F8E321074A1268C3F8EF
S214446490E4217047641B4020A0744020601B4020C9
S2144464A05C1B4020581B4020541B40204D4B4E4AFA
S2144464B01B78012B5BD14D4B4D491B6809689B00EB
S2144464C001F0030103F00C030B434A490968090130
S2144464D001F030010B43484909688901C9B20B43AE
S2144464E046490968090201F440710B434449096866
S2144464F0890201F440610B4342490968090301F4E7
S21444650040510B4340490968890389B20B433F49CC
S2144465100968090401F440310B433D49096889047C
S21444652001F440210B43D2F8C811090D09050B4369
S214446530C2F8C831374B1B7803F00301364B1B783F
S21444654003F003031B0143EA81133449097801F03D
S214446550030143EA0123B2F8CA1121F47C710B43C8
S214446560A2F8CA312E4B1B8882F8CC317047002BD8
S21444657033D12C4B2C491B6809689B0001F003015E
S21444658003F00C030B4329490968090101F0300163
S2144465900B43274909688901C9B20B432549096851
S2144465A0090201F440710B4323490968890201F446
S2144465B040610B4321490968090301F440510B43E8
S2144465C01F490968890389B20B431E4909680904AF
S2144465D001F440310B431C49A0E7023B012BA9D8E8
S2144465E0C7E700BF26184020A0744020001A402069
S2144465F0041A4020FC194020F8194020F419402081
S214446600F0194020EC194020E8194020E4194020B5
S214446610E0194020E71A4020E61A4020E81A4020B5
S214446620E41A4020241D4020281D4020201D4020E0
S2144466301C1D4020181D4020141D4020101D4020C5
S2144466400C1D4020081D4020041D4020124B1349B9
S2144466501B7803F00302124B1B7803F0030343EA50
S2144466608203104A127802F0030243EA02130E4AE7
S214446670127802F0030243EA82130C4A127802F0BC
S214446680030243EA0223B1F8D02102F47C421343C6
S214446690A1F8D031704700BF271B4020A07440208B
S2144466A0281B4020261B4020251B4020241B40201E
S2144466B0094B0A491A680A4B02F001021B6803F0A8
S2144466C0030343EA820391F8DC2122F007021343D2
S2144466D081F8DC31704700BF1C1B4020A07440206A
S2144466E0201B402038B5344B344D1868C83008F069
S2144466F079FD334908F082FE08F01EF90DF0E2F801
S214446700304B1C68304B64001B6804F0020403F0F2
S21444671001031C432D4B1B689B0003F004031C43DE
S2144467202B4B1B68DB0003F008031C43294B1B68F8
S2144467301B01DBB21C43284B1B681B0203F440734B
S2144467401C43264B1B689B0203F4E0531C43244B18
S2144467501B685B0303F4C0431C4308F01DFC214B39
S214446760214903EAC0331C43D5F8D43103F000432F
S2144467701C431E4BC5F8D441186808F083FC1049E6
S21444678008F03CFE08F0D8F80DF09CF808F004FC3D
S214446790174B1549A5F8D801186808F073FC084942
S2144467A008F02CFE08F0C8F80DF08CF808F0F4FB5E
S2144467B0A5F8DA0138BD00BFF01A4020A074402086
S2144467C00AD7233C0C1B4020101B4020081B4020AB
S2144467D0041B4020001B4020FC1A4020F81A40208E
S2144467E0F41A40200080FF7F00004843EC1A402003
S2144467F0181B4020274B2849186810B508F042FC5F
S214446800264908F0FBFD264C08F096F80DF05AF899
S21444681008F0C2FB234B2449A4F84C02186808F03D
S21444682031FC224908F0EAFD08F086F80DF04AF8F3
S21444683008F0B2FB1E4BA4F84E021B68A4F8503274
S2144468401C4B1A681C4B02F003021B6803F001033E
S21444685043EA4203194A126802F0030243EAC203B7
S214446860174A126802F0010243EA4213154A1268B4
S21444687002F00F0243EA8213134A126802F00F0230
S21444688043EA8223B4F8522202F440421343A4F863
S214446890523210BD101E4020000048430AD7233C05
S2144468A0A0744020D41C402000C023440AD7A33CF4
S2144468B0D81A4020141C4020D01A40200C1C4020DB
S2144468C0C41A4020C01A4020BC1A4020244B4FF023
S2144468D08E41244A1B6812681B0102F00F02DBB289
S2144468E01343214A1268120202F4706213431F4A89
S2144468F01268120302F4805213431D4A126852036C
S21444690002F4C04213431B4A1268D20302F4C03254
S2144469101343194A1268520410B502F0FF72174C1A
S2144469201343D4F8542202F07E421343C4F854323C
S214446930134B186808F0A6FB07F0FEFF0CF0C2FFE6
S21444694008F02AFB0F4BA4F858021A680E4B1B6833
S21444695003F00F0343EA021384F85A3210BD00BF13
S214446960B41A4020B81A4020B01A4020AC1A40202E
S214446970101C4020A41A4020BC1D4020A074402077
S214446980141E40209C1A4020A01A4020114B10B5DB
S214446990186807F0D1FF104C0CF094FF08F0FCFA8E
S2144469A00E4B84F85C021B6884F85D320C4B1B6803
S2144469B0A4F85E320B4B1B68A4F860320A4B1A6884
S2144469C00A4B1B6803F00F0343EA021384F862324F
S2144469D010BD00BF301C4020A07440202C1C40201A
S2144469E0041C4020081C4020841A4020881A40205A
S2144469F01C4A936CC3F3473382F89432B2F84A3055
S214446A00C3F3471382F89532B2F84230C3F3C71340
S214446A1082F8963292F85C3082F89732124B1968B4
S214446A20124B01F007011B6803F0010343EA4103DC
S214446A300F49097801F0010143EA01130D49096839
S214446A4001F00F0143EA41130B49096801F00F01B5
S214446A5043EA4123B2F8981201F460410B43A2F88A
S214446A6098327047A0744020C81D4020941D402092
S214446A70C21D4020801A40207C1A4020174B1868BC
S214446A8010B500F28F20164C08F0ACFB154908F000
S214446A90B5FC07F051FF0CF015FF08F07DFA124BD9
S214446AA0A4F82C02186800F2666008F09BFB0F49B5
S214446AB008F0A4FC07F040FF0CF004FF08F06CFA62
S214446AC00B4BA4F82E021A680A4B1B6803F00F03FC
S214446AD043EA021384F8303210BD00BF781A4020CF
S214446AE0A07440200AD7A33C741A4020CDCC4C3D19
S214446AF06C1A4020701A4020174B186810B500F2E4
S214446B008F20164C08F06EFB154908F077FC07F00A
S214446B1013FF0CF0D7FE08F03FFA124BA4F83402E9
S214446B20186800F2666008F05DFB0F4908F066FCE2
S214446B3007F002FF0CF0C6FE08F02EFA0B4BA4F842
S214446B4036021A680A4B1B6803F00F0343EA021323
S214446B5084F8383210BD00BF681A4020A074402024
S214446B600AD7A33C641A4020CDCC4C3D5C1A402046
S214446B70601A4020174B186810B500F28F20164C48
S214446B8008F030FB154908F039FC07F0D5FE0CF048
S214446B9099FE08F001FA124BA4F83C02186800F279
S214446BA0666008F01FFB0F4908F028FC07F0C4FE97
S214446BB00CF088FE08F0F0F90B4BA4F83E021A6875
S214446BC00A4B1B6803F00F0343EA021384F840326F
S214446BD010BD00BF581A4020A07440200AD7A33CDA
S214446BE0541A4020CDCC4C3D4C1A4020501A4020DC
S214446BF0174B186810B500F28F20164C08F0F2FABE
S214446C00154908F0FBFB07F097FE0CF05BFE08F016
S214446C10C3F9124BA4F84402186800F2666008F000
S214446C20E1FA0F4908F0EAFB07F086FE0CF04AFE4C
S214446C3008F0B2F90B4BA4F846021A680A4B1B68D4
S214446C4003F00F0343EA021384F8483210BD00BF32
S214446C50481A4020A07440200AD7A33C441A402037
S214446C60CDCC4C3D3C1A4020401A40204C4B4FF073
S214446C7084412DE9F04FDFF864A187B01B788AF889
S214446C80A832484B1B788AF8A932474B186808F054
S214446C90F9F94FF0834108F0FDFA07F04DFE0CF089
S214446CA011FE424B8046894618684FF0844108F0EE
S214446CB0E9F94FF0834108F0EDFA07F03DFE0CF099
S214446CC001FE3B4B06460F4693F800B0394B3A4913
S214446CD00BF0010B186808F0D5F9384908F08EFB1C
S214446CE007F02AFE0CF0EEFD354B364A1B78CDE90C
S214446CF0000110683449059308F0C4F9334908F094
S214446D007DFB07F019FE0CF0DDFD314A1478314A5C
S214446D1004F001041578240305F00105CDE90201C9
S214446D204946404608F038F9C0F30900AD023946F2
S214446D300543BAF8AA0200F4784005433046AAF858
S214446D40AA524FEA8B2508F027F9C0F3090BDDE970
S214446D50000108F021F9204A059B45EA0B0B02EA9C
S214446D60C02203F001034BEA020BDAF8AC224BEAEA
S214446D70C35302F07F421343DDE90201CAF8AC3242
S214446D8008F00AF9C0F30B000443BAF8B00200F462
S214446D9060400443AAF8B04207B0BDE8F08F00BF95
S214446DA02519402024194020201940201819402035
S214446DB0141940201019402033336F410AD7233C1E
S214446DC00C19402008194020CDCCCC42CDCC4C3DAB
S214446DD0041940201C19402000F87F00A07440206D
S214446DE0124B1A8DC3F86422114A1168114A01F0F5
S214446DF00F01126802F00F0242EA011293F82B10B8
S214446E0042EA0122A3F868229A8DC3F86C220A4A01
S214446E1011680A4A126802F00F0242EA011283F825
S214446E207022074A126883F871227047A074402083
S214446E30EC1E4020F01E4020DC1E4020E01E402079
S214446E40D81E4020114B1A8EC3F87422104A11687B
S214446E50104A126802F00F0242EA011283F87822BE
S214446E600D4A126883F879229A8EC3F87C220B4A1C
S214446E7011680B4A126802F00F0242EA011283F8C4
S214446E808022084A126883F881227047A074402002
S214446E90CC1E4020D01E4020C81E4020BC1E402091
S214446EA0C01E4020B81E40200F4B1A8FC3F88422C1
S214446EB00E4A11680E4A126802F00F0242EA0112A4
S214446EC083F888229A8FC3F88C220A4A11680A4AA1
S214446ED0126802F00F0242EA011283F89022074A2F
S214446EE0126883F891227047A0744020AC1E40205C
S214446EF0B01E4020A01E4020A41E40209C1E4020C1
S214446F00334B3449F0B51E78334B06F0030691F8FC
S214446F105C201D78314B42EA062205F003051C68C6
S214446F202F4B42EA8522240318682E4BA4B2000451
S214446F301B78224300F4702003F003072A4B1043C7
S214446F401B7803F0030343EA8703284F3F7807F090
S214446F50030743EA0713264F3F7807F0030743EA3D
S214446F608713244F3F7807F0030743EA0723224F4B
S214446F703F7807F0030743EA8723204F3F7807F01C
S214446F80030743EA07331E4F3F68BF03BFB23B4382
S214446F901C4F43EA06433F7843EA864307F0030719
S214446FA043EA065343EA865343EA066343EA87635F
S214446FB0D1F8087207F070473B43C1F80832D1F85D
S214446FC00C321B0D1B051843C1F80C02F0BD00BF64
S214446FD0041E4020A0744020051E402098194020DE
S214446FE094194020071E4020061E4020081E4020BC
S214446FF0091E40200A1E40200C1E40200B1E402026
S214447000001E40203118402008B5FFF7F1FCBDE8CB
S2144470100840FFF775BF214B214A70B51C68214BC9
S214447020B2F8605004F00F04186892F8603005F423
S214447030FF4592F8641000F00F0003F07F032B43E3
S214447040156E05F4FF052B43B2F86250C5F3C1151F
S21444705043EAC55392F86350C5F3410643EA466390
S214447060C5F3C106C5F3411543EAC66343EA45730F
S214447070D2F8105205F000452B43C2F8103201F006
S2144470803F03B2F8141243EA841301F4404143EA3E
S21444709080230B43A2F8143270BD00BF901D4020DD
S2144470A0A07440208C1D40201D4B1E4A1B6812684D
S2144470B09B001D4902F0030203F00C0313431B4AD2
S2144470C01268120102F030021343194A1268920100
S2144470D0D2B21343174A1268120202F440721343A0
S2144470E0154A1268920202F440621343134A126825
S2144470F0120302F440521343114A1268920302F4F4
S214447100703213430F4A1268920402F47012134307
S214447110D1F82822920D92051343C1F828327047BD
S2144471208419402088194020A074402080194020AB
S2144471307C1940207819402074194020701940204A
S2144471406C194020681940201A4B1B49186810B522
S21444715008F054F9194C07F0EFFB0CF0B3FB07F0BA
S2144471601BFF174B1449A4F81802186808F046F990
S21444717007F0E2FB0CF0A6FB07F00EFF114BA4F859
S2144471801A02188808F032F80B4908F037F907F065
S214447190D3FB0CF097FB07F0FFFE0B4BA4F81C0246
S2144471A01A680A4B1B6803F00F0343EA021384F879
S2144471B01E3210BD701D4020CDCCCC3DA074402066
S2144471C0741D40206E1D4020D41D4020D81D4020F4
S2144471D0124A92F8783010B582F82032104BD2F822
S2144471E020421878B2F87A30C3F38701936FC3F31A
S2144471F009231B0243EA81430A49097801F00F0137
S21444720043EA8163084921400B43C2F8203292F88E
S214447210243260F3030382F8243210BDA074402065
S2144472206419402065194020FF0000C0F8B53D4B66
S2144472303D4D1B783D4985F89C323D4B186808F017
S214447240DDF807F079FB0CF03DFB07F0A5FE394A64
S214447250394B03EA40231068D5F89C22000200F418
S21444726080700343354810400343C5F89C32344B82
S2144472701B7885F8A032334B1C68334B04F0030468
S2144472801F68324B07F001071E68314B44EA8704F7
S21444729006F00106186807F0A5FF4FF0814107F095
S2144472A0F9FF08F0BDF92B4A2B4B44EAC606D5F83D
S2144472B0A01203EA00231068284A800595F8A442E1
S2144472C000F4800024F00F0403431068244A264345
S2144472D0C005126800F4000085F8A4621206034351
S2144472E002F0407213431F4A1268920602F040624C
S2144472F013431D4A1268120702F0805213431B4A76
S2144473001268520702F000521343194A1268920751
S21444731002F080421343174A0A401343C5F8A0328A
S214447320F8BD00BF44194020A0744020CDCCCC3DCD
S214447330741F4020381A402000FEFF01FF0000FE64
S21444734045194020101A40200C1A4020081A4020A4
S214447350301A40202C1A402000FF3F00281A4020B4
S214447360141C4020201A40201C1A4020181A402082
S214447370141A4020FF000080084A094B1278094935
S21444738083F8B422084A0978127883F8B52293F829
S214447390B62261F3000283F8B6227047561940209D
S2144473A0A07440205419402055194020114B1249CE
S2144473B01B6810B5114C84F8D032114B1B6884F806
S2144473C0D132104B186807F05DFE0F4908F016F8E6
S2144473D007F0B2FA0CF076FA07F0DEFD0B4A94F8A2
S2144473E0D4321278A4F8D20262F3000384F8D4327A
S2144473F010BD00BF5019402000C02344A074402054
S2144474004C194020481940200AD7A33C461940202E
S214447410F8B5204B204D186807F0E4FE4FF0814144
S21444742007F038FF08F0FCF81C4B04461F681C4B5A
S214447430C4F30D0407F001071E681A4B44EA873468
S214447440186844EAC63407F0CDFE4FF0814107F091
S21444745021FF08F0E5F8144AC0F30D03A5F8CC4222
S2144474601068124A800300F4804003431068104AB0
S214447470C003126800F4FF00D205034302F0FF4243
S2144474801343D5F8C82202F000421343C5F8C83265
S214447490F8BD00BF30194020A07440202C1940206D
S2144474A028194020401940203C19402038194020D3
S2144474B0341940200D4B0E4A1B780E4982F8DC32B4
S2144474C00D4B09781B7801F0010182F8DD320B4B35
S2144474D01B785B0003F002030B4392F8DE1221F0A4
S2144474E003010B4382F8DE32704700BF0319402085
S2144474F0A074402001194020021940200019402061
S2144475000C4B0D4A1B680D4982F8D8320C4B09784F
S2144475101B6801F0030182F8D9320A4B1B789B00A2
S21444752003F00C030B430849097843EA011382F835
S214447530DA327047FC184020A0744020F7184020E8
S214447540F8184020F6184020F5184020F8B5254B8A
S214447550254C1B78254F84F8E032254B1B7884F85D
S214447560E132244B1878323007F040FE014607F0EB
S21444757089FD08F055F8204984F8E2020E781F4940
S2144475803F780D781E4907F001071E4B08781E49C0
S2144475901A78303009781D4B49001B7801F03E01BB
S2144475A0394394F8E37227F03F07394384F8E312EB
S2144475B003F03F0102F01F0306F00F0243EA4113B3
S2144475C043EAC22305F03F0243EAC23300F03F02D7
S2144475D043EA4253D4F8E42202F078421343C4F810
S2144475E0E432F8BDF4184020A0744020F11840203E
S2144475F0F3184020F2184020ED184020EC184020A4
S214447600EB184020EF184020F0184020EE18402099
S21444761038B50C4B0C4C5D68284607F08DF90CF0D9
S21444762051F907F0B9FC0949C4F8C402284607F0E2
S214447630E5FE07F081F90CF045F907F0ADFCC4F817
S214447640C00238BD00464020A074402000000842D6
S2144476502DE9F74F374D384E686807F0E1FF86F856
S214447660E802A86807F0DCFF344986F8E90268694E
S21444767007F008FD324907F0C1FE07F0D1FF834604
S214447680A86907F0CDFF2D490446E86907F0FAFCDF
S2144476902B4907F0B3FECBF3090B07F0C1FF824634
S2144476A0286A07F0BDFF25498146686A07F0EAFC68
S2144476B0234907F0A3FE07F0B3FF8046A86A07F005
S2144476C0AFFF1E4900F00107E86807F0DBFC1C49E1
S2144476D007F094FE07F0A4FFC0F30903286901935A
S2144476E007F09EFF019B00F0010043EA8023B6F8B2
S2144476F0EA0200F4784003431248A6F8EA32A302AA
S21444770000EACA2A03F480634FEA495043EA0B036B
S21444771000F4001043EA0A03034343EA8853C6F8D6
S214447720EC3296F8F03267F3000386F8F03203B092
S214447730BDE8F08F00464020A07440206666724143
S214447740CDCC4C3D00F81F00084A094B1278094935
S21444775083F81823084A0978127883F8192393F88B
S2144477601A2361F3000283F81A237047EA1840206C
S214447770A0744020E8184020E918402070B5194C01
S214447780194D26682946304607F040FF08B1256063
S21444779006E0164D3046294607F01AFF0028F6D173
S2144477A0134B144D1B68144A85F80833134B127850
S2144477B01B68134985F8093395F80C3362F30003C4
S2144477C085F80C33206807F05DFC0E4907F016FE7A
S2144477D007F0B2F80CF076F807F0DEFBA5F80A03DB
S2144477E070BD00BFDC1840200000D7430000D7C35C
S2144477F0E4184020A0744020DA184020E0184020C6
S21444780000C023440AD7A33C264B274910B5274C2F
S2144478101B7884F80033264B186807F0EFFD07F012
S214447820FFFE244A244B03EA40231068D4F800237E
S214447830000200F48070034320481040204A03436B
S2144478401268C4F8003312021E4B02F480721B788E
S21444785084F804331C4B1B685B0203F4C063134375
S2144478601A4A1268D20202F4C0521343184A1268E3
S214447870520302F400521343164A1268920302F467
S21444788080421343144A1268D20302F4C0321343AC
S214447890D4F8042322F4FF3222F480721343C4F84B
S2144478A0043310BDD8184020CDCCCC3DA074402025
S2144478B0D0184020D418402000FEFF01FF0000FEF0
S2144478C0CC184020D9184020C8184020C41840205E
S2144478D0C0184020BC184020B81840203A4B4FF0FF
S2144478E084412DE9F047394E1B7886F8F432384BFC
S2144478F01B7886F8F532374B186807F0C3FB4FF011
S214447900834107F0C7FC07F08BFE334B04463349EC
S21444791093F800A0324B0AF0010A186807F0B2FB4D
S214447920304907F06BFD07F07BFE2F4B81462F490D
S21444793093F800802E4B08F00108186807F0A2FB65
S2144479402C4907F05BFD07F06BFE2B4B05464FF0CA
S21444795084411F78294BC5F30B0507F001071868C7
S21444796007F090FB4FF0834107F094FC07F058FE75
S214447970234BC0F3090245EA07351878C4F30903D4
S21444798000F0010043EA8A2342EA8022B6F8F6026F
S21444799000F4784002431B4800EAC929A6F8F622B8
S2144479A0D6F8F82243EA090302F07F4243EAC85372
S2144479B01343C6F8F832B6F8FC3203F460431D436A
S2144479C0A6F8FC52BDE8F087B5184020A0744020C5
S2144479D0B4184020A8184020A418402033336F41E0
S2144479E0A01840200AD7233C9C184020CDCCCC423B
S2144479F098184020CDCC4C3D94184020B0184020D8
S214447A00AC18402000F87F002DE9F74F374D384E2C
S214447A10686807F005FE86F83803A86807F000FE95
S214447A20344986F83903686907F02CFB324907F075
S214447A30E5FC07F0F5FD8346A86907F0F1FD2D49FE
S214447A400446E86907F01EFB2B4907F0D7FCCBF346
S214447A50090B07F0E5FD8246286A07F0E1FD254953
S214447A608146686A07F00EFB234907F0C7FC07F017
S214447A70D7FD8046A86A07F0D3FD1E4900F00107EB
S214447A80E86807F0FFFA1C4907F0B8FC07F0C8FDA1
S214447A90C0F309032869019307F0C2FD019B00F077
S214447AA0010043EA8023B6F83A0300F478400343DF
S214447AB01248A6F83A33A30200EACA2A03F48063BB
S214447AC04FEA495043EA0B0300F4001043EA0A0322
S214447AD0034343EA8853C6F83C3396F8403367F387
S214447AE0000386F8403303B0BDE8F08F00464020DC
S214447AF0A074402066667241CDCC4C3D00F81F0011
S214447B000D4B0E4A1B780E4982F814330D4B0978F8
S214447B101B7801F0010182F815330B4B1B785B0090
S214447B2003F002030B4392F8161321F003010B43B0
S214447B3082F81633704700BF93184020A074402044
S214447B409118402092184020901840200C4B0D4A23
S214447B501B680D4982F810330C4B09781B6801F0FA
S214447B60030182F811330A4B1B789B0003F00C0385
S214447B700B430849097843EA011382F812337047E5
S214447B808C184020A0744020841840208818402038
S214447B908318402082184020F8B5254B254C1B7886
S214447BA0254F84F83033254B1B7884F83133244BE7
S214447BB01878323007F01AFB014607F063FA07F0EC
S214447BC02FFD204984F832030E781F493F780D78FC
S214447BD01E4907F001071E4B08781E491A783030B4
S214447BE009781D4B49001B7801F03E01394394F84F
S214447BF0337327F03F07394384F8331303F03F01C8
S214447C0002F01F0306F00F0243EA411343EAC2237D
S214447C1005F03F0243EAC23300F03F0243EA4253D0
S214447C20D4F8342302F078421343C4F83433F8BD0E
S214447C3081184020A07440207E18402080184020A0
S214447C407F1840207A184020791840207818402021
S214447C507C1840207D1840207B18402008B5FFF74C
S214447C6075FCBDE80840FFF797BF38B50C4B0D4C84
S214447C705D68284606F060FE0BF024FE07F08CF99B
S214447C800949C4F82C03284607F0B8FB06F054FE0E
S214447C900BF018FE07F080F9C4F8280338BD00BF7F
S214447CA000464020A07440200000084208B5FEF775
S214447CB0DAF8FEF71FF9FEF779F9FEF7B7F9FEF79B
S214447CC0C3F9FEF7F3F9FEF723FAFEF7CBFAFEF70D
S214447CD00FFBFEF74DFBFEF789FBFEF7C5FBFEF7F1
S214447CE0E5FBFEF7B3FCFEF7E3FCFEF7FBFCFEF712
S214447CF081FDFEF7EBFDFEF749FEFEF7BFFEFEF7FD
S214447D00FBFEFEF737FFFEF773FFFFF769F8FFF752
S214447D1099F8FFF7C9F8FFF77EF9FFF715FAFFF76A
S214447D2057FAFFF7C1F9FEF7A1FFFFF771FCFFF71B
S214447D30D5FDBDE80840FFF798BF114B11491B68B5
S214447D4010B5114C84F84433104B1B6884F8453303
S214447D500F4B186807F096F90E4907F04FFB06F0EC
S214447D60EBFD0BF0AFFD07F017F90B4A94F84833D8
S214447D701278A4F8460362F3000384F8483310BD2F
S214447D807418402000C02344A0744020701840203B
S214447D906C1840200AD7A33C691840200D4B0E4A65
S214447DA01B780E4982F850330D4B09781B7801F046
S214447DB0010182F851330B4B1B785B0003F002033E
S214447DC00B4392F8521321F003010B4382F85233CB
S214447DD0704700BF68184020A074402066184020B2
S214447DE067184020651840200C4B0D4A1B780D49F7
S214447DF082F84C330C4B09781B7801F0030182F867
S214447E004D330A4B1B789B0003F00C030B43084985
S214447E10097843EA011382F84E33704764184020C9
S214447E20A074402062184020631840206118402007
S214447E3060184020114B12491B6810B5114C84F849
S214447E405433114B1B6884F85533104B186807F0AD
S214447E5019F90F4907F0D2FA06F06EFD0BF032FD21
S214447E6007F09AF80B4A94F858331278A4F8560355
S214447E7062F3000384F8583310BD00BF5C184020FA
S214447E8000C02344A0744020581840205418402072
S214447E900AD7A33C501840200D4B0E4A1B780E4977
S214447EA082F85C330D4B09781B7801F0010182F8A7
S214447EB05D330B4B1B785B0003F002030B4392F8D5
S214447EC05E1321F003010B4382F85E33704700BF14
S214447ED04F184020A07440204D1840204E18402093
S214447EE04C1840200C4B0D4A1B680D4982F86033F1
S214447EF00C4B09781B6801F0030182F861330A4B86
S214447F001B789B0003F00C030B430849097843EAAB
S214447F10011382F86233704748184020A07440200A
S214447F2040184020441840203F1840203E18402027
S214447F3008B5FFF721FAFFF739FAFFF777F9FFF7A5
S214447F4067FAFFF785FBFFF7B5FAFFF7D9FAFFF7AD
S214447F50FBFBFFF713FCFFF757FCFFF755FDFFF756
S214447F60CFFDFFF7F3FDFFF7E8FEFFF717FFFFF738
S214447F703BFFFFF75FFFFFF78FFFBDE80840FFF7C3
S214447F80B1BF074A0020074BD2F87811D2F87C21BB
S214447F909962DA62044B93E80600FBF707BD00BF1C
S214447FA0A074402008784020D46F4600144A1548F0
S214447FB092F8851192F8843110B4C1F3010480F824
S214447FC0283001F01C03C1F34111234380F82930C3
S214447FD0D2F88431C3F3C13492F88C31C3F3C0036E
S214447FE0DB0143EA84030B4380F82A30D2F8883115
S214447FF0C3620020044B10BC93E80600FBF7D6BCD3
S214448000A074402008784020DC6F46000B4A0020CD
S2144480100B4BD2F890119962B2F8941183F82C1055
S21444802092F8961192F8972183F82D1083F82E2013
S214448030044B93E80600FBF7B9BC00BFA07440208D
S21444804008784020FC6F4600064B0020064A93F80A
S214448050E831C3F3000382F82830044B93E8060063
S214448060FBF7A4BCA0744020087840200470460067
S214448070084B002093F8EC31C3F3000203F01E03D0
S2144480801343054A82F82830044B93E80600FBF76E
S2144480908DBC00BFA0744020087840200C70460079
S2144480A0084B002093F8F031C3F3000203F01E039C
S2144480B01343054A82F82830044B93E80600FBF73E
S2144480C075BC00BFA0744020087840201470460059
S2144480D0084B002093F8F431C3F3000203F00E0378
S2144480E01343054A82F82830044B93E80600FBF70E
S2144480F05DBC00BFA0744020087840201C70460039
S214448100064A0020064BD2F89811D2F89C21996270
S214448110DA62044B93E80600FBF748BCA0744020A0
S2144481200878402024704600064A0020064BD2F8C1
S214448130A011B2F8A42199629A85044B93E80600EC
S214448140FBF734BCA0744020087840202C704600CE
S21444815008B50A4B50200A4AD3F8A81193F8AC3114
S214448160283211600821137103F060FD054B00208E
S21444817093E80600BDE80840FBF718BCA07440200E
S21444818008784020A46F4600094B00200949D3F8DC
S214448190B02193F8B4318A6203F0F002C3F30303C8
S2144481A0134381F82F30044B93E80600FBF7FEBBDD
S2144481B0A074402008784020AC6F4600094B00204D
S2144481C00949D3F8B82193F8BC318A6203F0F00227
S2144481D0C3F30303134381F82F30044B93E806009C
S2144481E0FBF7E4BBA074402008784020B46F4600F8
S2144481F0094B00200949D3F8C02193F8C4318A6258
S21444820003F0F002C3F30303134381F82F30044B07
S21444821093E80600FBF7CABBA074402008784020C9
S214448220BC6F46000A4A00200A4BD2F8E01192F886
S214448230E421996283F82C2083F82D2083F82E209D
S21444824083F82F20044B93E80600FBF7AFBB00BF30
S214448250A074402008784020F46F4600254A2649FA
S21444826092F8C831C3F3010003F0FC03034310B48F
S21444827081F8283092F8C931C3F3010003F0FC03B7
S214448280034392F8CA0181F82930C0F3010400F090
S2144482900C0323438409C0F3011081F82A3092F872
S2144482A0CB3103F003039B0143EA8403034381F881
S2144482B02B3092F8CC3181F82C3092F8CD3103F043
S2144482C03800C3F30203034381F82D3092F8CE31CD
S2144482D0C3F38300D2F8CC31C3F3833343EA0013A9
S2144482E0002081F82F30054B10BC93E80600FBF7BE
S2144482F05DBB00BFA074402008784020C46F460091
S2144483000B490C4A91F8D031C3F3010003F0FC0347
S2144483100343002082F8283091F8D131C3F3010397
S21444832082F82930044B93E80600FBF73FBB00BFB6
S214448330A074402008784020E46F4600084B002094
S21444834093F8DC3103F00402C3F301031343054AF4
S21444835082F82830044B93E80600FBF727BB00BF9F
S214448360A074402008784020EC6F46001049114A1B
S21444837091F8D431C3F3000003F0FE03034382F8BC
S214448380283091F8D53103F07C00C3F3010303434E
S214448390002082F82930D1F8D431C3F3CF33538543
S2144483A0D1F8D831D362044B93E80600FBF7FEBA03
S2144483B0A074402008784020CC6F46001B4938B54E
S2144483C01B4CD1F84C3204F5FE52B1F850021360FF
S2144483D041F6C473E05291F85232C3F34100C3F3FA
S2144483E0C1050543C3F30000C3F3401340EA8500C8
S2144483F040EA430341F6C670235491F85332C3F31C
S2144484008300B1F8523241F6C771C3F3831343EA8B
S214448410001313206354082103F071FD054B01201B
S21444842093E80600BDE83840FBF7C0BAA074402085
S214448430087840207C7046002149224B91F854022B
S21444844003F5FE5210B500F0F004C0F303002043D9
S214448450107091F8550200F07004C0F303002043F6
S21444846041F6C174185541F6C274D1F85402C0F3AB
S214448470C130185541F6C374B1F85602C0F34700EC
S214448480185541F6C470B1F8584291F85A121C5423
S21444849041F6C57000241C5401F0F000C1F30301FA
S2144484A0014341F6C77019540821142003F027FDF0
S2144484B0054B012093E80600BDE81040FBF776BA6A
S2144484C0A07440200878402084704600154B164916
S2144484D003F5FE5291F85C0210B51070002441F684
S2144484E0C1701C5441F6C270B1F85E421C5241F64B
S2144484F0C470B1F8604291F862121C5201F0F00068
S214448500C1F30301014341F6C770195408211520ED
S21444851003F0F5FC054B012093E80600BDE8104047
S214448520FBF744BA08784020A07440208C7046007C
S21444853010B512490020124C01F5FE52D4F894327C
S214448540136041F6C473C85494F89932C3F3430095
S214448550B4F89832C3F3431343EA001341F6C770A2
S2144485600B540821162003F0CAFC064B012093E85E
S2144485700600BDE81040FBF719BA00BF0878402053
S214448580A0744020AC70460008B5FFF75DFDFFF7C9
S2144485906FFDFFF785FDFFF79BFDBDE80840FFF73D
S2144485A0C7BF08B5FDF7D2FBF9F74DF9FEF72CFD2A
S2144485B0BDE80840FFF7E8BF08B50E480E4B00F587
S2144485C0FE52D3F82C1293F83032116003F0F001C7
S2144485D0C3F303030B4341F6C771435408215020A9
S2144485E003F08DFC054B012093E80600BDE80840E7
S2144485F0FBF7DCB908784020A07440205C70460045
S21444860008B50E480E4B00F5FE52D3F8341293F8D4
S2144486103832116003F0F001C3F303030B4341F611
S214448620C77143540821512003F069FC054B0120CF
S21444863093E80600BDE80840FBF7B8B90878402040
S214448640A07440206470460008B50E480E4B00F5F2
S214448650FE52D3F83C1293F84032116003F0F00116
S214448660C3F303030B4341F6C77143540821602008
S21444867003F045FC054B012093E80600BDE808409E
S214448680FBF794B908784020A07440206C704600EC
S21444869008B50E480E4B00F5FE52D3F8441293F834
S2144486A04832116003F0F001C3F303030B4341F671
S2144486B0C77143540821612003F021FC054B012077
S2144486C093E80600BDE80840FBF770B908784020F8
S2144486D0A074402074704600194B1A4A03F5FE51A4
S2144486E0B2F86402088092F8681201F0F000C1F310
S2144486F00301014341F6C270195441F6C37192F81E
S2144487006902585441F6C47092F86C12195441F6F2
S214448710C570195492F8701201F0F000C1F30301C9
S214448720014341F6C6701954012092F8711241F67D
S214448730C7729954044B93E80600FBF737B900BF59
S21444874008784020A074402094704600194B1A4A7A
S21444875003F5FE51B2F87402088092F8781201F0DC
S214448760F000C1F30301014341F6C270195441F6C7
S214448770C37192F87902585441F6C47092F87C1248
S214448780195441F6C570195492F8801201F0F0005D
S214448790C1F30301014341F6C6701954012092F80F
S2144487A0811241F6C7729954044B93E80600FBF7CE
S2144487B0FDB800BF08784020A07440209C70460056
S2144487C0174B184A03F5FE51B2F88402088092F813
S2144487D0881201F0F000C1F30301014341F6C27070
S2144487E0195441F6C370D2F88C121954090A41F64A
S2144487F0C470195492F8901201F0F000C1F30301CA
S214448800014341F6C6701954012092F8911241F67C
S214448810C7729954044B93E80600FBF7C7B800BFE9
S21444882008784020A0744020A4704600284829496F
S21444883090F8083201F5FE5270B5C3F3010403F014
S214448840FC032343137090F80932C3F3010403F086
S214448850FC03234341F6C1740B5541F6C27390F8AA
S2144488600A422501A609C4F30114CD5490F80B52CC
S21444887005F00303C5F381051B0143EA860323433E
S21444888041F6C37443EA85130B5541F6C47390F816
S2144488900C42CC5441F6C57490F80D3290F80E0252
S2144488A01D01C3F3031300F00F000D5543EA0013F4
S2144488B041F6C7700B5408214FF4AE6003F01FFB1B
S2144488C0054B012093E80600BDE87040FBF76EB800
S2144488D0A074402008784020347046002D4991F812
S2144488E0100238B5C0F3001500F008032A4C43EADA
S2144488F04513C0F3020504F5FE522B43C0F340155E
S214448900C0F3801043EA851343EAC01341F6C170AE
S2144489101370B1F81032C3F3C713235441F6C27030
S214448920D1F81032C3F3C733235491F81302C0F37B
S214448930C103C0F34105C0F341101B0143EA85035C
S214448940B1F81252C5F3C1152B4343EA801341F6DE
S214448950C370235441F6C47091F814329B002354D8
S21444896091F81532C3F38300B1F8143241F6C77157
S214448970C3F3831343EA00134FF4B06063540821EF
S21444898003F0BDFA054B012093E80600BDE83840E5
S214448990FBF70CB8A0744020087840203C70460092
S2144489A01849194891F8283200F5FE5210B5C3F319
S2144489B0010403F0FC032343137091F8293203F0B7
S2144489C03C04C3F30103234341F6C174035591F8B1
S2144489D02A32C3F38304D1F8283241F6C771C3F36D
S2144489E0833343EA04134354082140F2855003F08A
S2144489F086FA064B012093E80600BDE81040FAF7D5
S214448A00D5BF00BFA074402008784020547046006C
S214448A101149124B01F5FE52D3F8180210B5B3F8BB
S214448A201C42106041F6C47093F81E320C5203F098
S214448A30F000C3F30303034341F6C7700B54082105
S214448A404FF4B26003F05BFA054B012093E806004E
S214448A50BDE81040FAF7AABF08784020A07440202A
S214448A60447046001749184891F8203200F5FE52E3
S214448A7010B5137041F6C174D1F82032C3F30923FC
S214448A80035541F6C274B1F82232C3F38103035549
S214448A9091F8243203F00F0491F8233241F6C7715B
S214448AA0C3F3830343EA04134354082140F2955026
S214448AB003F025FA054B012093E80600BDE8104074
S214448AC0FAF774BFA0744020087840204C704600E3
S214448AD00D4843F65872B0F8B41208B549BA0B4B71
S214448AE099521A4490F8B61243F65A70C90119546A
S214448AF00321322003F09AF8054B022093E806003F
S214448B00BDE80840FAF752BFA074402008784020D9
S214448B10C4704600114B43F65870114AB3F8D0124D
S214448B2049BA10B5115243F65A74B3F8D21293F8B0
S214448B30D43249BA03F00103115343F65C719B01E6
S214448B40535402440521402002F0F9FE054B02200E
S214448B5093E80600BDE81040FAF728BFA07440200A
S214448B6008784020DC7046003048314A90F8A032FD
S214448B7090F89C1270B543F6587590F8A342535536
S214448B8043F65973D15443F65A71D0F89C32C3F322
S214448B904F235BBA5352C4F3801304F0100141EAE6
S214448BA0C301C4F30103194390F89D3203F0010353
S214448BB041EA4311C4F3810304F0200441EA8311DB
S214448BC043F65C73D15490F8A412C1F3800601F0C6
S214448BD00803C1F3010143EA06130B4390F8A212BB
S214448BE0D0F8A0022343CC09C1F3801143EA84138E
S214448BF043F65D741355C0F30D2343F65E74C0F319
S214448C0005409B001055642043EA410343F65F71D8
S214448C1053542A44082103F009F8064B022093E8EB
S214448C200600BDE87040FAF7C1BE00BFA0744020FD
S214448C3008784020B47046001F4843F658721F4BCD
S214448C40B0F8CA12C1F3C71170B5995443F65974B3
S214448C50D0F8C8121A44B0F8C852C1F3C731C5F3A5
S214448C600526195590F8CD4204F08001C4F38014CB
S214448C70314343F65A76995543F65B715D54B0F8E2
S214448C80CC5290F8C912C5F3052001F040010143C7
S214448C9043F65C7041EAC411195443F65D716A2088
S214448CA05D54062102F0C2FF054B022093E80600FD
S214448CB0BDE87040FAF77ABEA07440200878402099
S214448CC0D470460038B52C4B43F658702B4AB3F84C
S214448CD0A812B3F8B05249BA115293F8AE12CC095E
S214448CE0C5F3032141EA041193F8B142C4F30014D6
S214448CF041EA441193F8AB42C4F3800441EA841138
S214448D0093F8AD42C4F3800441EAC41143F65A745E
S214448D10115543F65B71B3F8AA42555443F65C7159
S214448D20C4F30905C4F387045454B3F8AC12D3F817
S214448D30AC32C1F30904C1F3051141EA851143F687
S214448D405D755155C3F3CB21C3F3C34343EA0413C0
S214448D5043F65E74135543F65F73D15402440821B8
S214448D60702002F063FF064B022093E80600BDE83D
S214448D703840FAF71BBE00BFA07440200878402055
S214448D80BC704600284A43F658702849B2F8E83280
S214448D905BBA30B40B5243F65A73B2F8EA02B2F8EE
S214448DA0EC52C0F30904C0F38700C854C5F301204D
S214448DB092F8EB3203F00403034392F8ED02C0F357
S214448DC0800043EAC00392F8EE02C0F3401043EA40
S214448DD0001392F8F00200F0010043EA401343F611
S214448DE05B7043EA841343F65D740B5443F65C733A
S214448DF0D2F8EC02CD54C0F3C923B2F8EE22C0F345
S214448E0047309B010855900943EA923343F65E7215
S214448E108B5443F65F73C8540220054B30BC93E82A
S214448E200600FAF7C3BD00BFA0744020087840206F
S214448E30FC704600104843F65871104A08B5B0F81E
S214448E40DC325BBA535290F8DE3203F00100C3F3CF
S214448E50400343EA400343F65A7013540A444FF41B
S214448E604470032102F06BFD054B022093E8060094
S214448E70BDE80840FAF79ABDA07440200878402020
S214448E80EC704600134843F65872134BB0F8D812A9
S214448E9049BA10B599521A4490F8DA1243F65A7001
S214448EA0C1F301041C54C1F3031443F65B70C1F3CD
S214448EB081011C5443F65C70195405214FF45470D8
S214448EC002F03DFD054B022093E80600BDE8104045
S214448ED0FAF76CBDA074402008784020E470460041
S214448EE0254943F65872B1F8E00238B540BA234BE8
S214448EF091F8E34298521A44D1F8E40204F001058A
S214448F00C4F34404C0F3C53040EAC51043F65A756A
S214448F10585543F65B75B1F8E402C0F3451058550E
S214448F2043F65C7591F8E402C0F304005855B1F872
S214448F30E602C0F3022500F4FC6045EAC40443F6A6
S214448F405D755C5591F8E542C4F3C304204343F68B
S214448F505E74185591F8E20243F65F71585408213E
S214448F604FF4617002F062FE054B022093E806005F
S214448F70BDE83840FAF71ABDA0744020087840206F
S214448F80F4704600094943F65870094AD1F8C0328D
S214448F901BBA13500220D1F8C43243F65C711BBA94
S214448FA05350044B93E80600FAF700BDA0744020E3
S214448FB008784020CC7046000E4845F6F062B0F87B
S214448FC0181308B549BA0C4B99521A4490F81A1318
S214448FD045F6F260C1F3000119540321332002F030
S214448FE025FE064B032093E80600BDE80840FAF742
S214448FF0DDBC00BFA0744020087840202C71460099
S214449000114B45F6F060114AB3F8081349BA10B547
S214449010115245F6F264B3F80A1393F80C3349BA7E
S21444902003F00103115345F6F4619B015354024483
S2144490300521402002F0E0FC054B032093E806009F
S214449040BDE81040FAF7B2BCA0744020087840202F
S214449050147146002248234A90F8001338B590F815
S214449060043345F6F064135545F6F163D15445F69A
S214449070F261D0F80033C3F34F235BBA535290F8EF
S2144490800513C1F34013C1F380151B0143EAC5031E
S214449090C1F341052B4390F8015305F0010543EA1B
S2144490A04513C1F3C10501F0010143EA851345F6B2
S2144490B0F4655355D0F804336520C3F3C13343EA0B
S2144490C0811145F6F563D1542244082102F0AEFDE1
S2144490D0054B032093E80600BDE83840FAF766BC23
S2144490E0A0744020087840200C71460038B52C4BBC
S2144490F045F6F0602B4AB3F8F412B3F8FC5249BA7A
S214449100115293F8FA12CC09C5F3032141EA04112B
S21444911093F8FD42C4F3001441EA441193F8F7422D
S214449120C4F3800441EA841193F8F942C4F38004FA
S21444913041EAC41145F6F264115545F6F361B3F8B5
S214449140F642555445F6F461C4F30905C4F387045E
S2144491505454B3F8F812D3F8F832C1F30904C1F3FF
S214449160051141EA851145F6F5655155C3F3CB2102
S214449170C3F3C34343EA041345F6F664135545F66E
S214449180F763D15402440821712002F04FFD064B88
S214449190032093E80600BDE83840FAF707BC00BF52
S2144491A0A0744020087840200471460008B5FEF7B5
S2144491B0E8FEFEF7FBFEFEF729FFFEF7C9FFFEF7C3
S2144491C0E3FFFFF72FF8FFF749F8FFF799F8FFF7A3
S2144491D0B5F8FFF7CBF8FFF7F1F8FFF72DF9FFF7EF
S2144491E075F9FFF70DFAFFF72FFAFFF751FAFFF775
S2144491F0E3F9FFF771FAFFF7A9FAFFF7E1FAFFF789
S21444920015FBFFF76BFBFFF703FCFFF7C9FBFFF704
S21444921029FCFFF757FDBDE80840FFF767BF284A1B
S21444922045F6F0602749B2F838335BBA30B40B528F
S21444923045F6F263B2F83A03B2F83C53C0F3090475
S214449240C0F38700C854C5F3012092F83B3303F0BB
S2144492500403034392F83D03C0F3800043EAC0038B
S21444926092F83E03C0F3401043EA001392F84003DA
S21444927000F0010043EA401345F6F36043EA8413E2
S21444928045F6F5640B5445F6F463D2F83C03CD54E6
S214449290C0F3C923B2F83E23C0F347309B010855B8
S2144492A0900943EA923345F6F6628B5445F6F763E3
S2144492B0C8540320044B30BC93E80600FAF776BB48
S2144492C0A07440200878402044714600104845F673
S2144492D0F061104A08B5B0F814335BBA535290F8AC
S2144492E0163303F00100C3F3400343EA400345F654
S2144492F0F26013540A444FF44470032102F07CFB9A
S214449300054B032093E80600BDE80840FAF74EBB39
S214449310A07440200878402024714600134845F63F
S214449320F062134BB0F8101349BA10B599521A4468
S21444933090F8121345F6F260C1F301041C54C1F3CD
S214449340031445F6F360C1F381011C5445F6F460FA
S214449350195405214FF4547002F04EFB054B03207C
S21444936093E80600BDE81040FAF720BBA0744020FE
S214449370087840201C714600254945F6F062B1F84D
S214449380300338B540BA234B91F8334398521A44C5
S214449390D1F8340304F00105C4F34404C0F3C530E3
S2144493A040EAC51045F6F265585545F6F365B1F8FA
S2144493B03403C0F34510585545F6F46591F8340324
S2144493C0C0F304005855B1F83603C0F3022500F440
S2144493D0FC6045EAC40445F6F5655C5591F83543AA
S2144493E0C4F3C304204345F6F664185591F8320393
S2144493F045F6F7615854082140F2853002F016FCD1
S214449400054B032093E80600BDE83840FAF7CEBA89
S214449410A0744020087840203C71460008B5FFF709
S2144494205FFDBDE80840FFF7A7BF08B5F8F70DFA9B
S214449430FEF714FCBDE80840FFF7F0BF094945F6BF
S214449440F060094AD1F828331BBA13500320D1F8E8
S2144494502C3345F6F4611BBA5350044B93E806008C
S214449460FAF7A4BAA0744020087840203471460025
S214449470114B47F68860114AB3F8441349BA10B5FD
S214449480115247F68A64B3F8461393F8483349BAF8
S21444949003F00103115347F68C619B015354024475
S2144494A00521402002F006FB054B042093E8060005
S2144494B0BDE81040FAF77ABAA074402008784020F5
S2144494C04C714600104847F68861104A08B5B0F813
S2144494D050335BBA535290F8523303F00100C3F34F
S2144494E0400343EA400347F68A6013540A444FF461
S2144494F04470032102F0DEFA054B042093E806008C
S214449500BDE80840FAF752BAA074402008784020D4
S21444951054714600134847F68862134BB0F84C1310
S21444952049BA10B599521A4490F84E1347F68A60D1
S214449530C1F301041C54C1F3031447F68B60C1F312
S21444954081011C5447F68C60195405214FF454701D
S21444955002F0B0FA054B042093E80600BDE810403C
S214449560FAF724BAA0744020087840205C7146007C
S21444957008B50A4B49F6226209494020B3F85633E7
S2144495805BBA8B520521074A02F0F2FA064B0520D5
S21444959093E80600BDE80840FAF708BAA0744020ED
S2144495A0087840202816412064714600134849F63E
S2144495B02062134BB0F8601349BA10B599521A4456
S2144495C090F8621349F62260C1F301041C54C1F3B7
S2144495D0810449F62360C1F303111C5449F6246000
S2144495E0195405214FF4547002F0C2FA054B052075
S2144495F093E80600BDE81040FAF7D8B9A0744020B6
S2144496000878402074714600104849F62061104A94
S21444961008B5B0F85C335BBA535290F85E3303F047
S2144496200100C3F3400343EA400349F6226013545F
S2144496300A444FF44470032102F09AFA054B05207D
S21444964093E80600BDE80840FAF7B0B9A074402095
S214449650087840206C71460008B5FFF739FAFFF7E2
S21444966059FAFFF781FAFFF7E7FAFFF7E3FBFFF74C
S21444967009FCFFF7A1FCFFF7C3FCFFF7EBFCFFF781
S21444968025FEFFF74BFEFFF7F3FEFFF71BFFFFF742
S21444969041FFFFF76DFFFFF7B7FFBDE80840FFF750
S2144496A085BF08B5FCF7C6FBF8F7B5F8FEF740FCEF
S2144496B0BDE80840FFF7D0BF704770477047704713
S2144496C0064AB2F82832B2F8681003F44043C1F3AD
S2144496D00D010B43A2F82832704700BFA074402007
S2144496E0044BB3F81221A3F82C22B3F80C21A3F8A8
S2144496F02E227047A0744020044BB3F8A620A3F84B
S2144497003422B3F8A020A3F836227047A074402031
S21444971070477047054BB3F86C21A3F83C22D3F846
S2144497206821C2F30F12A3F83E227047A07440206B
S214449730054BB3F87421A3F84422D3F87021C2F33E
S2144497400F12A3F846227047A0744020054BB3F886
S2144497506C21A3F8B821D3F86821C2F30F12A3F8FA
S214449760BA217047A0744020054BB3F87421A3F87F
S214449770C021D3F87021C2F30F12A3F8C221704758
S214449780A074402008B5FFF7E1FFFFF7EDFFFFF7B1
S21444979097FFFFF7A5FFFFF7AFFFFFF7BBFFBDE857
S2144497A00840FFF7C5BF08B5FCF76AFAF8F734F87F
S2144497B0FEF77CFAFFF7E6FFBDE80840FFF7F6BC85
S2144497C070477047704770470B4AD2F8C831D2F892
S2144497D094101B0DC1F313011B050B43D2F89810CC
S2144497E0C2F8C83101F47F11D2F8CC3123F47F1388
S2144497F00B43C2F8CC317047A074402008B5F9F743
S21444980075F9BDE80840F8F7BFBB7047F8F701B8EC
S214449810FFF747BFFFF7C7BFFBF71BBB7047074AB7
S2144498201378632B96BF01330023DBB21370044ACC
S214449830136801331360FEF7B4BE00BF08394120F5
S214449840C020402008B5FAF7CDF8BDE8084001F03E
S21444985045BD08B5FFF7E9FD4CF24053044AD058DD
S214449860B0FA80F0BDE808404009F9F7B9B900BF3E
S2144498700C394120014900201DF026BA389646008E
S21444988000201DF025BA0022114610461DF024BAC9
S214449890704700BF044B1A78044B1B78134302BF2F
S2144498A0034B02221A7070472F1840202B18402072
S2144498B030184020064B01221A70064B1B78934200
S2144498C004D1054A13707822044B1A80704700BFAF
S2144498D0E71A40202B184020E61A4020E41A40207D
S2144498E0074B08480849094A10B51B78084C012B11
S2144498F018BF0023237003700B70137010BD00BF95
S214449900E81A4020351840203418402033184020A8
S21444991036184020124B134870B51978124B01295B
S21444992000781C78114B124D1A78124B1B780CD1C8
S214449930012C0AD1012A08D1012B06D1012804D1D1
S214449940002328700C4A137070BD214300260A4336
S2144499502E70134303430CBF01233346F2E700BF84
S21444996038184020331840203618402035184020F8
S2144499703D184020341840203C184020044B012217
S2144499801A600022034B1A700322034B1A70704766
S214449990C82040203A1840203018402008B5FFF729
S2144499A09FFFFFF7B7FF044B1B78012B03D1BDE89D
S2144499B00840FFF7E3BF08BD3D184020054B1B7821
S2144499C0012B06D1044B1B78012B02BF034B00220C
S2144499D01A7070472B184020391840203018402001
S2144499E0094B1A78094B2AB909490878012804BF53
S2144499F01A700A70002207490A7007490A801A78C2
S214449A0001321A70704700BF2A184020E2174020DF
S214449A10E71A4020E61A4020E41A4020FFF77ABFAF
S214449A20124B70B51D78124B1C78124B1878124B9B
S214449A301978124B1A7845EA040303430B4313433D
S214449A400F4B04D101221A7100225A710CE00026F1
S214449A50012D5E71F8D1012CF6D10128F4D10129EB
S214449A60F2D1012AF0D11A7170BD00BF38184020D7
S214449A7036184020351840203418402033184020EB
S214449A80C8204020FFF7ACBF054B02221A70054B96
S214449A90054A1B78042B94BF002301231370704798
S214449AA0E71A4020F4174020E81A4020114B70B5BE
S214449AB01878114B01281D78104B1978104B1A78DA
S214449AC0104B1C78104B0BD1012D09D1012907D11D
S214449AD0012A05D1012C03D11C7100225A7108E0D9
S214449AE02843002601435E710A432243F5D10122EE
S214449AF01A7170BD3818402036184020351840205A
S214449B003418402033184020C820402008B5FFF7BA
S214449B1001FF0A4B1B68022B01D1FFF761FFFFF7D9
S214449B20B3FFFFF7C3FF064B1B78012B04D1054A4E
S214449B3000211160044A137008BD00BF141C402065
S214449B403C184020C82040203018402008B5FFF775
S214449B5067FFFFF745FFFFF797FFFFF795FFFFF710
S214449B60A5FF034B00229A600122024B1A7008BDDF
S214449B70C82040203018402038B504460D461046CC
S214449B80194609F0E7FE2B46224604F02DFF049BB7
S214449B90C3E9000138BD70B5064B1646002204469C
S214449BA00D4605F093F908B10024024DC6E9004578
S214449BB070BD00BF0080614070B5064B164600225B
S214449BC004460D4605F0A0F908B10024014DC6E947
S214449BD0004570BD008061C02DE9F04FBC4EBBB05F
S214449BE04FF00008DFF80C93D6E91C34CDE91E3458
S214449BF0B6F87E308BB9B06F04F07CFE42464B46D6
S214449C0004F0F2FE42464B4604460D4605F07CF907
S214449C10002801F00F80C6E930899BA3D3E90023CE
S214449C20D6E93645CDE9362320460022A94B2946B7
S214449C30D6E9348905F068F9002840F0FF87002209
S214449C40A54B2046294605F041F9002840F0FA87FE
S214449C5042464B462046294604F00EFD04460D4631
S214449C608BA3D3E90023CDE9384505F039F900281C
S214449C7000F0EC872046294687A3D3E9002305F065
S214449C8025F9002840F0E78742464B4620462946B9
S214449C9004F0F4FC02460B46CDE9222380A3D3E924
S214449CA0002304F0A1FE38AB024600930B46CDE9F0
S214449CB020018A49D1E90001FFF75EFF7AA3D3E980
S214449CC00023DDE9380104F08FFE79A3D3E90023AD
S214449CD004F08AFE0022824B04460D4605F014F931
S214449CE0002840F0BD87002200232046294605F080
S214449CF0EDF808B10024002520462946D6E9326707
S214449D0032463B4604F0B8FC04460D465EA3D3E90F
S214449D10002305F0E5F870B1204629460FF298195D
S214449D20D9E9008942464B4605F0D0F8002800F0B1
S214449D309B87CDE93689DDE936233046394604F03B
S214449D409DFC02460B46624ECDE938235CA3D3E91C
S214449D50002304F049FE0022624BD6E90245CDE9D1
S214449D6024012046294605F0B1F8002800F08087F3
S214449D70D6E912ABD6E90C675046594632463B46BE
S214449D8005F0AEF808B9B246BB46514B5046594664
S214449D90D3E97E6732463B4604F06EFC80468946ED
S214449DA049A3D3E9002305F0AFF8002800F06687FE
S214449DB03046394644A3D3E9002304F05FFC824688
S214449DC08B46434BD3E93812D3E90E67CDE90212EA
S214449DD0C3E97EABD3E9142330463946CDE906239E
S214449DE00022002305F068F8002800F05A87002275
S214449DF00023DDE9060105F073F850B100223A4B22
S214449E002046294605F076F818B100220023CDE90D
S214449E1002232F4ED6E90023CDE90E2396F8383296
S214449E20002B40F0968740F20113A6F83832DFF84C
S214449E30A08000220023DDE90201C8E9982300221D
S214449E402A4B05F039F8031E4FF00002204618BF8F
S214449E50012329460893264B05F042F8041E4FF08A
S214449E6000024FF0804318BF01245946504605F07F
S214449E7037F8089B00280CBF2046601C184404F0A2
S214449E8049FD39E0AFF30080FCA9F1D24D62903F22
S214449E90FCA9F1D24D62603FFCA9F1D24D6260BF8D
S214449EA0399D52A246DF913FE3A59BC420B0D23FE2
S214449EB0578C22C76075B53F7B14AE47E17AC4BF62
S214449EC09A9999999999E93FFCA9F1D24D62703FC4
S214449ED090FE412000002440000024C0D873460071
S214449EE000004E4000004940000059400000084031
S214449EF00000344000408F40D8E99A2304F0BEFB6B
S214449F000022BD4B04F0F6FF0022D8E986670028FD
S214449F1000F0428700233046394604F0CDFF18B19E
S214449F2000220023C8E98C23B44E0023B44C0022FC
S214449F30C6E98634D6E93034CDE90434C6E98834F3
S214449F40D6E98C45AF4B2046294604F0BFFF60B1A6
S214449F5020462946DDE92423C6E98A2394A3D3E987
S214449F60002304F08BFBC6E98C010023A44CC6E90D
S214449F7098340022A24BDDE9020104F09DFF00283C
S214449F8040F0528700229F4B0026DDE9020104F090
S214449F9093FF002800F04C87994F984900229A4B2B
S214449FA0D1E93A0104F020FD0022984B04F01CFD50
S214449FB00022974B04460D4604F0A6FF002840F0C6
S214449FC03A87002200232046294604F07FFF08B142
S214449FD00024002532463B462046294604F004FD2C
S214449FE0864B04460D46D3E9806732463B4604F02A
S214449FF043FB0022834B8046894604F085FF0022BB
S21444A000002800F01C877F4B3046394604F036FB68
S21444A01004460D46794B002220462946C3E980452E
S21444A0207B4B04F071FF002840F019870022002380
S21444A0302046294604F04AFF08B1002400250022A1
S21444A0404FF08043DDE91E0104F036FF002800F09F
S21444A0500A8700226F4BDDE9060104F0C5FC06467C
S21444A0600F460FF25419D9E9008942464B4604F08C
S21444A0704BFF002800F0FF86604BC3E990895F4B96
S21444A080DDE90412C3E9A045C3E99E120022002379
S21444A090DDE9020104F010FF0446002840F0FD8686
S21444A0A000224FF08043DDE9020104F005FF00285A
S21444A0B040F02C870022524BDDE9020104F0FCFEFE
S21444A0C0002840F025874F4B0022DDE9020104F0CA
S21444A0D0F3FE0023002840F07F87002400225046E9
S21444A0E05946CDE90C344A4B04F07EFC34A3D3E9FC
S21444A0F0002304F0A3FD34A3D3E9002304F074FC46
S21444A1000022454B04F070FC31A3D3E9002304F04D
S21444A11095FD04460D46089804F0FCFB02460B46A3
S21444A1202046294604F060FC02460B46CDE90A2345
S21444A130324BD3E9824522462B4604F09DFA064626
S21444A1400F4625A3D3E9002304F0DEFE002800F0E2
S21444A150E6862046294620A3D3E9002304F08EFA57
S21444A160CDE90A01254CDDE90A23DDE90A01C4E903
S21444A1708223D4E93C2304F081FA19A3D3E90023CB
S21444A18004F032FC06460F4617A3D3E90023D4E96D
S21444A1903E0104F029FC02460B463046394604F09C
S21444A1A06DFA13A3D3E9002338E000BFAFF3008071
S21444A1B07B14AE47E17A743F00000000007097407D
S21444A1C0000000000020AC405C8FC2F528DC27402D
S21444A1D0B46155D0CC38FB3F9A9999999999D93F0F
S21444A1E0FCA9F1D24D62603FB428207983A6BA3FD9
S21444A1F054434F56A8ACBB3F0000104090FE41204D
S21444A2000000F03F000008400000B03F000054C08B
S21444A21000408F400000594000004E4004F00EFDC0
S21444A22002460B46CDE90423D4E9402304F024FA3D
S21444A2300022C54B04F0D8FBD4E9422304F01CFAB0
S21444A24002460B46CDE91023D4E9442304F014FA1D
S21444A2500022BD4B04F0C8FBD4E9462304F00CFAB4
S21444A26002460B46CDE91223D4E9482304F004FA07
S21444A2700022B54B04F0B8FBD4E94A2304F0FCF9B9
S21444A28095A3D3E90023CDE92601DDE9040104F0D2
S21444A290ABFB06460F4692A3D3E90023DDE9100143
S21444A2A004F0A2FB32463B4604F0E8F98046894671
S21444A2B08DA3D3E90023DDE9120104F095FB0246A1
S21444A2C00B464046494604F0D9F9DDE9262304F016
S21444A2D0D5F987A3D3E9002304F086FBD4E94C23BD
S21444A2E0CDE914011046194604F0C8F9DDE91423F3
S21444A2F004F0C4F9D4E9202304F0C0F97EA3D3E9DA
S21444A300002304F071FB804689467DA3D3E90023ED
S21444A310D4E94E0104F068FB02460B4640464946E3
S21444A32004F0ACF98046894677A3D3E90023D4E900
S21444A330240104F059FB02460B464046494604F0C5
S21444A3409BF973A3D3E9002304F078FC02460B463A
S21444A350CDE91623D4E9502304F090F96EA3D3E94B
S21444A360002304F041FB804689466DA3D3E90023CD
S21444A370D4E9520104F038FB02460B4640464946AF
S21444A38004F07CF968A3D3E9002304F057FCDDE924
S21444A3900E23CDE92801DDE9040104F06DF900221D
S21444A3A06A4B04460D4604F0AFFD002840F0CA85CB
S21444A3B0204629465EA3D3E9002304F087FD0028FF
S21444A3C040F0D3850022624B2046294604F09CFD8B
S21444A3D0002800F0BB8500225D4B2046294604F049
S21444A3E04BF9804689465B4CDDE90401D4E95423A5
S21444A3F004F042F90022544B04F0F6FAD4E956230A
S21444A40004F03AF902460B46CDE91823D4E958231A
S21444A41004F032F900224C4B04F0E6FAD4E95A230D
S21444A42004F02AF902460B46CDE91A23D4E95C2304
S21444A43004F022F90022444B04F0D6FAD4E95E2311
S21444A44004F01AF926A3D3E90023CDE92A01DDE96D
S21444A450180104F0C9FA32463B4604F00FF90646A2
S21444A4600F4621A3D3E90023DDE91A0104F0BCFA20
S21444A47002460B463046394604F000F9DDE92A2305
S21444A48004F0FCF81AA3D3E9002304F0ADFAD4E9A7
S21444A490842304F0F1F802460B46CDE93223D4E98E
S21444A4A0602304F0EBF81CA3D3E9002304F09CFAE1
S21444A4B006460F4620A3D3E90023D4E9620104F0FC
S21444A4C093FA02460B463046394604F0D7F81CA3A6
S21444A4D0D3E9002340E000BF9A999999999963403B
S21444A4E09A99999999996A40CDCCCCCCCCCC3540A4
S21444A4F0E3F36EFB79D0E33E277845D92444D93F2D
S21444A500FB50D7647BD71C403043BB3975F10440BD
S21444A5106D0D4BFEC9AF1840FCA9F1D24D62603FA9
S21444A520EBF33CDE4AA2813FE9C8B5C771D3893F05
S21444A5300000000000409FC05ED817C2038C9E3FB8
S21444A5406F216A9B4B52A13F00408F4000409F4082
S21444A5500000494090FE412004F070FBD4E9642397
S21444A560CDE90E011046194604F088F8DDE90E23BD
S21444A57004F084F8D4E9282304F080F8B6A3D3E999
S21444A580002304F031FA06460F46B5A3D3E9002368
S21444A590D4E9660104F028FA02460B4630463946AA
S21444A5A004F06CF806460F46AFA3D3E90023D4E97B
S21444A5B02C0104F019FA02460B463046394604F09C
S21444A5C05BF8ABA3D3E9002304F038FB0022B84B76
S21444A5D0CDE91C01DDE9060104F078FC002840F0D2
S21444A5E0CE840022B24BDDE9060104F045F8A2A36E
S21444A5F0D3E9002304F0F8F90022AE4B04460D4696
S21444A60004F078FC002840F0BE84CDE936459CA38F
S21444A610D3E90023DDE91C0104F0E6F90022A64B49
S21444A6200C46064604F052FC0546002840F0B18429
S21444A6300022A24B3046214604F066FC002840F037
S21444A640AC84354604F10044404649468EA3D3E9DB
S21444A650002304F0C9F9DDE9282304F00FF8064680
S21444A6600F4628462146DDE9362304F0BDF9324636
S21444A6703B4604F003F802460B46CDE90823002285
S21444A6808F4B04F041FC002840F08A8400228D4B16
S21444A690DDE9080104F01AFC18B10023894CCDE921
S21444A6A0083400224FF08043DDE91E0104F004FC28
S21444A6B0002840F07984DDE90C23DDE9080104F044
S21444A6C093F9814EDDE90234C6E99601C6E9A6341B
S21444A6D050465946DDE9062303F0CEFFDDE924342F
S21444A6E0CDE93401C6E99434DDE922347749C6E934
S21444A6F09C3436ABD1E902010093DDE92023FFF711
S21444A7003BFAD6E96823D6E9040103F0B7FF60A311
S21444A710D3E9002304F068F904460D465EA3D3E962
S21444A7200023D6E96A0104F05FF902460B46204648
S21444A730294603F0A3FF5AA3D3E9002304F07EFA84
S21444A740D6E96C23CDE92401D6E9060103F096FF49
S21444A7504FA3D3E9002304F047F904460D464EA31D
S21444A760D3E90023D6E96E0104F03EF902460B46CF
S21444A7702046294603F082FF49A3D3E9002304F088
S21444A7805DFAD6E97023CDE90601D6E9080103F05F
S21444A79075FF3FA3D3E9002304F026F904460D468B
S21444A7A03DA3D3E90023D6E9720104F01DF902461D
S21444A7B00B462046294603F061FF39A3D3E900231C
S21444A7C004F03CFADDE90623CDE90C0110461946AF
S21444A7D004F00AF904460D46DDE90C2310461946F2
S21444A7E004F002F902460B462046294603F046FF8B
S21444A7F009F0F6F80022002304460D4604F05CFBFC
S21444A800002800F0D583CDE93645D6E93634DDE96F
S21444A8103601CDE91E3424A3D3E9002304F0E4F83A
S21444A82002460B46DDE91E0103F026FFD6E90A344C
S21444A830CDE92C01CDE92034DDE92001D6E97623A3
S21444A84003F01CFF12A3D3E9002304F0CDF804461A
S21444A8500D463DE0AFF300802ED7D19C0A49373FE2
S21444A8607119ABB745FF1F40ECBC164D8E930F4095
S21444A8701988C921F33610409A9999999999C93FEC
S21444A880CDCCCCCCCCCCEC3F3B08AA2A23DCA63F90
S21444A890FCA9F1D24D62603FFEF2469F2892AF3F3C
S21444A8A01F94D22C39CFB03FF8C1631ADCA54C4074
S21444A8B0000014400000F03F00003EC000003E4050
S21444A8C000005440000054C090FE4120D873460017
S21444A8D09FA3D3E90023D6E9780104F085F802461D
S21444A8E00B462046294603F0C9FE9BA3D3E9002322
S21444A8F004F0A4F900229C4BCDE92E01D6E91401BC
S21444A90004F072F802460B460020984903F0B4FE61
S21444A9100022974B0C460546954E04F0D7FA00287D
S21444A9200BBF28460020214631468DA3D3E9002399
S21444A93004F05AF88B468F498246D1E97A23D1E906
S21444A9401601CDE93023CDE936AB03F095FE00225F
S21444A95080468946864B2846214604F0B7FA0028A6
S21444A96040F0318304F1004442464B465046594633
S21444A97004F0C0FA88B12846214679A3D3E90023D7
S21444A98004F032F842464B4606460F4604F0A8FA10
S21444A990002840F01B83CDE93667DDE93623DDE940
S21444A9A0300103F06BFECDE930017249DDE9302316
S21444A9B0D1E97C89C1E9922342464B46D1E9180144
S21444A9C0CDE936AB03F058FE06460F4602460B4624
S21444A9D05046594604F08EFA88B12846214660A36C
S21444A9E0D3E9002304F000F832463B4604460D46BD
S21444A9F004F076FA002840F0EC82CDE93645DDE9ED
S21444AA00362340464946DFF86CA103F037FE044639
S21444AA100D46DDE93823DAE97489CAE93223DDE9EB
S21444AA20222340464946CAE93423CAE9A2450022BD
S21444AA30514B03F0D9FF06460F4600224F4BDDE943
S21444AA402C0103F0D1FF02460B463046394603F04C
S21444AA5015FE02460B46DDE92E0103F00DFE40A32B
S21444AA60D3E9002303F0C0FFDDE91E2303F006FE0E
S21444AA70DDE90223CAE93601CAE93823DAE93A01AC
S21444AA8000223F4B03F0B0FFDDE9342303F0F6FD2C
S21444AA90DDE90A23CAE93A01CAE93C23DDE904238D
S21444AAA0CAE93E23CAE94023DDE91023CAE9422322
S21444AAB0CAE94423DDE91223CAE94623CAE94823FE
S21444AAC0DDE92623CAE94A23DDE91423CAE94C23EF
S21444AAD0DAE92223CAE92023DDE91423CAE922233A
S21444AAE0DDE91623CAE94E23DAE92623CAE92423F4
S21444AAF0DDE91623CAE92623CAE95023DDE92823DB
S21444AB00CAE95223DDE90823CAE98423DDE904239C
S21444AB10CAE95423DDE91823CAE95623CAE9582367
S21444AB20DDE91A23CAE95A23CAE95C23DDE92A2364
S21444AB30CAE95E23DDE93223CAE96023DDE90E2350
S21444AB40CAE96223CAE96423DAE92A231AE000BF81
S21444AB50FEF2469F2892AF3F1F94D22C39CFB03F87
S21444AB60FCA9F1D24D62603F00001A4000007940D3
S21444AB700080614090FE412000001440000059408F
S21444AB800000EE3FDDE92C01CAE92823DDE90E2367
S21444AB90CAE92A23DDE91C23CAE96623DAE92E2317
S21444ABA0CAE92C23DDE91C23CAE92E23DAE9042367
S21444ABB0CAE96823DDE92423CAE96A23DAE90623D5
S21444ABC0CAE96C23DDE90623CAE96E23DAE90823D9
S21444ABD0CAE97023DDE90C23CAE97223B2A3D3E998
S21444ABE0002303F001FF42464B4603F047FDDDE9F0
S21444ABF02023CAE97401CAE97623DDE92E23CAE98B
S21444AC007C45CAE97823DDE93023CAE97A23BAF8D1
S21444AC107E3023B9DAF878200132CAF87820013336
S21444AC209BB2B3F5FA7F28BF0023AAF87E303BB028
S21444AC30BDE8F08FC6E93045FEF7EFBF0024A84DC7
S21444AC40FFF706B80024A74DFFF702B896A5D5E946
S21444AC500045FFF719B896A5D5E90045FFF714B89F
S21444AC600024A14DFFF748B8CDE93645FFF763B851
S21444AC704FF0000A4FF0000BFFF787B88EA3D3E9D6
S21444AC8000234046494604F021F900283FF499A899
S21444AC90304639468AA3D3E9002303F0EDFCFFF798
S21444ACA08EB8DDE9020104F04FF903283FF6B1A857
S21444ACB0DFE800F002472A4700220023DDE90601C8
S21444ACC004F00EF900283FF4A4A80022874B30462F
S21444ACD0394604F0F1F80022002836D1844B304639
S21444ACE0394604F0E9F800224FF0804300287FF408
S21444ACF08EA83046394604F0DFF800283FF489A889
S21444AD00CDE90267FFF785B800220023DDE9060196
S21444AD1004F0E6F800283FF47CA80022754B204651
S21444AD20294604F0E7F800283FF473A800226F4B46
S21444AD303046394604F0C0F80028E1D100226C4B76
S21444AD40D7E700224FF08043D3E74FF08043FFF726
S21444AD505EB896F83932012B11D10022664BDDE9F4
S21444AD600E0104F0B3F820B1022386F83932FFF717
S21444AD705EB800220023C6E99A23FFF758B852A3C8
S21444AD80D3E90023DDE90E0104F0BEF808B101233F
S21444AD90EBE70022554BEEE7544B3046394604F079
S21444ADA08BF800283DD0D8E98A23D8E9100104F06E
S21444ADB0A1F850B3D8E9884545A3D3E900232046F3
S21444ADC0294603F011FE02460B462046294603F068
S21444ADD053FC04460D4640A3D3E9002304F076F81A
S21444ADE040B9C8E98845454BD3E98834CDE90434AD
S21444ADF0FFF7BFB800230024C8E98834C8E986347E
S21444AE00C8E98A34C8E98C34EDE7D8E93034CDE96A
S21444AE100434C8E988340023344CC8E99834FFF72E
S21444AE20A8B800230024E1E70026354FFFF7B5B85D
S21444AE300027FFF7B2B80024324DFFF7CBB8324BA9
S21444AE404046494604F042F800283FF4E3A800226E
S21444AE50274B3046394603F00FFCFFF7D9B8002499
S21444AE60284DFFF7ECB822462B46DDE9040103F0F3
S21444AE7005FCFFF7F4B8002300223046394604F0B8
S21444AE8025F81E4B28B100210022C3E99012FFF793
S21444AE90F6B8C3E99067FFF7F2B800230893002397
S21444AEA0FFF71BB9AFF30080FCA9F1D24D62603FB7
S21444AEB0FCA9F1D24D6260BFFCA9F1D24D6280BFBD
S21444AEC0FCA9F1D24D62803F0000000000C0624001
S21444AED09A9999999999A93F7B14AE47E17A843F08
S21444AEE000002440000024C000004E400000F03F14
S21444AEF00000084000005940000049C090FE412030
S21444AF000000F0BF00408F40000008C00894C6E729
S21444AF104FF0FF33384C08930023FFF7DFB830A3D5
S21444AF20D3E900233046394603F0D0FF00283FF4E7
S21444AF3019A9204629462CA3D3E9002303F09CFBF9
S21444AF40FFF70EB900242D4DFFF745BA00222C4BCF
S21444AF502046294603F0CEFF58B90022294B204606
S21444AF60294603F08BFBFFF73CBA21A5D5E90045FB
S21444AF70F3E74FF000084FF00009FFF734BA002417
S21444AF800025FFF742BB00231F4CCDE93634FFF7BC
S21444AF903EBB00251D4CFFF757BB1D4CFFF754BB6B
S21444AFA000231C4CFFF77BBB00200021FFF789BB26
S21444AFB022462B46DDE9240103F040FE08F0F4FA6D
S21444AFC0CDE9360121E40025134CCDE4CDE936899C
S21444AFD0E3E4CDE9366712E50B4CFFF77FB800BFD4
S21444AFE09A9999999999E9BF9A9999999999E93F1A
S21444AFF00000000000409FC00000F0BF00409F409B
S21444B000000049C0000049400000F03F00003E40B8
S21444B01000003EC000005440008061C07047704746
S21444B02038B5454B454C1D78002D55D1444B1868D2
S21444B03003F082FC434BC4E90201186803F05AFC4F
S21444B0400022414BC4E91223404BC4E90C01186862
S21444B05003F050FC3E4BC4E90E01186803F06CFC48
S21444B0603C4BC4E91601186803F066FCC4E91801B1
S21444B070394B1B78002B5BD1384B186803F05CFCCB
S21444B080374BC4E91001186803F056FCC4E90001C4
S21444B090284603F02FFC334BC4E91C01186803F020
S21444B0A04BFC314BC4E91401186803F045FC2F4BA4
S21444B0B0C4E90401186803F03FFC2D4BC4E90601BB
S21444B0C0186803F039FC2B4BC4E90801186803F0F0
S21444B0D033FCC4E90A0138BD012D22D1264B186839
S21444B0E003F02AFC254BC4E90201186803F002FC6D
S21444B0F0234BC4E90C01186803F0FCFB214BC4E95C
S21444B1001201186803F0F6FB1F4BC4E90E011868D9
S21444B11003F012FC00220023C4E91601C4E91823F4
S21444B120A6E7022DA4D100220023C4E90C239FE7FE
S21444B13000200021A4E700BF2618402090FE4120AE
S21444B140601D4020681D402000004440381D4020BB
S21444B150541D4020501D40202C184020101E4020D6
S21444B160141E4020301C4020C41E4020E41E4020B4
S21444B170A81E4020B41E40207C1F4020641F402050
S21444B180341F40204C1F4020701F40202DE9F74FAD
S21444B190414CDFF83881DFF838B1DFF838A1DFF802
S21444B1A03891D4E9000103F017FF3C4B054618607C
S21444B1B0D4E9060103F010FFC8F80000D4E90401FE
S21444B1C003F00AFF364B1860D4E9020103F004FF8B
S21444B1D00746CBF80000CAF80000D4E9120103F091
S21444B1E0FBFE304BC9F8000006461860D4E9160149
S21444B1F003F0D2FE2C4A2D4904461060384601918D
S21444B20004F004FA274BCDF80080984628B10199FB
S21444B210CBF80010CAF8001006E0254938460191DC
S21444B22004F0D6F90028F2D1224F3046394604F0CD
S21444B230EDF920B1C9F80070C8F8007006E01E4F5A
S21444B2403046394604F0C4F90028F3D11B4B1B782A
S21444B2506BB91B4B24F002041968012C194C0AD113
S21444B260284603F00FFF206003B0BDE8F08F012BA3
S21444B27003D1154BEEE72160F6E7022B02D1114BC2
S21444B2801D60F1E7032BEFD10023009A13600E4BA9
S21444B2901A680C4B1A60E7E7D00042206C1F402027
S21444B2A07C17402054184020141C40200000E143E2
S21444B2B00000E1C300004843000048C3261840206D
S21444B2C0601D4020741F40207C1F4020181B4020D7
S21444B2D048194020DC1840206C184020F8B5174B1D
S21444B2E0174C1E78174D66B1012E19D00021002048
S21444B2F0F6F7EAFA00210120F6F7E6FA00232B7067
S21444B3000CE02678002EF1D100213046F6F7DCFA20
S21444B3100D490120F6F7D8FA01232E702370F8BDA4
S21444B3202F78002FE2D108493846F6F7CDFA0021A7
S21444B3303046F6F7C9FA2E702770F0E726184020F4
S21444B340B0174020B11740200000C8422D4A2E496D
S21444B350106810B550B90B68012B07D12B48036011
S21444B3602B4803602B4803602B4803602B4B50202C
S21444B37018602B4B2B4818602B4B1B6813602B4BC9
S21444B3801B780B602A4B1C6874B92A4B002118683A
S21444B39004F014F988B1284B07221A600122274B7F
S21444B3A01C60274B1A6008E0012C07D10223224A6E
S21444B3B01360224A1360224A136010BD022C0FD138
S21444B3C01C4B0021186804F0F9F80028F5D01A4BF5
S21444B3D003221A600022194B1A60194B1C60ECE7D2
S21444B3E0032CEAD1134B0021186804F0E7F8002830
S21444B3F0E3D0114B04221A600122104B1A60022239
S21444B4000F4BCFE7F81A4020F41A4020041B402084
S21444B410081B40200C1B4020101B4020F01A4020E4
S21444B420EC1A4020000048C284194020C21D402027
S21444B430141C4020301C4020001B4020FC1A402096
S21444B440201B40200000000038B5174B00211C6824
S21444B450204604F0BDF808B104F10044134D2046DC
S21444B4602C6003F069FA0CA3D3E9002303F0E6FB4F
S21444B4700BA3D3E9002303F0B7FA00220C4B03F0E6
S21444B480B3FA0C4B002203F0D9FB03F0A5FD0A4B9C
S21444B4906860186038BD00BF5C8FC2F528DC274062
S21444B4A0B4A766033D39FB3F141E4020D4204020F9
S21444B4B000004E4000408F40301C4020244B1B6808
S21444B4C0012B244B0BD0244A1288012A07D0234A46
S21444B4D01068012803D0224A1268012A0CD102229D
S21444B4E01A601B681F4A13701F4B1B78013B012BC5
S21444B4F02CD80323137070471C4A11681C4A012930
S21444B500126807D1196803291BD1002AE8D0012AFA
S21444B510E7D118E0012A06D1186803280ED100297D
S21444B520DFD10122DCE719B9196809B90322D7E744
S21444B530002AD6D11A68012AD3D1F7E70029F3D0D6
S21444B540CFE7012AF4D10028EBD0CAE7704700BF02
S21444B550441F4020101C4020CC174020341D40205F
S21444B560541F402026184020EE174020441D4020FB
S21444B570501F402008B5FEF733FA144B1B886BB9AE
S21444B580134B144A1B681268134307D1124A1360BC
S21444B590124A1360124A1360124A13600023124A76
S21444B5A001211360114A1360114A1360114A136053
S21444B5B0114A1360114A1360114A1360114A13600A
S21444B5C0114A1160114A136008BD00BFCC174020D1
S21444B5D0441F4020341D4020281D4020241D402068
S21444B5E0001A4020041A4020181C4020C41A402048
S21444B5F0201D40201C1D4020181D4020141D4020A6
S21444B600101D40200C1D4020081D4020041D4020D5
S21444B61008B5FEF74FF9044B1B68012B1EBF034BBE
S21444B62000221A6008BD00BF341D4020C41A4020C2
S21444B63008B5FEF73FF9064B1B68012B1EBF054BAA
S21444B64000221A60044B1A68044B1A6008BD00BFF7
S21444B650441F4020181C4020341F40202C1C4020EF
S21444B660F8B5124A0223124F1360124E124A3B6038
S21444B670136033600123114D114C2B602360FEF799
S21444B680AFF9104B1B887BB90F4B104A1B681268E6
S21444B69013430F4A1268134306D103223B603360B8
S21444B6A02B6023600B4B1A60F8BD00BF201B402064
S21444B6B0281D4020241D4020141C4020181C4020D7
S21444B6C0C41A4020CC174020441F4020341D40203C
S21444B6D0541F4020101C402008B5174B186803F030
S21444B6E09FFF164B164A186001231360154A1360D1
S21444B6F0154A1360154A1168154A1160154A1649C9
S21444B7001370164A1370164A1370164A1370164A64
S21444B7101370164A137000220A7015490A701549A8
S21444B7200B7015490B7015490B7015490B70154B6A
S21444B7301A70154B1A7008BD181B4020301A40204A
S21444B7402C1A40201C1A4020C0184020141C4020AC
S21444B750C81840205419402091184020E81840202A
S21444B76046194020DA18402001194020001940208C
S21444B77090184020691840206518402066184020DC
S21444B780501840204C1840204D18402000230A4AA8
S21444B79015211370094A1370094A11700621094A83
S21444B7A01370094A1370094A1170094A1370182213
S21444B7B0084B1A70704700BFF2184020F11840201A
S21444B7C0F0184020EF184020EE184020ED18402096
S21444B7D0EC184020EB18402008B5FFF77DFFFFF734
S21444B7E0D5FFFFF76BFEFFF71BFCFEF7F5F9FFF7F7
S21444B7F0CDFC0D4B1B781BB9BDE80840FFF708BFCE
S21444B800012B03D1BDE80840FFF712BF022B03D13A
S21444B810BDE80840FFF724BF032B03D1BDE808402A
S21444B820FFF7A8BE08BD00BF26184020074B1922C4
S21444B8301A600522064B1A600F22064B1A60022233
S21444B840054B1A60054B064A1A607047641B402035
S21444B850601B40205C1B4020581B4020541B40204B
S21444B860EFAB030008B5074B186803F0BBFC064B68
S21444B8700649186003F0B6FE10B1054B03221A7051
S21444B88008BD00BFBC1D4020181840200000F041F1
S21444B8901C184020034B044A9B6FC3F309231370C0
S21444B8A0704700BFA0744020F4174020084B1B7814
S21444B8B0013B022B0AD80023064A00211370064A8D
S21444B8C01160064A13700322054B1A60704700BF86
S21444B8D0EE174020ED174020181B4020EC17402060
S21444B8E0101C4020044B054A1B781370013B012B67
S21444B8F001D8FFF7DBBF7047C81D4020EE17402035
S21444B900FE28D4BF01300020704770B50022FF23C4
S21444B910064ED4B2551C8C4202D3D843C0B270BD36
S21444B920025D53402A46F35CF3E700BFE8734600E3
S21444B9300721013008B5FFF7E8FFC0B208BDB0F5EF
S21444B940447F38B5144617D1244D204695F8DC324A
S21444B950FF2B14BF01330023DBB285F8DC3253706F
S21444B9601F4A1370FFF7E4FF1E4BC0B285F8DD0292
S21444B97020701870012038BD402818D0B0F5547F88
S21444B980F8D1164D204695F8D832FF2B14BF013314
S21444B9900023DAB285F8D8226270134A1360FFF7A0
S21444B9A0C7FFC0B2114B85F8D902207014E00B4D86
S21444B9B0204695F8D032FF2B14BF01330023DAB269
S21444B9C085F8D02262700A4A1360FFF7B1FF094B2C
S21444B9D0C0B285F8D10220701860CBE7A07440202E
S21444B9E00319402002194020FC184020F818402033
S21444B9F0501940204C194020402838B5144616D1DA
S21444BA00254D204695F80833FF2B14BF01330023F9
S21444BA10DAB285F808236270204A1360FFF788FF7D
S21444BA201F4BC0B285F809032070186005E0B0F5D6
S21444BA30547F04D0B0F5447F17D0012038BD164D4E
S21444BA40204695F81033FF2B14BF01330023DAB297
S21444BA5085F810236270134A1360FFF769FFC0B27B
S21444BA60114B85F811032070DFE70B4D204695F8FF
S21444BA701433FF2B14BF01330023DBB285F8143391
S21444BA8053700A4A1370FFF753FF094BC0B285F848
S21444BA90150320701870D0E7A0744020E4184020A6
S21444BAA0E01840208C1840208818402093184020E6
S21444BAB092184020402838B5144617D1254D2046C4
S21444BAC095F80833FF2B14BF01330023DAB285F808
S21444BAD044236270204A1360FFF72AFF1F4BC0B20C
S21444BAE085F8450320701860012038BDB0F5547FB2
S21444BAF018D0B0F5447FF7D1164D204695F850330C
S21444BB00FF2B14BF01330023DBB285F85033537048
S21444BB10134A1370FFF70CFFC0B2124B85F851035B
S21444BB20207014E00B4D204695F84C33FF2B14BF81
S21444BB3001330023DBB285F84C3353700A4A137042
S21444BB40FFF7F6FE094BC0B285F84D032070187017
S21444BB50CAE700BFA07440207418402070184020E4
S21444BB606818402067184020641840206318402016
S21444BB70402838B5144616D1254D204695F85433FA
S21444BB80FF2B14BF01330023DAB285F854236270C6
S21444BB90204A1360FFF7CCFE1F4BC0B285F855030E
S21444BBA02070186005E0B0F5547F04D0B0F5447FAB
S21444BBB017D0012038BD164D204695F86033FF2B2C
S21444BBC014BF01330023DAB285F860236270134A47
S21444BBD01360FFF7ADFEC0B2114B85F861032070C9
S21444BBE0DFE70B4D204695F85C33FF2B14BF01333B
S21444BBF00023DBB285F85C3353700A4A1370FFF7B0
S21444BC0097FE094BC0B285F85D0320701870D0E7E4
S21444BC10A07440205C184020581840204818402003
S21444BC20441840204F1840204E184020502870B5E5
S21444BC300546144616D18C4A92F8AC31FF2B14BFF5
S21444BC4001330023D9B282F8AC11884A21711360BB
S21444BC5040F285339D4200F0DD80162D00F0F080E2
S21444BC60012070BD642826D065283BD032284FD0AA
S21444BC70702863D0712877D0332800F08C806A28E7
S21444BC8000F09F80B0F5617FE2D1774D204695F86D
S21444BC90E032FF2B14BF01330023DBB285F8E032D9
S21444BCA05370734A1370FFF743FEC0B2714B85F866
S21444BCB0E10220706DE06C4E204696F89C32FF2BD5
S21444BCC014BF01330023DBB286F89C3253706A4AB1
S21444BCD01370FFF72DFE694BC0B286F8A0022070A1
S21444BCE01870B5E7604E204696F80033FF2B14BF15
S21444BCF001330023DBB286F800335370604A137076
S21444BD00FFF716FEC0B25F4B86F804032070E7E7E1
S21444BD10554E204696F8B432FF2B14BF0133002309
S21444BD20DBB286F8B4325370574A1370FFF700FEFE
S21444BD30C0B2564B86F8B5022070D1E74A4E20462C
S21444BD4096F8A832FF2B14BF01330023DBB286F8E3
S21444BD50A83253704E4A1370FFF7EAFDC0B24D4BFB
S21444BD6086F8A9022070BBE73F4D204695F8F4328A
S21444BD70FF2B14BF01330023DBB285F8F432537033
S21444BD80454A1370FFF7D4FD444BC0B285F8F5021C
S21444BD902070187064E7344D204695F81833FF2B0E
S21444BDA014BF01330023DBB285F8183353703C4A82
S21444BDB01370FFF7BDFDC0B23A4B85F819032070E7
S21444BDC0E7E7294D2046D5F8C832D5F8C822C3F34C
S21444BDD0C733FF2B14BF01330023DBB263F3D632E1
S21444BDE0C5F8C8226370D5F8C8322F4AC3F3C733A0
S21444BDF01360FFF79DFDB5F8CA32C0B22B4A60F314
S21444BE00CE13A5F8CA322070B5F8CA32C3F3C713A6
S21444BE10136025E7144D2046254A95F83033FF2B0A
S21444BE2014BF01330023DBB285F8303363701370DC
S21444BE30FFF77EFDC0B21F4B85F831032070A8E79C
S21444BE400949B1F89822C2F34313013303F00F03B0
S21444BE5063F34812A1F898226370B1F89832164AF0
S21444BE60C3F34313D4E700BFA0744020E41B402030
S21444BE70F4184020F3184020441940204519402027
S21444BE80D8184020D918402056194020551940202B
S21444BE902519402024194020B5184020B4184020C5
S21444BEA0EA184020E9184020381940203419402028
S21444BEB08118402080184020801A40200F28D4BF84
S21444BEC001300020704770B50022FF23074ED4B2DD
S21444BED0551C8C4205D3DB4383EA131303F00F004F
S21444BEE070BD025D53402A46F35CF0E7E8744600B2
S21444BEF00721013008B5FFF7E6FFC0B208BDB0F52C
S21444BF00AE6F70B5054614461AD1C04D204695F816
S21444BF100D221309013363F3071203F00F0385F868
S21444BF200D22BB4A1360FFF7E3FF95F80E3260F329
S21444BF30030300F00F0085F80E32B64B1860C0E0DD
S21444BF40B0F5B06F1DD0B0F5B26F35D1AF4D2046C9
S21444BF5095F81E2202F00F03013363F3030203F045
S21444BF600F0385F81E22AC4A1360FFF7C1FF95F80D
S21444BF701E3260F3071300F00F0085F81E32A74BFD
S21444BF80DCE7A24D2046B5F81422C2F383130133EE
S21444BF9063F3891203F00F03A5F81422A04A136032
S21444BFA0FFF7A6FF95F8153260F3850300F00F00FF
S21444BFB085F815329B4BC1E740F29553984222D000
S21444BFC040F28553984258D050287CD0512835D1D9
S21444BFD08E4D204695F8382202F00F03013363F362
S21444BFE0030203F00F0385F838228F4A1360FFF7E5
S21444BFF07FFF95F8383260F3071300F00F0085F89A
S21444C00038328A4B9AE7814E204696F82322C2F36A
S21444C0108303013303F00F0363F3850286F8232278
S21444C020834A1370FFF764FF96F8243200F00F003B
S21444C03060F3030386F824327E4B1870602D5DD07F
S21444C040612D35D1714D204695F8482202F00F03F4
S21444C050013363F3030203F00F0385F84822764A5C
S21444C0601360FFF745FF95F8483260F3071300F076
S21444C0700F0085F84832714B60E7644E2046D6F888
S21444C0802822C2F38333013363F3913203F00F0360
S21444C090C6F828226A4A1360FFF72AFF96F82A321F
S21444C0A060F3850300F00F0086F82A32654B18606B
S21444C0B0132D3ED0142D57D0152D70D0162D00F0CC
S21444C0C08980012070BD514D204695F8302202F0FB
S21444C0D00F03013363F3030203F00F0385F83022A2
S21444C0E0594A1360FFF704FF95F8303260F307139C
S21444C0F000F00F0085F83032544B1FE7434D20467E
S21444C10095F8402202F00F03013363F3030203F071
S21444C1100F0385F840224E4A1360FFF7E9FE95F870
S21444C120403260F3071300F00F0085F84032494B65
S21444C13004E7364D2046B5F85222C2F38313013342
S21444C14063F3891203F00F03A5F85222424A1360A0
S21444C150FFF7CEFE95F8533260F3850300F00F00E8
S21444C16085F853323D4BE9E6284D204695F85A2249
S21444C17002F00F03013363F3030203F00F0385F861
S21444C1805A22374A1360FFF7B3FE95F85A3260F3E3
S21444C190071300F00F0085F85A32324BCEE61B4D9B
S21444C1A0204695F8622202F00F03013363F303023C
S21444C1B003F00F0385F862222B4A1360FFF798FEBC
S21444C1C095F8623260F3071300F00F0085F8623288
S21444C1D0264BB3E60D4D2046B5F89822C2F34313DA
S21444C1E0013363F3481203F00F03A5F89822204A5C
S21444C1F01360FFF77DFE95F8993260F3440300F030
S21444C2000F0085F899321B4B98E600BFA074402077
S21444C2109819402094194020D81D4020D41D402011
S21444C220901D40208C1D4020601A40205C1A4020FF
S21444C2306519402064194020401A40203C1A40208A
S21444C2406C19402068194020701A40206C1A40200F
S21444C250501A40204C1A4020C01A4020BC1A402095
S21444C260A01A40209C1A4020881A4020841A402055
S21444C270801A40207C1A402038B53E4B1A783E4BF4
S21444C2801B7813433ED13D4B1B78013B18BF01231B
S21444C2903B4A13703B4B1A683B4B1B6813433B4B60
S21444C2A014BF012200221A70394B1A78394B1B7876
S21444C2B01343394B14BF012200221A70374B384AB5
S21444C2C01B78013B18BF01231370364B364A1B7844
S21444C2D0003B18BF01231370344B354A1B78003B90
S21444C2E018BF01231370334B1C789CB9324D2B78FE
S21444C2F0012B09D1314B1C70FFF798FABDE8384042
S21444C300FFF7B0BA0123C3E7022B21D1BDE838407A
S21444C310FDF71CBC012C20D1274B1B78012B05D1E3
S21444C320264A1370BDE83840FDF7B4BA022B03D151
S21444C330BDE83840FDF732BB032B0ED1FFF74CFA6D
S21444C340FFF7D0FAFFF702F8BDE83840FFF77CB8AD
S21444C350032B03D1FFF79EFA2C7038BD002BFCD17B
S21444C360174A01211160174A1360BDE83840FDF7AB
S21444C370CDBB00BF8A1D4020891D4020C01D4020E3
S21444C3802F184020341E4020301E40202C184020B9
S21444C390791D4020781D40202D184020C11D402086
S21444C3A02E184020C21D40202B184020CC1D402073
S21444C3B02A1840203118402030184020E81A4020DF
S21444C3C0201B4020141C40207047704730B53D4C1D
S21444C3D085B03D48237801A90193019B1B02019334
S21444C3E0019A637813440193019B1B020193019ABB
S21444C3F0A37813440193019B1B020193019AE378AB
S21444C4001344019323790293029B1B020293029ADC
S21444C410637913440293029B1B020293029AA37904
S21444C42013440293029B1B020293029AE379134439
S21444C4300293237A0193019B1B020193019A637A28
S21444C44013440193019B1B020193019AA37A13445C
S21444C4500193019B1B020193019AE37A13440193CF
S21444C460237B0293029B1B020293029A637B134430
S21444C4700293029B1B020293029AA37B13440293E9
S21444C480029B1B020293029AE37B1344029342F2FA
S21444C4901273019342F21373029300F0B0FB04F15B
S21444C4A0100004F1080104F11802082314F8015B93
S21444C4B0013B00F8015B11F8015B02F8015BF5D122
S21444C4C005B030BD30014220808080000C4A0823ED
S21444C4D0002102F1280030B402F1080502F12004DC
S21444C4E0013B02F8011B05F8011B13F0FF0304F897
S21444C4F0011B00F8011BF3D130BCFFF767BF00BF38
S21444C500300142204F4BF0B51B688BB002934E4B24
S21444C5101A6803925A6804929B68059342F212730F
S21444C520029A9A4200F08980484800F013FBFFF7CD
S21444C530CDFF002346480AAA50F8231002EB830294
S21444C5400133082B42F8201CF5D1002340480AAAA0
S21444C55050F8231002EB83020133082B42F8201CC8
S21444C560F5D102990025039A049B0598394C00900E
S21444C5703948264600F0EEFA029B38481B0E2370D4
S21444C580029B1B0C6370029B1B0AA370029BE37006
S21444C590039B1B0E2371039B1B0C6371039B1B0A9B
S21444C5A0A371039BE371049B1B0E2372049B1B0C19
S21444C5B06372049B1B0AA372049BE372059B1B0EC7
S21444C5C02373059B1B0C6373059B1B0AA373059B74
S21444C5D0E37300F0B6FA013516F8010B00F0DAFA08
S21444C5E0082DF8D11E4D002600F0CBFA1D482F46E4
S21444C5F000F0A7FA013617F8010B00F0CBFA082E24
S21444C600F8D100F0BEFA184B002203F1080703F1F4
S21444C610100003F118019446013214F8016B15F822
S21444C62001EB082A03F8016B07F801EB00F8016BED
S21444C63001F801CBF0D10BB0F0BD0C4800F08AFAFB
S21444C64077E700BF80808000848080004A7B460075
S21444C65010808000300142206E7B46008B7B460073
S21444C66038014220957B460040014220607B4600CC
S21444C670194A08211948F0B592F8A53100F1100C72
S21444C68000F1080500F11807012B9CBF002382F82F
S21444C690D431002310F8014B01391CF8016B17F80C
S21444C6A001EBB4422E7818BF013344EA060418BF9F
S21444C6B0DBB2764505F8014B1CBF0133DBB211F003
S21444C6C0FF01E7D133B1B2F8BE301BB9BDE8F04044
S21444C6D0FFF77CBEF0BD00BF6C0142203001422013
S21444C6E01FB5144B01A953F820305A1E073312F8CD
S21444C6F0010F9A4201F8010BF9D19DF80430002449
S21444C700502B8DF80C4007D0432B0CD0422B0DD029
S21444C710552B08BF4FF440040DF1050000F04CFAC9
S21444C720204404B010BD4FF48004F5E74FF40004F1
S21444C730F2E700BFDC2040202DE9F04F5C4D8DB081
S21444C74082462B6805F1080806AC09A963F07C43C9
S21444C75040462E46A9462B604246082316F8017BDF
S21444C760013B04F8017B9BB210F8017B01F8017B86
S21444C770002BF3D1BAF10A0F0BD141464C4C082397
S21444C780FF20013B04F8010B01F8010B9BB2002B80
S21444C790F7D1484BC8240021013C03F8011BA4B23E
S21444C7A0002CF9D126464449DFF808B104F10803C1
S21444C7B080279BB200932B781F4203D198F8003011
S21444C7C01F4248D051F824300DF10C0C581E073344
S21444C7D010F801EF98420CF801EBF9D14FF0000342
S21444C7E08DF814309DF80C30502B59D0432B59D02B
S21444C7F0422B5AD0552B34D14FF440030DF10D0043
S21444C800019300F0D9F9019B95F800C0184498F8B4
S21444C81000302A4A3B404FEA102E274918BF0823C7
S21444C82017EA0C0F4FEA104C18BF43F001030BF8FD
S21444C83006C006F1010C1FFA8CFC0BF80CE006F15E
S21444C840020C1FFA8CFC0BF80C00F01C043680B269
S21444C850B6B20BF800300134009B7F08A4B2A34262
S21444C860A9D1013508F1010895429FD1BAF10A0FC2
S21444C8700FD19DF81A30BDF8182089F80230A9F86F
S21444C88000209DF82630BDF8242089F80A30A9F8FF
S21444C8900820084B002230469A550DB0BDE8F08F6C
S21444C8A00023ABE74FF48003A8E74FF40003A5E763
S21444C8B03001422012224020DC2040203801422011
S21444C8C0F0B50D4C0822002004F1080514F8016B5D
S21444C8D0082380210E4202D12F78394201D00130FC
S21444C8E080B2013B49089BB2002BF3D1013A013593
S21444C8F092B2002AEAD1F0BD300142202DE9F04F31
S21444C900DFF8B480002685B08346A8F1080A34468A
S21444C910284B022E4FF080094FF0000234BF082700
S21444C92003272744BFB29AF8001019EA010F04D12E
S21444C93098F8001019EA010F2DD053F8241001ADD1
S21444C940481E073110F801CF814205F801CBF9D1D2
S21444C9509DF804108DF80C20502914D0432914D087
S21444C960422915D055291CD14FF440050DF1050038
S21444C97000F022F905440F4B00225D450BD1E0B28E
S21444C98005B0BDE8F08F0025F0E74FF48005EDE7ED
S21444C9904FF40005EAE701344FEA5909A4B2A74226
S21444C9A0C1D1013608F101080AF1010A082EB0D1B6
S21444C9B0FF20E5E7DC204020380142202DE9FF47F0
S21444C9C000240746204EA146022C4FF0000834BFF0
S21444C9D04FF0080A4FF0030A336801A95A1E07337A
S21444C9E012F8010F9A4201F8010BF9D19DF8043070
S21444C9F08DF80C90502B0DD0432B15D0422B16D0CF
S21444CA00552B17D001340436082CDDD1FF2004B052
S21444CA10BDE8F08700250DF1050000F0CDF805448B
S21444CA20BD420AD1E0B2F2E74FF48005F3E74FF493
S21444CA300005F0E74FF44005EDE708F101081FFA5A
S21444CA4088F39A45C8D8DDE7DC2040202DE9F04F2E
S21444CA50DFF8C490002585B08346A9F108082C4623
S21444CA602B4A022D4FF0800A4FF0000134BF0827AE
S21444CA7003272744BFB298F800001AEA000F04D1EF
S21444CA8099F800001AEA000F32D052F824000DF14B
S21444CA90040C461E073016F801EFB0420CF801EBC2
S21444CAA0F9D19DF804008DF80C10502818D043286E
S21444CAB018D0422819D0552820D14FF440060DF1FD
S21444CAC0050000F079F80644124B00215E45104AF2
S21444CAD00ED15955E0B21D44297205B0BDE8F08F19
S21444CAE00026ECE74FF48006E9E74FF40006E6E755
S21444CAF001344FEA5A0AA4B2A742BCD1013509F11F
S21444CB00010908F10108082DABD1FF20E5E700BF75
S21444CB10DC2040203001422038014220704709285A
S21444CB2094BF30303730C0B2704707B501220DF19C
S21444CB3007018DF80700002013F08AFB03B05DF868
S21444CB4004FB10B5441E14F8010F00B910BDFFF7DE
S21444CB50ECFFF8E70FB400B5C3B044AA02A852F8F5
S21444CB60041B019204F068FC002302A88DF80531EA
S21444CB708DF80631FFF7E5FF43B05DF804EB04B0EB
S21444CB8070470D2008B5FFF7D0FF0A20BDE80840DF
S21444CB90FFF7CBBF10B504460009FFF7C0FFFFF709
S21444CBA0C4FF04F00F00FFF7BAFFFFF7BEFF2C20C8
S21444CBB0BDE81040FFF7B9BF002330B51A46441EFF
S21444CBC0184614F8011F392908D82F290AD95D1C9C
S21444CBD001F00F0303EB00102B4606E0A1F14105DC
S21444CBE0052D06D900B943B108220132072AE8D9EF
S21444CBF030BD5D1CA1F13703ECE71D46EAE7002093
S21444CC0070470000034A92F89E30013382F89E3003
S21444CC10704700BF6C01422010B52A4C94F89A30F5
S21444CC20642B94BF0133002384F89A3094F8C630BA
S21444CC3043B1013BDBB284F8C6301BB984F8C53037
S21444CC4084F88A3194F8C73053B1013BDBB284F898
S21444CC50C7302BB994F88A21032A08BF84F88A314E
S21444CC60B4F8E4315BB1013B9BB2A4F8E43133B988
S21444CC70012284F8CF3184F8C13184F8A52194F890
S21444CC80C231013384F8C231FFF7F2FC94F8A13183
S21444CC9023B1002084F8A10101F01FFCB4F8BE3093
S21444CCA073B1013B9BB2A4F8BE304BB984F88A31C9
S21444CCB084F8C53084F8A33184F8C13184F8DC3173
S21444CCC010BD00BF6C014220034A92F898300133ED
S21444CCD082F89830704700BF6C01422070470323A7
S21444CCE0002010B5064CA4F8EC3104F15402082395
S21444CCF0E16CF5F715FE002384F8953010BD00BFAF
S21444CD006C014220024B0022C3E91522704700BF43
S21444CD106C01422030B5224B002201244FF4FB60C4
S21444CD204FF4FA61082583F8A541A3F89820A3F8A0
S21444CD30B420C3F8D420A3F8CA20A3F8CC2083F8A0
S21444CD408121A3F8822183F88C2183F89C21C3F89F
S21444CD50A02183F8D62183F8DB2183F8DC21A3F8CD
S21444CD60E42183F8EA21A3F8C220C3F8C420D86497
S21444CD70196083F89450A3F8C621C3F8D02183F8E9
S21444CD80D421C3E972424FF40C14C3E92E22C3E9FA
S21444CD906122C3F8C04183F8C421C3E92B1030BDD7
S21444CDA06C014220144B002293F88D1183F88A219B
S21444CDB0E1B90322A3F8861183F8542093F8882116
S21444CDC042F0400283F8552093F89C21012A01BF83
S21444CDD07F2283F85520002283F89C21B3F88621CD
S21444CDE052BAA3F8562000229A65704746F6036264
S21444CDF0A3F85420E8E700BF6C014220054B3022DC
S21444CE00A3F854200A2283F856200D2283F8C7201C
S21444CE10704700BF6C014220034B012283F8C520B3
S21444CE200B2283F8C62070476C01422008B5FFF7F2
S21444CE3083FC0330284B81B2284AC0B207291DD848
S21444CE405921C3F8982183F8540083F8551093F871
S21444CE509E1183F85610FF2183F85710117883F8F3
S21444CE605810517883F859109178D27883F85A102C
S21444CE7083F85B200422A3F8CA2008BDA3F8CC108C
S21444CE80090AC3F8982141F0100183F8550083F845
S21444CE905410592183F8561093F89E1183F857106E
S21444CEA0FF2183F85810117883F8591051789278F6
S21444CEB083F85A1083F85B200322A3F8CA20012281
S21444CEC083F8C520022283F88A21212283F88C2104
S21444CED0222283F88821D0E76C0142201222402087
S21444CEE0024B002283F85420704700BF6C01422056
S21444CEF038B5CB1C40F6FF749BB2A34228BF2346EA
S21444CF00174C1D0A84F855306223A4F8CC1045F01B
S21444CF10100584F8580084F85630030A84F85450B0
S21444CF20022163F00F03C4F8982184F85730012394
S21444CF30A4F8CA301378A4F8CA1084F85930537841
S21444CF4084F85A300323A4F8CA30937884F85B30C4
S21444CF50FFF762FF212384F88A1184F88C3138BDA8
S21444CF606C014220F0B5C84C87B094F8C231013306
S21444CF70DAB21B064ABF002384F8C22184F8C231C1
S21444CF80B4F8C63113B1013BA4F8C63194F8A031C5
S21444CF9023B1002384F8A031FFF798FA94F88A5115
S21444CFA0012D40F0288194F888312E2B3DD146F649
S21444CFB00362A4F854206289A4F8562094F88D217C
S21444CFC00D2A0BD1002384F88A31012384F8953046
S21444CFD040F2F513A4F8BE3007B0F0BD0E2AF4D1E3
S21444CFE094F88911A9480491A9490391B4F8CA1040
S21444CFF0CDE9012194F8C52029460092B4F884214D
S21444D000FFF7A8FD94F88931012B03D1002001F0E5
S21444D01064FAD7E7022B03D1002001F079FAD1E76E
S21444D020FF2BCFD184F8CB51CCE7222BCAD1B4F80E
S21444D0308431B3F5A06F6BD1964D0022964915F80E
S21444D040010B134601321F2892B204D9322A01F842
S21444D050010BF4D11346E2182C213A2082F8E4104E
S21444D0605A1C422114FA82F282F8E4109A1C4F2188
S21444D07014FA82F282F8E410DA1C14FA82F282F885
S21444D080E4101A1D542114FA82F282F8E4105A1D50
S21444D090562114FA82F282F8E410991DDA1D14FA25
S21444D0A081F192B281F8E4007C49087842281FD086
S21444D0B022444E2182F8E41003F10802302114FA87
S21444D0C082F282F8E41003F10A010933202289B27D
S21444D0D014FA83F383F8E4206318002201314FF4F2
S21444D0E0A06083F8E42089B26B4AFFF701FF6CE73F
S21444D0F00B466B4D1878114601321F2892B2EBD975
S21444D10001332144AB4281F8E400F3D11146E3E70E
S21444D110644EB4F8862106EB4316B4F886C14FEA4B
S21444D120122E3789D0B29CFA9CFCF268FB1C99B24A
S21444D130DBB207292FD984F85530C1F30321622383
S21444D14084F857E041F0100184F8580084F85630CB
S21444D150002384F854100221A4F8CA30C4F8982155
S21444D160A4F8CC701378A4F8CA5084F8593053788D
S21444D170A4F8CA1084F85A30937884F85B300323B2
S21444D180A4F8CA30FFF748FE322384F88A1184F89C
S21444D190C630212374E0622184F85430A4F856C083
S21444D1A0013384F855100021C4F89821DBB2A4F862
S21444D1B0CA10A4F8CC701078A4F8CA5084F8580062
S21444D1C0507884F859000220A4F8CA00907884F86D
S21444D1D05A000320A4F8CA00D27884F85B200422BC
S21444D1E0A4F8CA20DAB2082A3FF4ECAEE2180133B7
S21444D1F082F85410F6E7022D7FF4EEAE94F8C5306C
S21444D200002B7FF4E9AE94F88831222B7FF4DDAE10
S21444D21094F8C430012B06D9023BDBB284F8C43000
S21444D220002B7FF4D9AE94F8C330072194F88C21B0
S21444D2302E27B4F8CC50D4F89861134884F8C430F8
S21444D24084F85420B4F8CA3001390130AB4238BFB0
S21444D25016F803C003F101032CBF80F8547080F81D
S21444D26054C09BB211F0FF01A4F8CA30EAD19D42E3
S21444D27002F10103DBB298BF84F88A112F2B88D8B9
S21444D28084F88C31A1E600BF6C0142208E7E4600B5
S21444D2900403422000014400500242202010400073
S21444D2A039104000E8754600FFF75CBE38B51B4CA5
S21444D2B06389A4F89E31FFF713FE94F89E5105F057
S21444D2C0F703022B05D10123002584F89D31284617
S21444D2D038BD012D0FD145F6061384F85650A4F8F0
S21444D2E0543094F89F3184F85730FFF7E9FA40BA3F
S21444D2F0A4F85800EBE7032D12BF47F6027345F631
S21444D300021384F856504FF001051BBFA4F854305E
S21444D3101223A4F8543084F85630D8E76C014220DF
S21444D32008B5FFF7DDFD0B4B4CF20252A3F8542030
S21444D3309A7A012A83F8562004D1002283F8D4210D
S21444D340012008BD022A01D10122F7E77F2283F893
S21444D3505520F5E76C014220064B47F60372A3F8C6
S21444D3605420012283F8560083F8571083F89C21F2
S21444D370704700BF6C014220074B93F8D621132A0E
S21444D38009D093F8A521032A1FBF7F2283F8D6210C
S21444D390012283F89C2170476C014220002310B57B
S21444D3A06B4C84F8D63194F8CE30222B07D194F8BF
S21444D3B0D531032B09D0132384F8D63105E0202B2E
S21444D3C014D194F8D531022BF5D894F8D63163B1FC
S21444D3D047F6037284F857300123A4F8542094F88F
S21444D3E0CE2084F89C3184F8562010BD102B0BD1E7
S21444D3F094F8D531022BDED1A37A03F07F03013BA8
S21444D400022BE2D91223D7E7852B12D1A37A013B0C
S21444D410012B84BF122384F8D63194F8D531022BDD
S21444D42002D0132384F8D63194F8D601FFF7A4FF2C
S21444D430CBE7272B05D194F8D53103F0FB03022B19
S21444D440B8E7192B18D194F8D531012BB3D0A27A6A
S21444D4500A2AF4D0032AF2D0022AAAD0042A08D1EF
S21444D460062BA8D1A37B012BAFD0FF2BADD0312305
S21444D470A2E7012AC6D19CE7282B1DD194F8D511E2
S21444D480A27A032902F07F0305D0002BC9D0032BD0
S21444D490C7D0022902D0591E0129C2D912F07C0FE6
S21444D4A001D01223BEE7E27A013A022ABCD90BB174
S21444D4B0032BB9D13123B5E7142B1CD194F8D531BD
S21444D4C0042B7FF478AFE07AA37A00EB0323207B27
S21444D4D000EB03206FF07F439842C4F8D0013FF43A
S21444D4E074AF1C4B98423FF470AFFFF767FAFF28BF
S21444D4F07FF46BAFBBE73E2B11D194F8D531022BAA
S21444D5007FF459AFA37A13F07F0F4FF4FA7318BF22
S21444D5101222A4F8E43118BF84F8D62155E7312BFB
S21444D52009D194F8D531062B3FF645AFA37A013B93
S21444D530022B9CD849E72E2B05D194F8D531022BE3
S21444D5407FF639AF41E70F2B3FF63FAF112333E762
S21444D5506C014220FF0040004FF287139842134B61
S21444D5600ED10A290AD1002283F8D62193F8D6216F
S21444D570003A18BF012283F8DB2170471322F3E7F1
S21444D5804FF28B12904201D10429EBE74FF29512E9
S21444D590904201D10329E5E74FF293129042F9D025
S21444D5A04FF28C129042DED10729DBE76C01422011
S21444D5B00B4B024693F90A00997A0028B3BF01F050
S21444D5C07F02012083F855200020B8BF9A724FF09E
S21444D5D00102A8BF83F8540083F8A521704700BF12
S21444D5E06C014220274B014610B593F90A009A7AFB
S21444D5F00028BBBF02F07F02002001209A729A7A6C
S21444D600541E022C31D8062483F85510022A4FF0B3
S21444D610000183F854404FF4997483F85620A3F8D5
S21444D62058404FF0F40483F8571083F85A404FF4A8
S21444D630FA7483F8A521A3F8E44112D1124A127869
S21444D640422A06D102F5800202F6DF7212784F2A89
S21444D65003D0012283F89C2103E00122084683F884
S21444D660CA21002283F8CF2110BD47F60372A3F8DF
S21444D670542093F8CE2083F85620122283F857205D
S21444D680E7E700BF6C0142202010400010B5214C53
S21444D690A37AE07A00EB032080B2B0F5754FA4F885
S21444D6A086010BD14FF4A063A4F8843101230020F3
S21444D6B084F88A31222384F8883111E0B0F5704F1B
S21444D6C012D300F0A9FD4FF6FF73984209D1022306
S21444D6D0012084F85430637A43F0400384F855308C
S21444D6E010BDA4F88401E1E740F2DF73D4F8E0010A
S21444D6F0C01A47F60373A4F8543018BF012094F8B0
S21444D700CE3084F85630312384F85730012384F8D9
S21444D7109C31E5E76C0142202DE9F0414E4C2E2326
S21444D720A27AE07A84F88831130900EB0220217B40
S21444D7300E2B84F88D3180B284F88911A4F88601C2
S21444D7400DD10123002084F88A3194F8DB31012B73
S21444D75071D1424A626584F89C31BDE8F081B0F5E7
S21444D760704F13D300F0C3FD0F230246A4F8840180
S21444D77084F88D314FF6FF73984204D0384E06EB4A
S21444D7804013D96921B9032384F8DB310120DCE74F
S21444D79094F8CF11012901D00223F5E7002084F83C
S21444D7A09C0194F8DB010028F0D19B6894F8D501DD
S21444D7B00333DBB2984207D013232A4884F8DB119C
S21444D7C084F8D631FFF7C6F9B4F884310027DFF879
S21444D7D09C80042506EB4313A4F8CA70DA689B6859
S21444D7E0C4F89421A4F8CC30B4F8CA3018F8011B15
S21444D7F0D4F89421D154B4F8CA30B4F8CC200133C8
S21444D8009BB29A42A4F8CA30C0D90020FFF7CAFA9D
S21444D81094F89C3184F8DB7143B9B4F8843106EB50
S21444D8204313DB69012B08BF84F8A131013D15F091
S21444D830FF05D9D1AAE7022B03D10B4B636501231D
S21444D84089E7032B01BF03F1445303F5391303F56A
S21444D8507C53636581E700BF6C014220037F2E132F
S21444D860E8754600DF7E4600037F2E33780142206B
S21444D870204B014630B593F90A009A7A0028BBBF7C
S21444D88002F07F02002001209A72DA7A02F0FD0448
S21444D890012C22D19A7A02F0FD05012D11D183F88C
S21444D8A0DC5193F8A521012A4FF0020283F8542054
S21444D8B01AD87F225A7222229A72002283F8DC21D6
S21444D8C030BD12B983F8DC21EBE7022A06BF0020FC
S21444D8D083F8DC4183F89C41E3E7022A1FBF7F229A
S21444D8E05A7212229A72DCE79A7A83F8551083F8B1
S21444D8F05620E5E76C0142207047704770477047F2
S21444D90050B123230549013B00284FEA40009BB20F
S21444D910B8BF4840002BF6D1704700BF69696C6CAD
S21444D920F8B56C4B064693F8A5211C46012A0BD83D
S21444D93047F60372A3F854205A7A83F856207F2277
S21444D94083F8572001253DE0997A01F0FB05012D27
S21444D9504AD1062384F8550084F8561084F8543087
S21444D96094F8CF31012B2FD101292DD10023A4F8CF
S21444D970A631A4F8A83194F8A661012994F8A72101
S21444D98094F8A83118BF022184F8582002EB0622E6
S21444D99094F8A90184F8593003EB022384F85A001A
S21444D9A000EB032084F85760FFF7AAFF030E84F8C1
S21444D9B0A631030C40BA84F8A7310123A4F8A80181
S21444D9C084F8C1312846F8BD94F8C23103F11102F7
S21444D9D084F8A63184F8A72103F12202343384F86C
S21444D9E0A82184F8A931C6E7022DABD193F8C1210A
S21444D9F0012A4FF0000210D083F8C12147F6037283
S21444DA000125A3F8542093F8CE2083F89C5183F83C
S21444DA105620242283F85720D4E783F8C121DA7AA3
S21444DA2093F8A6319A420AD1227B94F8A7319A42B7
S21444DA3005D1B4F8A821B4F80D309A421DD047F663
S21444DA4003730629A4F8543094F8CE3084F856303C
S21444DA504FF0350384F857304FF0010384F89C3177
S21444DA607FF470AF1C4B1B78422B08D001231B4815
S21444DA7084F89C31FFF76EF801E00629F2D094F85A
S21444DA809C51002D7FF45EAFA37A022784F855603C
S21444DA9084F8563084F85470FFF721F9A37A062B9D
S21444DAA00ED101230E4884F8CF7184F8CA31FFF7AB
S21444DAB048F80B48FFF745F80948FFF742F881E76E
S21444DAC094F8A531023B012B9CBF012384F8CF3147
S21444DAD078E700BF6C01422020104000F37E4600E9
S21444DAE0517F4600114B002293F89C1183F8D621AF
S21444DAF0012904BF7F2183F89C2193F8CE2008BFD8
S21444DB0083F85510312A0DD193F8D511062903D937
S21444DB10132283F8D62103E0997A01390229F8D8EA
S21444DB2001207047342AFBD11222F2E76C014220CE
S21444DB3070B5674C0025637A264694F8DD2184F850
S21444DB40CE30237A84F89C519A4284F8D53101D851
S21444DB5000200FE0013B062BFAD8FFF71FFC94F891
S21444DB609C31012B0FD1D4F8E02140F2DF739A4266
S21444DB7001D0012070BD94F8D631113B012BF8D862
S21444DB8084F89C51E4E7627A94F8CE30102A43F045
S21444DB90400003D1BDE87040FFF724BD202A03D1DE
S21444DBA0BDE87040FFF704BD852A03D1BDE8704048
S21444DBB0FFF7B6BB2A2B0AD1E37A84F8C33146F67C
S21444DBC00223A4F85430A37A84F85630D1E7222BA3
S21444DBD004D16220BDE87040FFF758BD2E2B04D117
S21444DBE06E20BDE87040FFF797BD282B04D168200F
S21444DBF0BDE87040FFF73CBE2F2B0ED146F60673A9
S21444DC00344AA4F854300623013B12F8011B13F09F
S21444DC10FF0382F84B10F7D1ABE7142B15D1FFF76F
S21444DC205FF9D4F8D0016FF07F43984202D02A4B74
S21444DC30984207D1012386F8A03145F20143A6F85D
S21444DC40543096E7FEF702FFF7E7272B04D1672008
S21444DC50BDE87040FFF764BE192B03D1BDE87040A1
S21444DC60FFF724BB312B0BD11C4A0723013B12F888
S21444DC70011B13F0FF0382F8DA10F7D1712079E71D
S21444DC80112B0FD145F20213A4F85430A37A84F82A
S21444DC905630FFF724F81248FEF753FF1148FEF7B4
S21444DCA050FF66E73E2B0FD194F90A10A37A002959
S21444DCB0FFF64EAF022142F0400284F8563084F814
S21444DCC0541084F8552054E7FEF79CFF40E700BF05
S21444DCD06C01422076014220FF004000750142203C
S21444DCE0FD7E4600127F460038B5424C0F2384F82A
S21444DCF08D312546237A217B03F00F02637AE07A3E
S21444DD0003EB022304F1E40201EB0020C4F894215F
S21444DD1042F2030280B2A4F8CC30A4F88A2194F8E4
S21444DD20CE202F2A23D1033B2E22A4F87A019BB27D
S21444DD3084F8882104F22F12A4F88601A4F8CC3083
S21444DD4084F87931A37BC4F8942184F831310423D0
S21444DD50627BA4F8CA30E37B84F87C2184F82F11D4
S21444DD6084F8302184F83231FFF748F814E0A4F8F8
S21444DD70860100F051FA4FF6FF7398420ED147F6EB
S21444DD8003723123A5F8542095F8CE2085F8D63171
S21444DD9085F8562085F85730012038BD164B03EBDE
S21444DDA04013DA69002AEAD02E22A4F8840184F8C3
S21444DDB08821032284F88A21DA689B68C4F894216F
S21444DDC0A4F8CC300123A4F8CA30637B1370B4F8AB
S21444DDD0CA30D4F89421591CA4F8CA10A17BD15453
S21444DDE0B4F8CA30D4F89421591CA4F8CA10E17B7C
S21444DDF0D154B9E76C014220E875460008B51A4B81
S21444DE000022197A83F88D2101F00F00597AA3F87D
S21444DE10842101EB00219A7AC82983F888211A7B49
S21444DE2088BFC82183F8E520A3F8CC10D97A02EB42
S21444DE3001205A7B83F8E41083F8E6209A7BA3F803
S21444DE40860142F2030083F8E720DA7BA3F88A01CE
S21444DE5083F8E82005220548A3F8CA20C3F89401AD
S21444DE60FEF7CCFF012008BD6C0142201222402060
S21444DE70184B0022987A83F8D62183F89C21A0F187
S21444DE802E0283F8CE00D1B208291DD840F249129A
S21444DE90CA40D24312F0010216D12E2883F8DB2161
S21444DEA014D193F8A521012A02D993F8CF216AB94F
S21444DEB07E2283F8D62102F17E2202F5381285327C
S21444DEC05A65012283F89C21012070470020FFF701
S21444DED00BBF00BF6C014220002340F2F51210B580
S21444DEE0884C84F8983084F89C31A4F8BE204FF4CB
S21444DEF0FA72C4E915332368A4F8E421B3F5FA6F3B
S21444DF0017D1431E04F10802073013F8011F984244
S21444DF1002F8011BF9D14FF4FA63C4F8E031227ACF
S21444DF2012F0F0032BD1FFF703FE002840F08B805D
S21444DF304CE040F2DF72934220D1037813F0F00FA6
S21444DF401CD14278A2F11003DBB2182B11D9852AD2
S21444DF5001D03E2A12D140F2DF736B4AC4F8E03156
S21444DF60431E073013F8011F834202F8011BF9D100
S21444DF70D5E7664A22FA03F3DB07ECD410BD102B30
S21444DF8002D1FFF775FFD0E7202B40F08F8094F83E
S21444DF90CE302E3BD9B206295CD84923CB40DB434E
S21444DFA013F0010356D194F88A1103290ED194F83C
S21444DFB0DD11072910D8B4F8CA3001391944B4F829
S21444DFC0CC30994202D2002384F88A31002384F864
S21444DFD09C3184F89830D1E794F88B11914205D15E
S21444DFE04B4884F88A31FEF7ACFDEFE784F88B2182
S21444DFF00D2284F8C72094F8DB2132B9E218D4F80D
S21444E0009411507AB4F8CA208854B4F8CA20B4F8A4
S21444E010CC10013292B29142A4F8CA2042D894F865
S21444E020DB31012B1AD147F60372A4F8542094F836
S21444E030CE2084F85620132284F8572084F89C3146
S21444E040002384F8DB3194F89C31012B04BF7F23F2
S21444E05084F85530012384F89530B7E7022B0CD169
S21444E06047F60373A4F8543094F8CE3084F8563008
S21444E070332384F857300123E0E70020FEF792FE6E
S21444E080B4F88421234B94F89C1103EB42132248A2
S21444E090DA69012A08BF84F8A12194F8A131FEF771
S21444E0A059FDCDE70133072BA5D18FE7302B8DD112
S21444E0B094F8DD31022B86D9312A03D10B2384F818
S21444E0C0C63083E794F8C5305BB9322A09D146F2A4
S21444E0D00323A4F85430B4F886315BBAA4F8563017
S21444E0E04CE7A37A0021312A03F1030384F8C510D0
S21444E0F084F8C610DBB284F8C33084F8C4303FF6E4
S21444E10062AF63E76C0142207401422013020401AB
S21444E110227F4600E87546003A7F46000A4810B516
S21444E120FEF718FD72B64FF0005308491022084C0B
S21444E1300848C3E90012FEF70DFDFBF7A4FB204692
S21444E140FEF708FDFBE700BF4C7F46007154CA3D0E
S21444E150737F4600597F460038B52C4B93F8C82148
S21444E1601C4632B9FEF7D6FD2948BDE83840FEF7CE
S21444E170E8BC93F89820002A3FD0002293F89D11DB
S21444E18083F8982081B193F89E0183F89D21FEF789
S21444E1904DFE012384F8953040F2F513A4F8BE30C2
S21444E1A0BDE83840FEF79BBD93F89550002DF3D15B
S21444E1B0184A13780133DBB2022B01D8137038BDEA
S21444E1C01570FEF7CFFE94F8993094F8C2210133C7
S21444E1D00132DBB284F8C221042B84F899300CD97E
S21444E1E084F89950FEF718FDB4F89C30C72B96BFB8
S21444E1F00133A4F89C50A4F89C3094F8CA2194F8AF
S21444E200CB311343DBD0FFF789FF00BF6C014220BC
S21444E210827F4600D82140204FF22803984218D8DF
S21444E2204FF20F03984259D9A0F570401138172879
S21444E2300DD8DFE800F056292B2D2F3131333537F2
S21444E240393B3D3F4143454547494B4D4F5104209B
S21444E25070474FF29313984245D00CD84FF2871329
S21444E260984242D04FF288124FF6FF73904214BF42
S21444E2701846012070474FF295124FF6FF739042AE
S21444E28014BF184602207047062070470720704780
S21444E29008207047092070470A2070470B207047B3
S21444E2A00C2070470D2070470E2070470F20704793
S21444E2B01020704711207047122070471320704773
S21444E2C01420704715207047162070471720704753
S21444E2D018207047192070471A2070474FF6FF7071
S21444E2E07047052070470320704700207047FFF7AB
S21444E2F093BF1C280146F0B585B037D83F4B420142
S21444E30003EB40169C584FF6FF739C422ED0F3699D
S21444E310012B2BD1756804F50004B368AD0822467A
S21444E320009337482B46FEF715FCD6E903639A1E3E
S21444E330012A1DD8002315E036F82310023389B28B
S21444E340029102990904029150880299014402916B
S21444E350918889B20391039909040391D188039A59
S21444E3600A4403929D4206EB8302E5D805B0F0BD0D
S21444E370043B012B3FD90027BD4206EB8701F5D964
S21444E38016F82730204602370834DBB20293029B45
S21444E3901B0602934A78029B03EB024302938A7855
S21444E3A0029B03EB02230293CB78029A1344029314
S21444E3B00B79DBB20393039B1B0603934A79039BB7
S21444E3C003EB024303938A79039B03EB02230393F1
S21444E3D0CB7902A9039A13440393FEF710FCCBE7C8
S21444E3E056F8231002330291526803929D4206EB7C
S21444E3F08302F5D8BAE70023F8E700BFE87546007D
S21444E4008D7F46001C28014630B403D92C4830BCC6
S21444E410FEF7A0BB42012B4B03EB40109B584FF634
S21444E420FF7293421FD0C269012A1CD10169072991
S21444E43019D0826803F50003C468881E012814D8DE
S21444E44052080234002191420DD253F8040B050CB5
S21444E45024F8025C4D1C954205D2023180B28A42B1
S21444E46024F8040BEFD830BC70470439012925D86A
S21444E47022F0030222449442F5D053F8041B44F895
S21444E480041BF8E75858050E25704D1CAA42EAD9D5
S21444E490C0F3074565708D1CAA42E4D9C0F307252E
S21444E4A0A570CD1CAA42DED90431C0B204348A42D7
S21444E4B004F8010CD7D99142E4D3D4E70021FAE713
S21444E4C0AE7F4600E875460010B50024A0B201347D
S21444E4D0FFF798FF1D2CF9D110BD1FB50024A0B23C
S21444E4E00134FFF706FF1D2CF9D1074B02A902930E
S21444E4F04FF47C730393054B01930198FEF77FFB1F
S21444E500002004B010BD00BF55EFCDAB1000800016
S21444E51008B508B9FFF7D8FF002008BD124B00B570
S21444E5201B688BB00293114B1A6803925A68049284
S21444E5309B6805930299039A049B059800900C489F
S21444E540FEF708FB039BB3F57C7F06D10948FEF72C
S21444E55001FB01200BB05DF804FB0748FEF7FAFA0E
S21444E5604FF0FF30F6E700BF100080001400800034
S21444E570BE7F4600D67F4600E17F460008B5FFF7DB
S21444E580CDFF012805D1FFF79FFFBDE80840FDF702
S21444E590B9BFFFF7C3FF0128F5D00020FFF79DFF62
S21444E5A0FFF7BCFFF1E700BF10F8012B11F8013B61
S21444E5B0012A28BF9A42F7D0D01A7047034613F868
S21444E5C0012B002AFBD1181A0138704700000000BE
S21444E5D001F0FF01102A2BDB10F0070F08D010F8CB
S21444E5E0013B013A8B422DD010F0070F42B3F6D1CF
S21444E5F0F0B441EA012141EA014122F007047FF0E8
S21444E60000070023F0E80256083C85EA010586EA3E
S21444E610010685FA47F5A3FA87F586FA47F6A5FA7A
S21444E62087F68EB9EED1F0BC01F0FF0102F0070286
S21444E63032B110F8013B013A83EA010313B1F8D131
S21444E6400020704701387047002D06BF3546033812
S21444E650073815F0010F07D1013015F4807F02BF4B
S21444E660013015F4C03F0130F0BC0138704700BF9C
S21444E67081F0004102E000BF83F0004330B54FEA2A
S21444E68041044FEA430594EA050F08BF90EA020F97
S21444E6901FBF54EA000C55EA020C7FEA645C7FEA2A
S21444E6A0655C00F0E2804FEA5454D4EB5555B8BF4D
S21444E6B06D420CDD2C4480EA020281EA030382EABE
S21444E6C0000083EA010180EA020281EA0303362D50
S21444E6D088BF30BD11F0004F4FEA01314FF4801C23
S21444E6E04CEA113102D0404261EB410113F0004F35
S21444E6F04FEA03334CEA133302D0524263EB4303EC
S21444E70094EA050F00F0A780A4F10104D5F1200E89
S21444E7100DDB02FA0EFC22FA05F2801841F10001E4
S21444E72003FA0EF2801843FA05F359410EE0A5F1B8
S21444E73020050EF1200E012A03FA0EFC28BF4CF0E9
S21444E740020C43FA05F3C01851EBE37101F000459F
S21444E75007D54FF0000EDCF1000C7EEB00006EEBAC
S21444E7600101B1F5801F1BD3B1F5001F0CD3490836
S21444E7705FEA30004FEA3C0C04F101044FEA44528D
S21444E78012F5800F80F09A80BCF1004F08BF5FEA14
S21444E790500C50F1000041EB045141EA050130BDF4
S21444E7A05FEA4C0C404141EB0101013C28BFB1F506
S21444E7B0801FE9D291F0000F04BF01460020B1FA51
S21444E7C081F308BF2033A3F10B03B3F120020CDA24
S21444E7D00C3208DD02F1140CC2F10C0201FA0CF002
S21444E7E021FA02F10CE002F11402D8BFC2F1200C67
S21444E7F001FA02F120FA0CFCDCBF41EA0C0190401D
S21444E800E41AA2BF01EB0451294330BD6FEA040465
S21444E8101F3C1CDA0C340EDC04F11404C4F1200250
S21444E82020FA04F001FA02F340EA030021FA04F362
S21444E83045EA030130BDC4F10C04C4F1200220FAB9
S21444E84002F001FA04F340EA0300294630BD21FAF7
S21444E85004F0294630BD94F0000F83F4801306BFBD
S21444E86081F480110134013D4EE77FEA645C18BFB1
S21444E8707FEA655C29D094EA050F08BF90EA020F48
S21444E88005D054EA000C04BF1946104630BD91EA40
S21444E890030F1EBF0021002030BD5FEA545C05D143
S21444E8A04000494128BF41F0004130BD14F5800482
S21444E8B03CBF01F5801130BD01F0004545F0FE41F6
S21444E8C041F470014FF0000030BD7FEA645C1ABF2B
S21444E8D0194610467FEA655C1CBF0B46024650EA62
S21444E8E0013406BF52EA033591EA030F41F400218E
S21444E8F030BD00BF90F0000F04BF0021704730B514
S21444E9004FF4806404F132044FF000054FF00001E8
S21444E91050E700BF90F0000F04BF0021704730B5A9
S21444E9204FF4806404F1320410F0004548BF40427E
S21444E9304FF000013EE700BF42004FEAE2014FEAD3
S21444E94031014FEA02701FBF12F07F4393F07F4FAE
S21444E95081F06051704732F07F4208BF704793F0B1
S21444E9607F4F04BF41F40021704730B54FF46074C4
S21444E97001F0004521F000411CE700BF50EA0102C7
S21444E98008BF704730B54FF000050AE050EA010270
S21444E99008BF704730B511F0004502D5404261EBE0
S21444E9A041014FF4806404F132045FEA915C3FF421
S21444E9B0D8AE4FF003025FEADC0C18BF03325FEABE
S21444E9C0DC0C18BF033202EBDC02C2F1200300FA6F
S21444E9D003FC20FA02F001FA03FE40EA0E0021FA94
S21444E9E002F11444BDE600BF70B54FF0FF0C4CF482
S21444E9F0E06C1CEA11541DBF1CEA135594EA0C0F34
S21444EA0095EA0C0F00F0DEF82C4481EA030621EA6E
S21444EA104C5123EA4C5350EA013518BF52EA0335A9
S21444EA2041F4801143F4801338D0A0FB02CE4FF05B
S21444EA300005E1FB02E506F00042E0FB03E54FF08B
S21444EA400006E1FB03569CF0000F18BF4EF0010E83
S21444EA50A4F1FF04B6F5007F64F5407404D25FEA7F
S21444EA604E0E6D4146EB060642EAC62141EA555132
S21444EA704FEAC52040EA5E504FEACE2EB4F1FD0C74
S21444EA8088BFBCF5E06F1ED8BEF1004F08BF5FEAF2
S21444EA90500E50F1000041EB045170BD06F00046A4
S21444EAA046EA010140EA020081EA0301B4EB5C0451
S21444EAB0C2BFD4EB0C0541EA045170BD41F4801149
S21444EAC04FF0000E013C00F3AB8014F1360FDEBF6E
S21444EAD0002001F0004170BDC4F10004203C35DA4A
S21444EAE00C341BDC04F11404C4F1200500FA05F3CD
S21444EAF020FA04F001FA05F240EA020001F000426E
S21444EB0021F0004110EBD37021FA04F642EB0601E3
S21444EB105EEA430E08BF20EAD37070BDC4F10C040D
S21444EB20C4F1200500FA04F320FA05F001FA04F2D1
S21444EB3040EA020001F0004110EBD37041F10001BD
S21444EB405EEA430E08BF20EAD37070BDC4F12005C8
S21444EB5000FA05F24EEA020E20FA04F301FA05F230
S21444EB6043EA020321FA04F001F0004121FA04F2D8
S21444EB7020EA020000EBD3705EEA430E08BF20EAA8
S21444EB80D37070BD94F0000F0FD101F000464000E2
S21444EB9041EB010111F4801F08BF013CF7D041EA64
S21444EBA0060195F0000F18BF704703F00046520068
S21444EBB043EB030313F4801F08BF013DF7D043EA39
S21444EBC00603704794EA0C0F0CEA135518BF95EAEF
S21444EBD00C0F0CD050EA410618BF52EA4306D1D176
S21444EBE081EA030101F000414FF0000070BD50EA95
S21444EBF0410606BF1046194652EA430619D094EA1F
S21444EC000C0F02D150EA013613D195EA0C0F05D108
S21444EC1052EA03361CBF104619460AD181EA03015C
S21444EC2001F0004141F0FE4141F470014FF0000014
S21444EC3070BD41F0FE4141F4780170BD70B54FF0AF
S21444EC40FF0C4CF4E06C1CEA11541DBF1CEA13552F
S21444EC5094EA0C0F95EA0C0F00F0A7F8A4EB050411
S21444EC6081EA030E52EA03354FEA013100F0888008
S21444EC704FEA03334FF0805545EA131343EA1263D1
S21444EC804FEA022245EA111545EA10654FEA002686
S21444EC900EF000419D4208BF964244F1FD0404F53F
S21444ECA0407402D25B084FEA3202B61A65EB03059B
S21444ECB05B084FEA32024FF480104FF4002CB6EB58
S21444ECC0020E75EB030E22BFB61A754640EA0C00D8
S21444ECD05B084FEA3202B6EB020E75EB030E22BF18
S21444ECE0B61A754640EA5C005B084FEA3202B6EB59
S21444ECF0020E75EB030E22BFB61A754640EA9C0018
S21444ED005B084FEA3202B6EB020E75EB030E22BFE7
S21444ED10B61A754640EADC0055EA060E18D04FEAA5
S21444ED20051545EA16754FEA06164FEAC30343EA45
S21444ED3052734FEAC2025FEA1C1CC0D111F4801F12
S21444ED400BD141EA00014FF000004FF0004CB6E70B
S21444ED5011F4801F04BF01430020B4F1FD0C88BFAA
S21444ED60BCF5E06F3FF6AFAEB5EB030C04BFB6EBB5
S21444ED70020C5FEA500C50F1000041EB045170BDA8
S21444ED800EF0004E4EEA113114EB5C04C2BFD4EBD5
S21444ED900C0541EA045170BD41F480114FF0000E59
S21444EDA0013C90E645EA060E8DE60CEA135594EAD5
S21444EDB00C0F08BF95EA0C0F3FF43BAF94EA0C0FD8
S21444EDC00AD150EA01347FF434AF95EA0C0F7FF44D
S21444EDD025AF104619462CE795EA0C0F06D152EAA1
S21444EDE003353FF4FDAE1046194622E750EA410685
S21444EDF018BF52EA43067FF4C5AE50EA41047FF496
S21444EE000DAF52EA43057FF4EBAE12E74FF0FF3CFA
S21444EE1006E000BF4FF0010C02E000BF4FF0010CCB
S21444EE204DF804CD4FEA410C7FEA6C5C4FEA430C44
S21444EE3018BF7FEA6C5C1BD001B050EA410C0CBF93
S21444EE4052EA430C91EA030F02BF90EA020F0020F5
S21444EE50704710F1000F91EA030F58BF994208BF5C
S21444EE6090422CBFD8176FEAE37040F00100704719
S21444EE704FEA410C7FEA6C5C02D150EA013C07D170
S21444EE804FEA430C7FEA6C5CD6D152EA033CD3D0BB
S21444EE905DF8040B704700BF8446104662468C46B5
S21444EEA01946634600E000BF01B5FFF7B7FF0028E8
S21444EEB048BF10F1000F01BD4DF808EDFFF7F4FF11
S21444EEC00CBF012000205DF808FB00BF4DF808ED9C
S21444EED0FFF7EAFF34BF012000205DF808FB00BFBF
S21444EEE04DF808EDFFF7E0FF94BF012000205DF8E1
S21444EEF008FB00BF4DF808EDFFF7CEFF94BF012096
S21444EF0000205DF808FB00BF4DF808EDFFF7C4FF8E
S21444EF1034BF012000205DF808FB00BF4FEA410CD7
S21444EF207FEA6C5C02D150EA013C0AD14FEA430CBA
S21444EF307FEA6C5C02D152EA033C02D14FF00000F7
S21444EF4070474FF0010070474FEA410212F5001235
S21444EF5015D211D56FF47873B3EB625212D94FEAD7
S21444EF60C12343F0004343EA505311F0004F23FAC1
S21444EF7002F018BF404270474FF00000704750EA16
S21444EF80013005D111F0004008BF6FF000407047D3
S21444EF904FF00000704700BF4A0011D212F500122D
S21444EFA011D20DD56FF47873B3EB62520ED44FEA98
S21444EFB0C12343F0004343EA505323FA02F0704718
S21444EFC04FF00000704750EA013002D14FF0FF3056
S21444EFD070474FF0000070474FEA4102B2F1E043F9
S21444EFE024BFB3F5001CDCF1FE5C0DD901F0004CE7
S21444EFF04FEAC0024CEA5070B2F1004F40EB830037
S21444F00008BF20F00100704711F0804F21D113F162
S21444F0103872BCBF01F00040704741F480114FEA9B
S21444F0205252C2F11802C2F1200C10FA0CF320FA24
S21444F03002F018BF40F001004FEAC1234FEAD32341
S21444F04003FA0CFC40EA0C0023FA02F34FEA4303AB
S21444F050CCE77FEA625307D150EA01331EBF4FF034
S21444F060FE4040F44000704701F0004040F0FE404F
S21444F07040F40000704700BF80F0004002E000BF4C
S21444F08081F0004142001FBF5FEA410392EA030F4A
S21444F0907FEA226C7FEA236C6AD04FEA1262D2EB94
S21444F0A01363C1BFD218414048404140B8BF5B4299
S21444F0B0192B88BF704710F0004F40F4000020F032
S21444F0C07F4018BF404211F0004F41F4000121F048
S21444F0D07F4118BF494292EA030F3FD0A2F1010292
S21444F0E041FA03FC10EB0C00C3F1200301FA03F1D0
S21444F0F000F0004302D5494260EB4000B0F5000FF3
S21444F10013D3B0F1807F06D340084FEA310102F1B1
S21444F1100102FE2A51D2B1F1004F40EBC25008BF63
S21444F12020F0010040EA03007047490040EB00002D
S21444F130013A28BFB0F5000FEDD2B0FA80FCACF12E
S21444F140080CB2EB0C0200FA0CF0AABF00EBC2505B
S21444F15052421843BCBFD0401843704792F0000F49
S21444F16081F4000106BF80F400000132013BB5E79C
S21444F1704FEA41037FEA226C18BF7FEA236C21D012
S21444F18092EA030F04D092F0000F08BF0846704777
S21444F19090EA010F1CBF0020704712F07F4F04D145
S21444F1A0400028BF40F00040704712F100723CBF58
S21444F1B000F50000704700F0004343F0FE4040F482
S21444F1C0000070477FEA226216BF08467FEA236340
S21444F1D00146420206BF5FEA412390EA010F40F42B
S21444F1E0800070474FF0000304E000BF10F0004377
S21444F1F048BF40425FEA000C08BF704743F096435E
S21444F20001464FF000001CE050EA010208BF704778
S21444F2104FF000030AE000BF50EA010208BF7047FF
S21444F22011F0004302D5404261EB41015FEA010C14
S21444F23002BF84460146002043F0B64308BFA3F10C
S21444F2408053A3F50003BCFA8CF2083AA3EBC253EE
S21444F25010DB01FA02FC634400FA02FCC2F120020D
S21444F260BCF1004F20FA02F243EB020008BF20F044
S21444F2700100704702F1200201FA02FCC2F12002AA
S21444F28050EA4C0021FA02F243EB020008BF20EA9F
S21444F290DC7070474FF0FF0C1CEAD0521EBF1CEACD
S21444F2A0D15392EA0C0F93EA0C0F6FD01A4480EABB
S21444F2B0010C400218BF5FEA41211ED04FF00063A4
S21444F2C043EA501043EA5111A0FB01310CF00040D0
S21444F2D0B1F5000F3EBF490041EAD3715B0040EAF6
S21444F2E0010062F17F02FD2A1DD8B3F1004F40EBC6
S21444F2F0C25008BF20F00100704790F0000F0CF099
S21444F300004C08BF49024CEA502040EA51207F3A5C
S21444F310C2BFD2F1FF0340EAC250704740F4000037
S21444F3204FF00003013A5DDC12F1190FDCBF00F028
S21444F33000407047C2F10002410021FA02F1C2F1D6
S21444F340200200FA02FC5FEA310040F1000053EA72
S21444F3504C0308BF20EADC70704792F0000F00F0C0
S21444F360004C02BF400010F4000F013AF9D040EAC6
S21444F3700C0093F0000F01F0004C02BF490011F45A
S21444F380000F013BF9D041EA0C018FE70CEAD15358
S21444F39092EA0C0F18BF93EA0C0F0AD030F0004CD8
S21444F3A018BF31F0004CD8D180EA010000F000408C
S21444F3B0704790F0000F17BF90F0004F084691F04A
S21444F3C0000F91F0004F14D092EA0C0F01D1420284
S21444F3D00FD193EA0C0F03D14B0218BF084608D14D
S21444F3E080EA010000F0004040F0FE4040F4000097
S21444F3F0704740F0FE4040F4400070474FF0FF0C2A
S21444F4001CEAD0521EBF1CEAD15392EA0C0F93EA70
S21444F4100C0F69D0A2EB030280EA010C49024FEAC2
S21444F420402037D04FF0805343EA111143EA10137B
S21444F4300CF000408B4238BF5B0042F17D024FF433
S21444F440000C8B4224BF5B1A40EA0C00B3EB510F0E
S21444F45024BFA3EB510340EA5C00B3EB910F24BFF7
S21444F460A3EB910340EA9C00B3EBD10F24BFA3EB7C
S21444F470D10340EADC001B0118BF5FEA1C1CE0D144
S21444F480FD2A3FF650AF8B4240EBC25008BF20F0F7
S21444F490010070470CF0004C4CEA50207F32C2BF4B
S21444F4A0D2F1FF0340EAC250704740F400004FF0E8
S21444F4B00003013A37E792F0000F00F0004C02BF19
S21444F4C0400010F4000F013AF9D040EA0C0093F0E3
S21444F4D0000F01F0004C02BF490011F4000F013B3D
S21444F4E0F9D041EA0C0195E70CEAD15392EA0C0FA5
S21444F4F008D142027FF47DAF93EA0C0F7FF470AFDD
S21444F500084676E793EA0C0F04D14B023FF44CAF1F
S21444F51008466EE730F0004C18BF31F0004CCAD1B4
S21444F52030F000427FF45CAF31F000437FF43CAFF0
S21444F5305FE700BF4FF0FF3C06E000BF4FF0010C12
S21444F54002E000BF4FF0010C4DF804CD4FEA4002F4
S21444F5504FEA41037FEA226C18BF7FEA236C11D03E
S21444F56001B052EA530C18BF90EA010F58BFB2EBF1
S21444F570030088BFC81738BF6FEAE17018BF40F071
S21444F580010070477FEA226C02D15FEA402C05D125
S21444F5907FEA236CE4D15FEA412CE1D05DF8040BAA
S21444F5A0704700BF844608466146FFE70FB5FFF73D
S21444F5B0C9FF002848BF10F1000F0FBD4DF808EDF5
S21444F5C0FFF7F4FF0CBF012000205DF808FB00BFE6
S21444F5D04DF808EDFFF7EAFF34BF012000205DF840
S21444F5E008FB00BF4DF808EDFFF7E0FF94BF01208D
S21444F5F000205DF808FB00BF4DF808EDFFF7D2FF8A
S21444F60094BF012000205DF808FB00BF4DF808EDCC
S21444F610FFF7C8FF34BF012000205DF808FB00BF99
S21444F62042000ED2B2F1FE4F0BD34FF09E03B3EB23
S21444F630126209D44FEA002343F0004323FA02F04F
S21444F64070474FF00000704712F1610F01D142023B
S21444F65002D14FF0FF3070474FF00000704700BFB4
S21444F66053B94AB9002908BF00281CBF4FF0FF31E0
S21444F6704FF0FF3000F0A6B9ADF1080C6DE904CEAA
S21444F68000F03EF8DDF804E0DDE9022304B07047FC
S21444F69038B505460C462846214600220023FFF787
S21444F6A015FC28B928462146BDE8384000F00AB87B
S21444F6B0284604F1004100F005F8404261EB410160
S21444F6C038BD00BFD0B50C4B002206460F46FFF7A8
S21444F6D08BF9FFF761FC0446FFF70CF9074B002251
S21444F6E0FFF782F902460B4630463946FEF7C4FF1A
S21444F6F0FFF752FC2146D0BD0000F03D0000F0412B
S21444F7002DE9F047089D0E4604468C46002B40F0F3
S21444F71081808A42174645D9B2FA82F24AB1C2F18A
S21444F720200106FA02F320FA01F1974041EA030C5D
S21444F73094404FEA174E230CBCFBFEF6B9B20EFBC0
S21444F74016CC43EA0C4306FB01F0984209D9FB1851
S21444F75006F1FF3C80F01581984240F21281023E49
S21444F7603B441B1AA4B2B3FBFEF00EFB103344EA30
S21444F770034400FB01F1A14209D93C1900F1FF33CF
S21444F78080F00181A14240F2FE8002383C44641A73
S21444F79040EA064000211DB1D4400023C5E9004399
S21444F7A0BDE8F08702B9FFDEB2FA82F2002A4FD1F2
S21444F7B0CB1B4FEA174E1FFA87F80121B3FBFEFC1A
S21444F7C0260C0EFB1C3346EA034608FB0CF3B342F6
S21444F7D007D9BE190CF1FF3002D2B34200F2EB80D7
S21444F7E08446F61AA3B2B6FBFEF00EFB106643EA56
S21444F7F0064408FB00F8A04507D93C1900F1FF333E
S21444F80002D2A04500F2D2801846A4EB080440EA8F
S21444F8100C40C0E78B4208D9002D00F0AF80002191
S21444F820C5E900060846BDE8F087B3FA83F1002927
S21444F83049D1B34202D3824200F2BB80841A66EBBB
S21444F840030301209C46002DAAD0C5E9004CA7E737
S21444F850C2F120039740D8409140DE404FEA174E0D
S21444F86008434FEA104CB6FBFEF11FFA87F80EFB2E
S21444F87011664CEA064601FB08F3B34204FA02F466
S21444F88009D9BE1901F1FF3C80F08E80B34240F2A4
S21444F8908B8002393E44F31A86B2B3FBFEF00EFB6D
S21444F8A0103346EA034600FB08F3B34207D9BE19B1
S21444F8B000F1FF3C74D2B34272D902383E44F31A84
S21444F8C040EA01417AE7C1F1200703FA01F422FA3B
S21444F8D007F31C4320FA07F906FA01F34FEA144CDF
S21444F8E0FE4049EA03094FEA1943B6FBFCFE1FFAF9
S21444F8F084F80CFB1E6643EA06460EFB08FAB2453D
S21444F90002FA01F200FA01F308D9A6190EF1FF3003
S21444F91048D2B24546D9AEF1020E2644A6EB0A06B4
S21444F9201FFA89F9B6FBFCF00CFB106649EA06465A
S21444F93000FB08F8B04507D9A61900F1FF3C2DD2C4
S21444F940B0452BD90238264440EA0E40A6EB0806BA
S21444F950A0FB02894E45C446CE4618D315D075B38F
S21444F960B3EB0C0266EB0E0606FA07F722FA01F32F
S21444F970CE401F43C5E90076002111E729462846B4
S21444F9800EE76646EDE6184601E74345E7D2B8EB90
S21444F990020C69EB04040138A646E0E76046D3E768
S21444F9A060468CE78646B9E7614674E702383C44CD
S21444F9B02BE7084647E7ACF1020C3E4411E72946DC
S21444F9C0EEE600BF704700BF2DE9F04788B0002B35
S21444F9D01F461446B8BF03F10043129A109DDDF843
S21444F9E04CA0B6BF1F4600232D231370149B23F050
S21444F9F02008B8F1460F05D0B8F1450F00D10135BF
S21444FA00022300E0032307AA049206AACDE902A231
S21444FA10CDE9003522463B4601F0A6FDB8F1470F36
S21444FA20064602D1119BDB0722D5B8F1460F06EBFA
S21444FA30050910D13378302B0AD100220023204602
S21444FA403946FFF739FA18B9C5F10105CAF8005026
S21444FA50DAF8003099440022002320463946FFF75E
S21444FA602BFA08B1CDF81C903022079B4B4507D3A0
S21444FA70079B159A9B1B3046136008B0BDE8F08779
S21444FA80591C07911A70F0E7F7B503460029B8BF2A
S21444FA90494203F8022BB4BF2D222B220929427077
S21444FAA02ADD0DF10704A4460A27A6460A4691FB1A
S21444FAB0F7F607FB16153035632A04F1FF340EF8C3
S21444FAC0015C3146F1DC3031AEF1020504F8011C2C
S21444FAD0441C294661450AD30DF10902A2EB0E02E5
S21444FAE0654588BF00221344181A03B0F0BD11F8C8
S21444FAF0012B04F8012FEDE7302330318370C170B9
S21444FB00031DF1E72DE9F04F91B00C46DDF868800F
S21444FB1016461F46054602F04DFE036809931846EE
S21444FB20FEF74CFD00230E93D8F800300A900733B6
S21444FB3023F0070303F1080294F81890D4F800B0B1
S21444FB40C8F80020D3E90023C4E91223D4E9128A72
S21444FB502AF000430B930B999C4B4FF0FF324046E0
S21444FB60FFF7DCF970BB994B0B994FF0FF324046D8
S21444FB70FFF7B6F930BB0022002340465146FFF754
S21444FB80A5F910B12D2384F84330914B9148B9F12F
S21444FB90470F94BF98468046032323612BF0040303
S21444FBA023604FF0000A009733460FAA21462846A2
S21444FBB000F0D2F9013040F08F804FF0FF3011B0A2
S21444FBC0BDE8F08F4246534640465146FFF7A6F9F5
S21444FBD040B1BAF1000FBCBF2D2384F843307E48B1
S21444FBE07E4BD4E763685A1C09F0DF0142D10623F2
S21444FBF06360002206920EAACDE904920DAA4BF445
S21444FC00806303920DF13302CDE9013223606368C9
S21444FC1000934246534628460B91FFF7D5FE0B9970
S21444FC20472980460D9908D1C81C02DB636899426F
S21444FC3040DDA9F102095FFA89F9B9F1650F1FD8C9
S21444FC4001394A4604F150000D91FFF71DFF0E9A04
S21444FC501318012A8246236102DC2268D20701D5A2
S21444FC60013323619DF83330002B9CD02D2384F838
S21444FC70433098E74729BCD1002BBAD10123B7E7D4
S21444FC80B9F1660F18D1002963680BDD216113B9F9
S21444FC902268D00702D501330B442361A1654FF097
S21444FCA0000ADFE713B92268D20701D50233F4E726
S21444FCB00123F2E74FF067090E9B994205DB236860
S21444FCC02161D807EAD54B1CE7E70029D4BFC1F128
S21444FCD0020201221344E0E723685A0507D4236945
S21444FCE0424631462846B84701302BD165E7B9F13C
S21444FCF0650F40F2DC80D4E9120100220023FFF7AE
S21444FD00DBF8002833D0364A012331462846B84724
S21444FD1001303FF452AFDDE90D239A4202DB2368FB
S21444FD20D8070FD5DDE9092331462846B8470130C0
S21444FD303FF443AF4FF0000804F11A090E9B013B11
S21444FD40434509DC23689B0700F10181E0680F9B6B
S21444FD509842B8BF184632E701234A4631462846F9
S21444FD60B84701303FF429AF08F10108E6E70D9B98
S21444FD70002B37DC1A4A012331462846B84701305F
S21444FD803FF41BAFDDE90D23134302D12368D907A3
S21444FD90D8D5DDE9092331462846B84701303FF433
S21444FDA00CAF4FF0000904F11A0A0D9B5B424B4519
S21444FDB001DC0E9B94E70123524631462846B84759
S21444FDC001303FF4FAAE09F10109EEE7FFFFEF7F99
S21444FDD0EE7F4600F27F4600FA7F4600F67F4600F6
S21444FDE0FE7F46000E9AA36D9A42A8BF1A46002A82
S21444FDF0914637DC4FF0000B29EAE97904F11A0200
S21444FE00D4F858A0AAEB09035B4533DCDDE90D239F
S21444FE109A423BDB2368DA0738D40E9A0D99A2EB54
S21444FE200A03A2EB01099945A8BF9946B9F1000F08
S21444FE3034DC4FF0000829EAE97904F11A0ADDE9CE
S21444FE400D239B1AA3EB090343457FF77BAF01239E
S21444FE50524631462846B84701303FF4AEAE08F124
S21444FE600108ECE71346314642462846B847013077
S21444FE70C0D1A2E60123314628460B92B84701304A
S21444FE803FF49BAE0B9A0BF1010BB9E7DDE909236E
S21444FE9031462846B8470130BFD18EE64B4608EB7C
S21444FEA00A0231462846B8470130C2D185E60E9A42
S21444FEB0012A01DCDB0737D5012342463146284672
S21444FEC0B84701303FF479AEDDE909233146284688
S21444FED0B84701303FF471AED4E912010022002342
S21444FEE0FEF7EAFFD8B90E9B08F10102013B314602
S21444FEF02846B84701300ED15FE601234A463146CC
S21444FF002846B84701303FF458AE08F101080E9B26
S21444FF10013B4345F1DC534604F15002E1E64FF021
S21444FF20000804F11A09F2E701234246DFE70123F9
S21444FF304A4631462846B84701303FF43EAE08F1BB
S21444FF400108E3680F995B1A4345F0DCFEE64FF080
S21444FF50000804F11909F4E72DE9F04716469946D6
S21444FF608A680B69DDF820809342B8BF1346336035
S21444FF7091F8432007460C460AB1013333602368A0
S21444FF80990642BF336802333360256815F0060588
S21444FF9006D104F1190AE36832689B1AAB4226DCA0
S21444FFA094F84320131E226818BF012392062BD4CC
S21444FFB004F1430249463846C04701301ED0236800
S21444FFC0E568326803F00603042B08BFAD1AA3683D
S21444FFD022690CBF25EAE57500259342C4BF9B1AE7
S21444FFE0ED1800261A34B5421AD1002008E0012341
S21444FFF0524649463846C047013003D14FF0FF3099
S214450000BDE8F0870135C6E7E1185A1C302081F86F
S2144500104300224494F8451082F843100233C7E75C
S2144500200123224649463846C0470130E6D00136C8
S214450030D9E700002DE9FF470C469146277E0C99E7
S214450040782F80469A4604F1430207D8622F0AD88D
S214450050002F00F0D880582F00F0A38004F1420608
S21445006084F842703AE0A7F16303152BF6D801A051
S21445007050F823F0CD004500E10045005D00450001
S2144500805D0045005D0045005D004500E10045001A
S2144500905D0045005D0045005D0045005D0045008E
S2144500A0ED01450011014500CF0145005D004500C5
S2144500B05D0045000F0245005D0045001101450005
S2144500C05D0045005D004500D70145000B681A1DDB
S2144500D01B680A6004F1420684F842300123A3E017
S2144500E0256808682E0600F104030AD505680B60E6
S2144500F0002D03DA2D236D4284F843305E480A23EB
S21445010019E015F0400F05680B6018BF2DB2EFE7F4
S2144501100B682568181D0860280601D51D6802E08D
S2144501206906FBD51D8854486F2F0CBF08230A2344
S214450130002184F843106668A660002EA2BF216899
S21445014021F0040121600DB9002E4DD01646B5FBB1
S214450150F3F103FB1157C75D06F8017D2F46BB42F9
S2144501600D46F4D9082B0BD12368DF0708D523693C
S21445017061689942DEBF302306F8013C06F1FF363A
S214450180921B2261CDF800A04B4603AA2146404665
S214450190FFF7E2FE01304CD14FF0FF3004B0BDE82A
S2144501A0F087354884F8457023680E681F0656F86C
S2144501B0045B0E6014D5D90744BF43F02003236083
S2144501C01DB9236823F0200323601023B0E7236876
S2144501D043F0200323607823284884F84530E3E736
S2144501E05E0648BFADB2E6E71646BBE70B6826682F
S2144501F060691D1D0D6035061B6801D5186002E057
S2144502007106FBD51880002323611646BAE70B68AE
S2144502101A1D0A601E68626800213046FEF7D8F946
S21445022008B1801B606063682361002384F843300F
S214450230A8E72369324649464046D0470130ABD009
S21445024023689B0713D4E068039B9842B8BF1846BB
S214450250A4E70123324649464046D04701309BD065
S2144502600135E36803995B1AAB42F2DCEBE7002500
S21445027004F11906F5E700BF0080460011804600E8
S2144502802DE9F04F87B0174603938B685A1EB2F593
S214450290AE7F83BF6FF4AE755B190293002386BFAE
S2144502A040F25D138B6002930B688B46002543F442
S2144502B0F0634BF81C3BCDE9045580460C465E463C
S2144502C0AA46A9460195A26852B13B681B784E2BB3
S2144502D064D8402B3CD8A3F12B01C8B20E283AD996
S2144502E0B9F1000F03D0236823F4807323600AF125
S2144502F0FF3ABAF1010F00F213815E4500F205811F
S2144503000125284607B0BDE8F08FA3F161020D2A06
S214450310E6D801A151F822F057044500E102450010
S214450320E1024500E1024500B70445008F0445005B
S214450330E1024500E102450065044500E10245004D
S214450340E1024500E1024500E10245001D04450085
S214450350A3F14102DBE70E29C2D801A050F821F0EF
S2144503600F044500E10245000F044500A30445007F
S214450370E1024500BD034500F9034500F903450084
S214450380F9034500F9034500F9034500F90345001F
S214450390F9034500F9034500F90345006E2B09D8D6
S2144503A0602BB2D8542B77D0592B99D1072D97D19E
S2144503B0082529E0742B6FD0792BF6E72168C80508
S2144503C01AD5029B21F08001216009F101091BB174
S2144503D0013B01320293A260A368013BA3602369F7
S2144503E0013323617B68013B002B7B6040F38480AF
S2144503F03B6801333B6066E71AEB050F7FF470AF49
S214450400226822F4C072226006F8013BE4E72268BF
S21445041010067FF565AF22F08002F4E7BAF1000FCB
S2144504200ED1B9F1000F0ED1226802F4E061B1F5A4
S214450430E06F08D122F4F06222604FF0010AE3E74C
S214450440BAF1020F55D0012D02D0042D7FF448AFE6
S2144504500135EDB2D8E7BAF1010F7FF441AF4FF061
S214450460020AD1E77DB9B9F1000F7FF43CAF2268A7
S21445047002F4E061B1F5E06F7FF439AF22F4F06243
S21445048022600125C0E7032DE2D0052DDEE7022DCB
S2144504907FF426AF0325B7E7062D7FF421AF072562
S2144504A0B2E7226891057FF51BAF22F420722260E1
S2144504B0CDF80490A8E7226802F4A061B1F5806FF4
S2144504C006D050057FF50CAFB9F1000F3FF40FAFDE
S2144504D0910558BF019922F4F06258BFA9EB010176
S2144504E042F4C07258BFCDE9041622604FF00009A9
S2144504F08AE74FF0030A87E7D4F880313946404605
S214450500984700283FF4DFAEEAE6D4F87C3116F883
S214450510011D3A46404698472369013B2361ECE670
S2144505206B1E062B25D8022D36D85E457FF6E8AEDF
S214450530D4F87C3116F8011D3A464046984723695B
S214450540013B2361F1E70298D4F87C3110F8011D90
S21445055002903A46404698472369013B23610AF193
S214450560FF3A5FFA8AFABAF1020FECD1033DEDB2D3
S214450570761B2368DA052FD55B0510D55E457FF6D5
S214450580BFAED4F87C3116F8011D3A46404698472A
S2144505902369013B2361F1E7AA460296DFE716F891
S2144505A0011C2369652903F1FF3306F1FF352361F5
S2144505B00CD045290AD0D4F87C313A46404698476F
S2144505C0236916F8021C013BB51E2361D4F87C311D
S2144505D03A46404698472E46256815F0100559D1A7
S2144505E03570236803F4C063B3F5806F1CD1019B57
S2144505F04B45A3EB090224D100225946404600F05C
S21445060083FED4F800C0039B1CF0020F1B68064609
S2144506100F4621D003991A1D0A601B68C3E9006777
S214450620E3680133E3606CE6049B002BE4D0059950
S2144506300A232A460131404600F0E6FE049B059E05
S214450640C21A04F26F139E4228BF04F5B7761249C4
S214450650304600F029F8CFE71CF0040F03F1040EEE
S21445066003D00399C1F800E0D7E7039AC2F800E043
S214450670D3F8008002460B46FEF750FC28B10748E3
S21445068000F00EF8C8F80000CAE730463946FEF7CF
S214450690A3FCF7E7002534E6228046000C7B46009F
S2144506A0004870470000C07F0EB400B59AB01BAB3B
S2144506B0019005906FF0004109480691039109495C
S2144506C053F8042B04910068009301A902F0E4FD59
S2144506D0019B00221A701AB05DF804EB03B0704710
S2144506E0EC2240200802FFFF2DE9F0410F469046D8
S2144506F002F084FB04460D46B8F1000F11D0C7F34F
S2144507000A53C3F16B03002B0BDD1B0503F17F5525
S214450710002405F5401522462B46FEF765F90446A6
S2144507200D4620462946BDE8F08100000000000041
S2144507302DE9F04FA1B09B4600231C939E4B179284
S2144507401F68824638460E46FDF738FF4FF00008CC
S21445075004464FF000091B961B9B1A782B2A4CD053
S2144507603AD80D2A33D8082A33D8002A3DD0002354
S2144507700C931B9D2B78302B40F0A9806B7803F0AB
S214450780DF03582B66D10C9B01931CAB00938B4A19
S214450790CDF808B01DAB1BA9504601F01FFD10F063
S2144507A00706044605D0062E29D1013500231B959C
S2144507B00C93179B002B40F08E850C9BD3B142467D
S2144507C009F100431046194621B0BDE8F08F202AAE
S2144507D0CDD101331B93BFE72D2AC8D101220C92F8
S2144507E05A1C1B925B78002BC3D1179B1B96002B7C
S2144507F040F06F8542464B46E4E70022EFE71C9AF9
S2144508003AB135211EA802F0F0FB1C99504602F07D
S21445081031F8013E042E06D8DFE806F00A03141721
S2144508200A00DDE91E892107C3D549F00049C0E71E
S214450830DDE91E831D9A23F4801302F2334243EA10
S2144508400259F0E7DFF87891EDE76FF000494FF091
S214450850FF38E8E71B9B5A1C1B925B78302BF9D078
S214450860002BA6D0012307931B9B08930023CDE9B5
S21445087005339B460A221B980578A5F13003D9B265
S214450880092926D92246394602F01CFE002832D0D0
S21445089000202B465C4604900246652B01D0452B2E
S2144508A013D11CB9079B03439FD000241B9E731C82
S2144508B01B9373782B2B78D02D2B7BD00027A3F159
S2144508C03001092940F282801B9600259EE00023D0
S2144508D0C9E7BBF1080FD5BF0699059902FB013359
S2144508E002FB013300F10100D4BF069305930BF1DB
S2144508F0010B1B90BFE71B9B1A191B921B5DBBF197
S214450900000F36D004905C46A3F13002092A12D96E
S2144509100122C2E71B9B5A1C1B925B780130302B89
S214450920F8D0A3F13102082A00F2DA841B9A049023
S214450930002008920446303B00F1010213D004998A
S21445094011440491224605190A21954213D12218CD
S214450950082A04F1010404441BDC06990A2202FB1A
S2144509600133069300221B9B591C1B915B7810464E
S214450970CAE75846D3E7082A04DC069F4F4306973E
S2144509800132E2E7571C102FDEBF059F4F43059700
S214450990F6E7102CDFBF05990A2202FB01330593C3
S2144509A0E0E70023049301227CE70027B31C1B9352
S2144509B0B37884E70127F9E7888146002880460012
S2144509C00000F07F1B9B591C1B915B78302BF9D0A0
S2144509D0A3F1310108293FF678AFA3F1300C1B9BF4
S2144509E009934FF00A0E1B9B591C1B915B78A3F18C
S2144509F03005092D35D9099D491B082944F61F653B
S214450A0002DC6545A8BF654607B16D42002C4CD152
S214450A10079901437FF4CDAE002A7FF4E6AE692BF5
S214450A2026D023DC492B23D04E2B7FF4DEAE9C49C3
S214450A301BA801F00FFE00283FF4D7AE1B9B1B7882
S214450A40282B2CD197491EAA1BA801F017FE05286E
S214450A5025D11F9BDDF8788043F0FF4949F4E0092E
S214450A60A7E60EFB0C3CACF1300CBCE76E2BDCE786
S214450A708D491BA801F0EEFD00283FF4B6AE1B9B42
S214450A808A49013B1BA81B9301F0E4FD10B91B9B4B
S214450A9001331B93DFF824924FF0000889E684481B
S214450AA002F00AFD8046894683E6049B0698EB1AC3
S214450AB0BBF1000F08BFA346102C07932646A8BFD8
S214450AC01026FDF717FF092C8046894613DD794B1E
S214450AD003EBC60353E91223FDF786FF80460598C8
S214450AE08946FDF707FF02460B4640464946FDF751
S214450AF0C5FD804689460F2C36DC079B002B3FF408
S214450B0058AE22DD162B09DC6A4C04EBC304D4E947
S214450B10000142464B46FDF767FFC3E7079AC4F117
S214450B202503934220DB634DC4F10F0405EBC40156
S214450B3042464B46D1E90001FDF756FF079B1C1B75
S214450B4005EBC405D5E90023E5E7079B16330BDB24
S214450B50049B584A5D1B02EBC505D5E90023404674
S214450B604946FEF76BF89DE7079BA61B1E44002EDD
S214450B7071DD16F00F030AD04E4901EBC30142461C
S214450B804B46D1E90001FDF72FFF8046894636F0F2
S214450B900F0650D0B6F59A7F27DD4FF0000BCDF8FF
S214450BA010B0CDF820B0CDF818B02223DFF80C9160
S214450BB0CAF800304FF00008089B002B3FF4F9AD0B
S214450BC01C99504601F056FE0699504601F052FED5
S214450BD00499504601F04EFE0899504601F04AFEEB
S214450BE05946504601F046FEE3E500233611404699
S214450BF049461F46012E21DC0BB1804689462E4BC1
S214450C00A9F1547903EBC70742464B46D7E900019D
S214450C10FDF7EAFE294B0A460B4029498B4280469A
S214450C20BBD8A1F580118B4286BFDFF898904FF070
S214450C30FF3802F15479002305937EE0F20707D585
S214450C401D4B03EBC703D3E90023FDF7CDFE012378
S214450C5001377610CEE7EED0764216F00F020AD070
S214450C60144B03EBC20340464946D3E90023FDF740
S214450C70E5FF804689463611DDD01F2E24DD4FF030
S214450C80000BCDF810B0CDF820B0CDF818B0222323
S214450C904FF000084FF00009CAF800308CE700BF57
S214450CA0FB7F46003C804600F37F46007C8146003D
S214450CB00C7B4600C8814600A08146000000F07FB8
S214450CC00000A07CFFFFEF7F16F0100318BF6A23D5
S214450CD0B34F0593404649460023F20704D5D7E966
S214450CE00023FDF781FE0123761007F10807F4D1AE
S214450CF00BB180468946059BBBB1C9F30A53C3F180
S214450D006B03002B494610DD1F2B40F32881342BFF
S214450D10DEBF203B4FF0FF3202FA03F34FF00008E8
S214450D20CCBF4FF05C7903EA010900220023404618
S214450D304946FEF7C1F80028A1D1069B00930899BD
S214450D4023465A46504601F0EAFD089000283FF4EF
S214450D5024AF049B5D1B079B002BB4BF2B4600238B
S214450D600E93079B4FF0000B23EAE3731693CDF8DB
S214450D7010B0089B5046596801F048FD069000287B
S214450D803FF413AF089B1A69023203F10C01920037
S214450D900C3001F02DFD1EAB01931DAB0093424672
S214450DA04B465046CDE90A8902F0A2F81C90002829
S214450DB03FF4FBAE0121504601F03DFE049003464C
S214450DC000283FF4F2AE1D9D1E9A002DABBF0E9B2C
S214450DD0169B169C0E9EACBFEE185C1B059BED1A2B
S214450DE01544704B013D9D42C2F1360280F2C980E2
S214450DF05B1B1F2BA2EB03024FF0010700F3B680E7
S214450E0007FA03F30F930025B718059BBE42144413
S214450E101C443346A8BF3B46A342A8BF2346002BE7
S214450E20C2BFFF1AE41AF61A0E9B002B17DD04996B
S214450E301A46504601F0A4FE049000283FF4B5AE8D
S214450E4001461C9A504601F0FFFD099000283FF4E4
S214450E50ACAE1C99504601F00DFD099B1C93002F26
S214450E6000F39380079B002B08DD169A069950469B
S214450E7001F086FE069000283FF497AE002C08DD6C
S214450E8006992246504601F0C9FE069000283FF4D2
S214450E908CAE002E08DD04993246504601F0BEFE63
S214450EA0049000283FF481AE069A1C99504601F0FE
S214450EB02FFF834600283FF478AE0024C368049984
S214450EC0C4600D9301F009FFA04271DA0D9B53EA09
S214450ED0080340F09780C9F31303002B40F0928037
S214450EE029F000431B0D1B05B3F1D66F40F28A80EF
S214450EF0DBF8143023B9DBF81030012B40F3828041
S214450F0059460122504601F089FE0499834601F070
S214450F10E4FE002876DD0599234A4B46002900F075
S214450F20928002EA0901B1F1D66F00F38C80B1F1E7
S214450F305C7F7FF7ACAE1D4A0023CDE914324046B0
S214450F40DDE914234946FDF74FFD0B46034308BF2D
S214450F5022238046894608BFCAF8003030E64FF05F
S214450F60FF3202FA03F303EA0808DEE6C5F17F45D9
S214450F7005F57F0505F57B45E23507FA05F50F9737
S214450F8042E7012300250F933EE71C993A46504613
S214450F9001F044FE1C9000287FF464AF05E600BFD0
S214450FA05080460002FCFFFF0000F07F00005039ED
S214450FB0CDF8249066D10D9AC9F313035AB39C4ACB
S214450FC093422CD1059B404603B39A4A4B461A405A
S214450FD0B2F1D46F4FF0FF311BD8120DC2F16B033F
S214450FE001FA03F398421AD1934B099A9A4202D1D1
S214450FF001303FF4DAAD8F4B099A1A4002F5801955
S2144510004FF00008059B002B95D1D9E54FF0FF33EF
S214451010E8E70B46E6E753EA08033FF47CAFE5B15D
S214451020099B1D42EED00D9B059A40464946C3B1E5
S214451030FFF75AFB02460B46DDE90A01FDF71EFBA4
S21445104080468946DEE71340A3F580136FEA1359B9
S2144510506FEA09594FF0FF38D4E70F9B13EA080F9C
S214451060E0E7FFF741FB02460B46DDE90A01FDF7DF
S21445107003FB0022002380468946FDF71DFF002816
S214451080C0D004E60499584601F081FF00224FF08F
S214451090804306460F46FDF723FF002875D00D9B77
S2144510A0002B47D0654F0026644D099B23F000432F
S2144510B01B0D1B050F930F9A614B9A4240F0C88053
S2144510C0DDE90A23CDE91423099BA3F1547940466B
S2144510D0494601F093FE02460B4630463946FDF733
S2144510E083FC42464B46FDF7C9FA0B465149554ADD
S2144510F01940914280465ED90B9B02F15472934249
S21445110003D10A9B01333FF450ADDFF82C914FF0E5
S214451110FF381C99504601F0ADFB0699504601F044
S214451120A9FB0499504601F0A5FB5946504601F0E7
S214451130A1FB1EE6B8F1000F19D1099BC3F31303B3
S214451140E3B93E4B002230463946FDF7BFFEC8B9E7
S2144511503D4B002230463946FDF746FC04460D46D3
S21445116005F1004318941993DDE918679DE7B8F132
S214451170010F03D1099B002B3FF489AD334F002661
S214451180002491E70D9C304DEAE72F4B0022304670
S2144511903946FDF729FC0D9B04460D4633B901F14A
S2144511A0004310901193DDE910677EE702460B4633
S2144511B0CDE91023F7E703F15479059B002BA8D119
S2144511C029F000430F9A1B0D1B059A42A1D12046D4
S2144511D02946FEF75DFAFDF7D9FB02460B46204643
S2144511E02946FDF749FA0D9AC9F3130343EA08035E
S2144511F0134304460D4666D009A3D3E90023FDF7FD
S21445120065FE00287FF4DCAC07A3D3E9002320461F
S2144512102946FDF779FE00283FF47BAFD0E400BFB2
S2144512209535A094FFFFDF3F35E5AF350000E03F3D
S214451230FFFF0F000000F07FFFFFEF7F0000F03F4D
S2144512400000E07FFFFF9F7C0000E03F0000F0BF0E
S214451250059B13B30F9BB3F1D46F1ED826A3D3E9D2
S214451260002320462946FDF73BFE90B129462046F9
S214451270FDF792FE012838BF0120FDF73BFB0D9B8D
S21445128004460D46D3B901F1004312901393DDE9A8
S21445129012670F9A07F1D6639F1ADDE90A0101F036
S2144512A0ADFD02460B4630463946FDF79DFBDDE96A
S2144512B00A23FDF7E3F9804689467EE702460B4654
S2144512C0CDE91223E3E70EA3D3E90023FDF7FEFDA0
S2144512D0A1E700230C93179A1B9B1360FFF76DBA83
S2144512E0652B3FF45EAB452B3FF45BAB0122FFF726
S2144512F08FBB00BFAFF300800000C0FFFFFFDF419C
S2144513009535A094FFFFCF3F014BFFF711BA00BFBD
S214451310542340202DE9F0473A4E86468C46604693
S2144513201CF8014BA55D15F00805F8D12D2C33D1D9
S2144513309CF800404FF0010800F1020C002B5CD0F1
S214451340102B0CD1302C0AD19CF8000000F0DF00A1
S21445135058284DD19CF8014010230CF1020C08F199
S2144513600047013F0026B7FBF3F9304603FB197AE1
S214451370A4F13005092D18D82C46A34224DD751C4A
S21445138007D081451DD301D1A2451ADB00FB03409A
S21445139001261CF8014BEBE72B2C08BF9CF80040B8
S2144513A0A84608BF00F1020CC8E7A4F14105192D6F
S2144513B001D8373CE1E7A4F16105192D04D8573C1F
S2144513C0DBE74FF0FF36E4E7731C06D12223CEF861
S2144513D00030384642B9BDE8F087B8F1000F00D076
S2144513E04042002AF7D00EB10CF1FF311160F2E70A
S2144513F03024002BB3D10823B1E7302CA4D00A23E0
S214451400ADE700BF79804600FFF784BF00B59BB0C7
S214451410019105916FF000410691039105490491AC
S21445142001A901F039FF019B00221A701BB05DF837
S21445143004FB00BF0802FFFF13460A460146024862
S2144514400068FFF7E3BF00BFEC2240202DE9F74FC9
S21445145003690C69A3420746C0F28180013C01F14D
S214451460140800F1140505EB8403019358F824305D
S21445147055F8242001339A424FEA840B08EB840939
S214451480B2FBF3F631D34FF0000E4046AC46F2467B
S21445149050F8042B93B206FB03E34FEA134E9BB278
S2144514A0AAEB0303120CDCF800A006FB02E213FAD3
S2144514B08AF34FEA124E1FFA82FADCF80020CAEB8E
S2144514C0124202EB23429BB243EA024381454CF863
S2144514D0043B4FEA224ADBD255F80B302BB9019B29
S2144514E0043B9D421A462ED33C61384601F0F5FB37
S2144514F0002824DB013628464FF0000C58F8042B0C
S214451500D0F800E093B2ACEB0303120C13FA8EF35B
S214451510C2EB1E4202EB23429BB243EA0243C1455D
S21445152040F8043B4FEA224CE8D255F8242005EB18
S214451530840322B9043B9D421A460AD33C61304691
S21445154003B0BDE8F08F1268043B002ACCD1013CBD
S214451550C7E71268043B002AF0D1013CEBE70020C0
S214451560EEE70000000000002DE9F04F446A99B010
S21445157016461F46CDE90467DDF8948005463CB916
S214451580102001F01BF9C0E9014468620460C4609C
S2144515906B6A196851B15A684A60012393408B605B
S2144515A0284601F067F96B6A00221A603B1EB9BFF0
S2144515B023F0004305930023C8F80030DDF8149067
S2144515C0A74BBCBF0122C8F8002033EA090319D14E
S2144515D0249A42F20F731360C9F31303334300F0A2
S2144515E06D85269B53B99F4B23E09F4B039308334A
S2144515F0269A1360039819B0BDE8F08F994B03936C
S2144516000333F5E7DDE90434CDE90C34DDE90C01B7
S21445161000220023FDF750FC804660B1249A012342
S2144516201360269B002B00F04685904B269A136048
S214451630013B0393DEE716AB019317AB00932846B1
S214451640DDE90C2301F054FCC9F30A548346002C0B
S2144516507ED00D9BCDF84C80C3F31303DDE90C011A
S21445166043F07F5141F44011A4F2FF34804B0022F1
S214451670FDF702F874A3D3E90023FDF7B5F974A383
S214451680D3E90023FCF7FAFF064620460F46FDF74A
S21445169041F971A3D3E90023FDF7A6F902460B46A7
S2144516A030463946FCF7EAFF06460F46FDF74CFC42
S2144516B000228246002330463946FDF707FC48B1EE
S2144516C05046FDF727F932463B46FDF7F5FB08B988
S2144516D00AF1FF3ABAF1160F57D8664B03EBCA0321
S2144516E0D3E90023DDE90C01FDF7F0FB00284ED0D9
S2144516F00AF1FF3A00230F93169B1C1B631E0993A2
S21445170045BFC4F101030693002300234CBF09934C
S2144517100693BAF1000F3CDB099BCDF838A053443D
S214451720099300230A93229B092B00F2B580052BCB
S214451730C4BF043B2293229BA3F10203CCBF0024E3
S2144517400124032B00F2B480DFE803F02D987AA439
S214451750DDE916431C4404F23243202BC3BFC3F1D4
S214451760400304F2124009FA03F3C3F12003C6BF4F
S21445177026FA00F0184306FA03F0FDF7BBF80123F6
S214451780A1F1F871013C139370E70123B3E70F907D
S214451790B2E7069BA3EB0A030693CAF100030A9336
S2144517A000230E93BFE700230B93239B002B00F3E8
S2144517B082804FF00109CDF820904B46CDF88C90AD
S2144517C06E6A00227260042202F114009842716823
S2144517D077D9284601F01AF86B6A30601B68039380
S2144517E0089B0E2B00F2EE80002C00F0EB80BAF141
S2144517F0000F7ADD1F4A0AF00F0302EBC303D3E955
S21445180000341AF4807FCDE910344FEA2A145CD0B0
S214451810194BDDE90C01D3E90823FDF70FFACDE9AD
S214451820040104F00F040327134E002C4FD1DDE9C5
S2144518301023DDE90401FDF701FACDE904016EE068
S2144518400123B1E7AFF3008061436F63A787D23FBB
S214451850B3C8608B288AC63FFB799F501344D33F55
S2144518600000F07F8281460079814600FF7F460072
S2144518700000F83FC8814600A081460000230B9330
S214451880239B0AEB030909F10103012B0893B8BF13
S214451890012395E70123F2E70124002322930B94C5
S2144518A04FF0FF390022CDF820901223239287E788
S2144518B001230B93F4E7DDF88C90CDF820904B464A
S2144518C07EE70131716052007EE70227ACE7E1070B
S2144518D008D5DDE91001D6E90023FDF785F8CDE901
S2144518E010010137641008369FE700F0A580CAF15D
S2144518F00004A44BA44E04F00F0203EBC203D3E945
S2144519000023DDE90C01FDF76FF8CDE9040124114C
S21445191000230227002C40F08480002B8DD10F9B9E
S214451920002B00F08B80DDE90434CDE91034DDE989
S2144519301001964B0022FDF7C9FA00287ED0089B79
S214451940002B7BD0B9F1000F38DDDDE91001904B57
S2144519500022FDF749F8CDE904010AF1FF380137C1
S2144519604C463846FCF7D6FFDDE90423FDF73CF840
S214451970884B0022FCF782FEA1F15076CDE9100196
S2144519801196002C5DD1DDE90401834B0022FCF75E
S21445199073FE02460B46CDE90423109A3346FDF7FF
S2144519A0B3FA002840F09782DDE90401109A06F163
S2144519B00043FDF78BFA002840F08B82DDE90C34B6
S2144519C0CDE90434179B002BC0F25181BAF10E0FB6
S2144519D000F34D816B4B03EBCA03D3E90034CDE9E5
S2144519E00634239B002B80F2DB80089B002B00F3FC
S2144519F0D78040F06D82684B0022DDE90601FCF792
S214451A00F3FFDDE90423FDF775FA089C2646002812
S214451A1040F04382039F312307F8013B0AF1010A50
S214451A203FE2E20705D5D6E90023FCF7DDFF01379F
S214451A300123641008366DE7022770E7089CD046F8
S214451A408FE703994F4B214412910B9903EBC4033F
S214451A50DDE9106753E90223002946D04F490020A7
S214451A60FDF7ECF83B463246FCF706FECDE910019D
S214451A70039FDDE90401FDF767FA0446FCF74AFFD4
S214451A8002460B46DDE90401FCF7F6FD3034024616
S214451A900B46CDE9042307F8014BDDE91023FDF796
S214451AA015FA002865D1DDE9042338490020FCF7FE
S214451AB0E3FDDDE91023FDF709FA002840F0B6807E
S214451AC0129B9F423FF47AAFDDE91001304B00226E
S214451AD0FCF78AFF2E4BCDE910010022DDE9040113
S214451AE0FCF782FFCDE90401C3E730463946FCF7EB
S214451AF07BFFCDE91001129B039C1493DDE904019D
S214451B00FDF722FA1590FCF705FF02460B46DDE980
S214451B100401FCF7B1FD159B303304F8013B129BDD
S214451B209C4206460F464FF0000224D11B4BDDE98A
S214451B301001FCF7A3FD02460B4630463946FDF735
S214451B40E3F9002871D1DDE9102314490020FCF79C
S214451B5093FD02460B4630463946FDF7B7F9002851
S214451B603FF42CAF149F7B1E149317F8013C302B83
S214451B70F8D0C24649E0064BFCF736FFCDE90401EE
S214451B80BCE700BFC8814600A08146000000F03F84
S214451B900000244000001C40000014400000E03FC8
S214451BA0DDE90489039FDDE9062340464946FDF7FE
S214451BB045F8FDF7C9F90446FCF7ACFEDDE9062312
S214451BC0FCF712FF04F130060B46024649464046EE
S214451BD0FCF752FD07F8016B039E089BBE1BB342FC
S214451BE038D102460B46FCF749FDDDE9062380461B
S214451BF08946FDF789F958BBDDE90623404649463F
S214451C00FDF75AF908B1E10722D42846594600F0AF
S214451C1031FE00233B70249B0AF101001860269B89
S214451C20002B3FF4E7AC1F60E4E427463B461F46DF
S214451C3013F8012D392A07D1039A9A42F7D1039909
S214451C40302208F101080A701A7801321A7090E7B6
S214451C50D046EBE7A14B0022FCF7C6FE0022002348
S214451C6080468946FDF728F900289CD0CDE70B9A93
S214451C70002A00F0CD80229A012A00F3AF80139AFD
S214451C80002A00F0A78003F233430A9C069F069A73
S214451C901A440692099A01211A442846099200F0E8
S214451CA0CAFE0646002F0CDD099B002B09DDBB420C
S214451CB0069AA8BF3B46D21A0692099AFF1AD31A25
S214451CC009930A9BF3B10B9B002B00F0A580002CD3
S214451CD010DD31462246284600F052FF5A46014658
S214451CE00646284600F0B0FE59468046284600F08F
S214451CF0C1FDC3460A9B1A1B04D05946284600F028
S214451D003FFF83460121284600F095FE0E9B002B9B
S214451D10044640F383801A460146284600F030FFC5
S214451D20229B012B04467CDD4FF00008236904EB1B
S214451D308303186900F031FEC0F12000099B184462
S214451D4010F01F0000F08E80C0F12003042B40F3F6
S214451D508780C0F11C00069B03440693099B0344F9
S214451D6007440993069B002B05DD59461A46284627
S214451D7000F054FF8346099B002B05DD21461A4695
S214451D80284600F04BFF04460F9B002B6CD021469F
S214451D90584600F0A2FF002866DA002359460A2274
S214451DA0284600F07EFD0B9B0AF1FF3A8346002B42
S214451DB000F08B81314600230A22284600F071FD4B
S214451DC0B9F1000F064600F39180229B022B40F3A3
S214451DD08D8051E0169BC3F1360356E7089B5C1E83
S214451DE00A9BA342BFBF0A9B0A94E21A0E9BB6BF44
S214451DF09B181C1B0E93089BB8BF0024002BB9BF2D
S214451E00069B089A069F089BBCBF9F1A00233EE781
S214451E100A9C069F0B9E45E70A9A6EE7229B012B76
S214451E2019DC049BBBB9059BC3F313039BB9059B00
S214451E3023F000431B0D1B0583B1069B0133069318
S214451E40099B013309934FF001080E9B002B7FF445
S214451E506DAF012072E74FF00008F6E79846F4E7C5
S214451E6080D018461C3076E7089B002B38DC229B32
S214451E70022B35DDDDF82090B9F1000F0DD1214656
S214451E804B460522284600F00CFD014604465846BA
S214451E9000F023FF00283FF7BDAD239B039F6FEA65
S214451EA0030A4FF000082146284600F0E3FC002EC2
S214451EB03FF4ABAEB8F1000F05D0B04503D0414670
S214451EC0284600F0D7FC3146284600F0D3FC9CE671
S214451ED000242646E1E7C24626469BE50000244008
S214451EE00B9BDDF82090002B00F0F680002F05DDDB
S214451EF031463A46284600F091FE0646B8F1000FB0
S214451F0055D07168284600F081FC32690232074692
S214451F10920006F10C010C3000F06AFC01223946AD
S214451F20284600F07BFE039B01330893039B4B44F6
S214451F300A93049B03F00103B04609930646089BA3
S214451F402146013B58460493FFF780FA0346303353
S214451F500690414658460B9300F0BFFE32468146F2
S214451F602146284600F0D4FEC2680B9B074602BBB6
S214451F700146584600F0B1FE0B9B024639462846B8
S214451F80CDE90B3200F076FC229B0C9A089F43EA7B
S214451F900201099B0B430B9B0DD1392B29D0B9F177
S214451FA0000F01DD069B3133049A13707BE73046FC
S214451FB0B9E70122E2E7B9F1000F06DB229941EACB
S214451FC00909099959EA010120D1002AECDD59464B
S214451FD001222846089300F021FE2146834600F05C
S214451FE07CFE0028089B02DCDED1DA07DCD5392BDF
S214451FF0D8D1049A392313703B461F46013B17F840
S214452000012C392A50D001321A704CE7002A03DDDC
S214452010392BEED00133C7E7089A0A9902F8013CF6
S2144520208A422AD0594600230A22284600F039FC1F
S214452030B04583464FF000034FF00A024146284616
S21445204007D100F02EFC80460646089B01330893D0
S21445205075E700F026FC3146804600230A222846CE
S21445206000F01FFC0646F0E7B9F1000F039ACCBF17
S2144520704F46012717444FF0000859460122284687
S214452080089300F0CBFD2146834600F026FE002847
S214452090B2DC02D1089BDB07AED43B461F4613F89D
S2144520A0012D302AFAD0FEE6039A9A42A5D10AF1C6
S2144520B0010A312379E7134BFFF7BBBA269B002B62
S2144520C07FF493AA104BFFF7B4BAB9F1000F03DCBF
S2144520D0229B022B3FF7D0AE039F21465846FFF77B
S2144520E0B5F900F1300307F8013B039ABA1A914552
S2144520F0BADD594600230A22284600F0D2FB83461D
S214452100EBE700BFFE7F4600798146000369B3EBE7
S214452110611F2DE9F0434FEA611200F1140445DDD5
S21445212011F01F0104EB830604EB82050CD100F188
S21445213010072946B14234D39B1A9B00EA1E9642A5
S21445214038BF0023234415E054F82270C1F1200817
S214452150CF4005F1040EA1467645F44615D89B1AA0
S2144521609A00043A0135AE4238BF0022A318A7505C
S21445217007B104331A1BA3424FEAA20208BF002345
S214452180026108BF4361BDE8F083DCF800C00CFA85
S21445219008FC4CEA070749F8047B5EF8047BCF4009
S2144521A0DAE751F804CB47F804CFC3E72346E1E71F
S2144521B0A0F13003092B02D82038C0B27047A0F1F1
S2144521C06103052B01D84738F7E7A0F14103052BF6
S2144521D001D82738F1E70020704700002DE9F04F79
S2144521E08BB08B460693BA4B02901B6803931846F2
S2144521F09046FCF7E3F9039BDBF800200344824650
S21445220013F8013C0793931CC2F1FF2202F57F02A7
S214452210FE32D1181F4613F8010B01913028F8D02D
S214452220FFF7C6FF044600283AD10399524638467A
S21445223001F048F90546002866D117F80A0007EB6D
S2144522400A06FFF7B5FF002860D0334618783028D1
S2144522501F4603F10103F9D0FFF7AAFF0123B0FAA1
S21445226080F46409354601933A461646013230787D
S214452270FFF79EFF0028F8D103995246304601F0F5
S21445228021F980B94DB906EB0A052A4616460132AC
S2144522903078FFF78DFF0028F8D1AD1BAD0004E080
S2144522A000242546E0E7002DF7D1337803F0DF0319
S2144522B0502B39D173782B2B2AD02D2B2CD0711C33
S2144522C04FF000090878FFF773FF431EDBB2182B63
S2144522D02AD8A0F1100211F8010FFFF769FF431E37
S2144522E0DBB2182B1BD9B9F1000F00D0524215446A
S2144522F0CBF80010D4B1019B002B14BF002706274E
S21445230038460BB0BDE8F08F3E4625460124CCE75F
S2144523104FF00009B11CD5E74FF00109FAE70A234B
S21445232003FB0202103AD6E73146E1E7F31B013BD1
S2144523302146072B50DC029800F068FA4FF0000B58
S21445234000F11409CAF101030446CDF81090CDF802
S21445235004B00893B74242D3049F019B47F8043B19
S214452360A7EB0907BF102761184600F016FB7F014B
S214452370D8F800603F1AB74265DDBF1B3946204690
S21445238000F056FE8246A8B17B1E591103F01F0287
S21445239059F821104FF0010A0AFA02F20A4209D00A
S2144523A0534505DDB91E204600F042FE002847D1BC
S2144523B04FF0020A39462046FFF7A8FE3D44D8F8B6
S2144523C00830AB424DDA0298214600F053FA149A8B
S2144523D000231360A32793E701315B10A9E7731E1B
S2144523E0079A059316F8013C934219D0BBF1200F86
S2144523F007D1049B019A43F8042B049300230193C9
S2144524009B4616F8010CFFF7D3FE019B00F00F0024
S21445241000FA0BF0034301930BF1040B059B0DE00B
S214452420059B089A1344BB42E0D318460399099383
S214452430524601F047F8099B0028D7D11E4689E742
S2144524404FF0030AB6E709DAF71B214602983A46E3
S21445245000F0E4FBED1B044600F114094FF0000ABA
S214452460ADE7D8F80400A8426DDD451BAE4231DC29
S214452470D8F80C30022B22D0032B24D0012B15D1B3
S214452480AE4213D1012E0BD1069AD8F8043013600C
S21445249001232361C9F80030149B62271C602FE78F
S2144524A0711E204600F0C4FD0028EDD10298214655
S2144524B000F0E0F9149A00231360502720E7159B97
S2144524C0002BF3D1E0E7159B002BDDD1EEE700BFEF
S2144524D0888146006F1EBAF1000F31D127B13946C3
S2144524E0204600F0A5FD82467B11012159F8233090
S2144524F007F01F0701FA07F71F422946204618BF6F
S2144525004AF0020A761BFFF701FED8F80450022768
S214452510BAF1000F48D0D8F80C30022B15D0032B53
S21445252017D0012B09D11AF0020F06D0D9F80000B2
S2144525304AEA000A1AF0010F0ED147F0100733E0B9
S2144525404FF0010AD0E70127E2E7159BC3F10103E7
S2144525501593159B002BF0D0D4F8109004F1140376
S2144525604FEA890B03EB89014FF0000C184653F8E8
S214452570042BB2F1FF3F1CD001320260022F04F15A
S214452580140338D1D8F80020013AB2420AD1711165
S214452590012253F8213006F01F0602FA06F61E42BF
S2144525A018BF174647F02007149B1C60069B1D6006
S2144525B0A6E6994243F804CCD8D8A368994512DBD9
S2144525C061680298013100F021F92269023204F16E
S2144525D00C01824692000C3000F00AF9214602981A
S2144525E000F048F9544623695A1C04EB83032261DC
S2144525F001225A61C2E722694A450BDD0121204680
S214452600FFF784FDD8F808300135AB42FFF6DBAE60
S2144526100127C7E716F01F06FAD09B44C6F12006E9
S2144526205BF8040C00F0B9F9B042E7DBF0E700BF11
S214452630C2F10802920070B5C2F1200643680468EC
S21445264003FA06F52C43D340046040F8043F88421D
S214452650F4D370BD30B50368013311F8014B14B996
S2144526600360012030BD13F8012BA2F14105192D59
S21445267098BF2032A242F0D00020F3E72DE9F04F74
S2144526800B6801685E1102EB860613F01F0387B0E0
S21445269018BF04360025371F82469046019346F8F4
S2144526A0045CB9463C460295AB464A784B1C0393B8
S2144526B042B3104605910492FFF77AFD00284FD1A4
S2144526C0049A0599202A18D8029B9B4513DD4C454C
S2144526D006D2072D04DC2A4649462046FFF7A8FFC2
S2144526E0444550D90023A4F1040944F8043CCDF8E8
S2144526F008B04C461D460399D7E7292A56D10231DC
S214452700CAF80010BBF1000F50D04C4506D2072D35
S21445271004DC2A4649462046FFF78AFF444534D915
S214452720A8F10402234653F8041B42F8041F9F42AF
S214452730F9D23B1B23F0030304330134033EB44272
S21445274088BF04234344002243F8042B9F42FBD210
S2144527503B681BB9474527D101233B60052026E04A
S2144527600135082D0BF1010B06DD4445C3D9002381
S21445277044F8043C0125043C226800F00F0040EA7A
S21445278002122260B7E70825B5E7019B002BDFD08C
S2144527904FF0FF32C3F1200322FA03F356F8042C18
S2144527A01A4046F8042CD3E7043FD1E7042007B087
S2144527B0BDE8F08F0048704744244020024B014650
S2144527C0186800F0B3BC00BFEC22402082B001B9C7
S2144527D001A942B14BB113780B601278101E18BF91
S2144527E0012002B070471046FBE76FF00100F8E79E
S2144527F00A44914200F1FF3300D1704710B511F8F5
S214452800014B03F8014F9142F9D110BD70B5466AA8
S21445281004460D463EB91020FFF7D0FFC0E90166D5
S21445282060620660C660666AF36883B1636ADB68A1
S21445283053F82500B8B9012101FA05F6721D920034
S214452840204600F016FC60B1C0E901560EE0212294
S2144528500421204600F00DFC636AF060DB68002B1F
